:0200000480007A
:100000006F0000091300000013000000130000003F
:100010001300000013000000130000001300000094
:10002000732E2034631E0E00130FC0FFF32E103406
:10003000B3FEEE01938E4E0073901E346F00C0012C
:10004000B70E0080337FDE0163180F00F32E1034EB
:10005000938E4E0073901E34B70E0080938E3E0038
:100060006396CE01930E800073B04E34B70E0080BD
:10007000938E7E006394CE0173504030B70E0080A3
:10008000938EBE006394CE017350403073002030D5
:10009000130E100073000000130E20009302800066
:1000A00073A002309302800073904230930280006C
:1000B00073A042341300000013000000130000007E
:1000C00013000000130000001300000013000000E4
:1000D00013000000130000001300000013000000D4
:1000E00013000000130E300093020008739042309A
:1000F00013000000130000001300000013000000B4
:10010000130000001300000013000000130E400055
:10011000B7120000938202807390423013000000F7
:100120001300000013000000130000001300000083
:100130001300000013000000130E5000B70110F070
:10014000938101F403A2010083A241001302F23F54
:1001500023A4410023A65100130E600013020008DF
:1001600073104230130E700073005010130E800095
:100170009301100023A04100130E90002390410032
:10018000130EA00003A20100130EB00003920100A1
:10019000130EC000130ED000832000006F0020005B
:1001A00083200000130EE00073002020130EF000E7
:1001B000B70010F0938000F603A10000130E0001B9
:0C01C00023A02000130E10016780000037
:1001D0001305000067800000130500006780000021
:1001E00013050000678000006FF09FFE13050000FC
:1001F000678000001305000067800000B70710F05B
:1002000023A0A7F067800000130101FF23248100D1
:10021000232611001304050003450500630A0500A9
:1002200013041400EFF09FFD03450400E31A05FEDC
:100230008320C100032481001301010167800000B5
:10024000130101FF23202101232611002324810013
:100250002322910013090600630E06001384050093
:10026000B384C5000345040013041400EFF01FF924
:10027000E39A84FE8320C100032481001305090052
:10028000832441000329010013010101678000005C
:100290006780000037050180130101FF1305856F9A
:1002A00023261100EF00C0058320C100B70710F01E
:1002B00023A007F21305000013010101678000006D
:1002C000130101FC2324C1022326D1022328E102C9
:1002D000232AF102232C0103232E11031386050088
:1002E0008325850093068102232E11002326D10049
:1002F000EF0040068320C101130101046780000064
:10030000130101FC2324C1022326D102232AF10276
:100310002322B1022328E102232C0103232E1103FF
:1003200097270100938707BE83A707009306410222
:100330001306050083A5870013850700232E1100EF
:100340002326D100EF0000018320C1011301010425
:1003500067800000130101E32326111C2322911C56
:100360002320211D232E311B232A511B1389050015
:1003700093040600938A06002324811C232C411B2E
:100380002328611B2326711B2324811B2322911BFD
:100390002320A11B232EB11993090500EF40104023
:1003A00083270500138507002324F102EF60502204
:1003B000232AA1002328010C232A010C232C010C41
:1003C000232E010C638A090083A789036396070023
:1003D00013850900EF20C04F8317C9001397270129
:1003E00063420702B726000003274906B3E7D70098
:1003F0002316F900B7E7FFFF9387F7FFB377F700FE
:100400002322F9068357C90093F78700638E0706F6
:1004100083270901638A07068357C9001307A000D1
:1004200093F7A7016390E7088317E90063CC0706F9
:1004300093860A00138604009305090013850900BA
:10044000EF10906E232CA1008320C11C0324811C7B
:10045000032581018324411C0329011C8329C11B1D
:10046000032A811B832A411B032B011B832BC11AE7
:10047000032C811A832C411A032D011A832DC119D3
:100480001301011D67800000930509001385090011
:10049000EF105075E30205F89307F0FF232CF100ED
:1004A0006FF09FFA9308C10E2322110D2326010C31
:1004B0002324010C130A0000232A0102232801022D
:1004C000232401002322010223260102232C010000
:1004D0001384040013075002834704006384070059
:1004E0006392E70C330B9440630A0B048327C10C1F
:1004F00023A0980023A26801B38767012326F10C8B
:100500008327810C13077000938888009387170056
:100510002324F10C635EF7001306410C93050900D8
:1005200013850900EF80D0066318054E9308C10EAD
:1005300083278101B3876701232CF10083470400DF
:10054000639407006F10905A930714002328F1005A
:10055000A303010A130BF0FF232E01001304000074
:10056000930B90009306A0051306A00283270101B8
:1005700003CD0700938717002328F10093070DFE92
:1005800063F4F6006F10C026170701001307C717A2
:1005900093972700B387E70083A70700B387E70097
:1005A00067800700130414006FF01FF39707010022
:1005B00093878730232AF10293770402639407001C
:1005C0006F10C004938A7A0093FA8AFF83AC0A0002
:1005D00003AC4A0093878A002326F1009377140026
:1005E000638E0700B3E78C01638A0700930700035B
:1005F0002304F10AA304A10B136424001374F4BFB1
:10060000930720006F001041138509002322110178
:10061000EF40D01883274500138507002326F102F9
:10062000EF60007B2322A10213850900EF40101721
:1006300083278500832841002324F100832741027A
:10064000E38207F283278100E38E07F083C7070068
:10065000E38A07F0136404406FF0DFF08347710A08
:10066000E39207F093070002A303F10A6FF09FEFF4
:10067000136414006FF01FEF83A70A00938A4A00E7
:10068000232EF100E3D007EEB307F040232EF10054
:10069000136444006FF01FED9307B0026FF0DFFCAE
:1006A0000327010183270101034D070093871700EA
:1006B0006310CD0403AB0A0013874A0063540B0098
:1006C000130BF0FF930A07002328F1006FF09FE956
:1006D0009305A0003303BB029387170003CDF7FFF8
:1006E000330BE30013070DFDE3F4EBFE6FF0DFE8DF
:1006F000130B00006FF01FFF136404086FF09FE6F8
:1007000083270101232E01000327C1019305A000C7
:10071000130D0DFD3307B702938717003307ED0064
:1007200003CDF7FF232EE10013070DFDE3FEEBFCE5
:100730006FF09FE4136484006FF0DFE28327010110
:1007400003C7070093078006631CF7008327010196
:1007500013640420938717002328F1006FF09FE0B3
:10076000136404046FF01FE08327010103C707002F
:100770009307C006631CF7008327010193871700C6
:100780002328F100136404026FF0DFDD1364040119
:100790006FF05FDD93874A002326F10083A70A00EC
:1007A000A303010A2306F11223220100130B1000F8
:1007B000930A0000130C0000930B0000930C000040
:1007C0009304C1126F0090351364040193770402FF
:1007D000638E0704938A7A0093FA8AFF83AC0A0037
:1007E00003AC4A0093878A002326F100635E0C0065
:1007F000B30C9041B3379001330C8041330CFC4073
:100800009307D002A303F10A9307F0FFE31EFB62F4
:10081000E3100C6C93079000E3EC976B938C0C0344
:10082000A30791199304F1186F00106893874A0089
:100830002326F100937704016388070083AC0A0044
:1008400013DCFC416FF09FFA9377040483AC0A0039
:1008500063880700939C0C0193DC0C416FF05FFEF2
:1008600093770420E38E07FC939C8C0193DC8C41EE
:100870006FF01FFD937784006382070C93874A0013
:100880002326F10083A70A0003A6070083A64700DA
:1008900003A7870083A7C7002328C10C232AD10CF4
:1008A000232CE10C232EF10C1305010D2322110141
:1008B000EF4000682326A10A930720008328410007
:1008C0006314F50C8327010D930501081305010935
:1008D0002328F1088327410D232001082322010842
:1008E000232AF1088327810D2324010823260108E8
:1008F000232CF1088327C10D232EF108EFC0903C73
:1009000083284100635605009307D002A303F10A30
:100910009307700497040100938404F863C6A70149
:1009200097040100938404F71374F4F72322010061
:10093000130B3000930A00006F001058938A7A005E
:1009400093FA8AFF83A50A0003A64A0093878A00C8
:1009500013050109232211012326F100EFF0C04AFB
:1009600083270109832841002328F10C83274109AB
:10097000232AF10C83278109232CF10C8327C10939
:10098000232EF10C6FF05FF2930710006318F5024D
:100990008327C10D63D607009307D002A303F10A92
:1009A0009307700497040100938484EFE3CEA7F7C4
:1009B00097040100938484EE6FF01FF7937BFDFD95
:1009C000930710046392FB06930700032304F10AC4
:1009D00013071006930780056314ED009307800743
:1009E000A304F10A930730061364240063D8674B0D
:1009F00093051B001385090023221101EF40D00548
:100A000093040500832841006310054A8357C900F9
:100A100093E707042316F9008357C90093F70704E7
:100A2000E38407A26FF05FA79307F0FF6302FB4820
:100A300093077004232201006394FB0063000B48BA
:100A4000032AC10D936704102320F102232C010215
:100A5000032E010D832D410D832C810D635A0A0055
:100A6000B707008033CA47019307D002232CF10255
:100A7000930710046398FB4813050109232411050B
:100A80002328C109232C9109232AB109232E4109C6
:100A9000EFF0C0591306C10AEF50506D13860500E0
:100AA0009305050013050109EFF0003683270109BE
:100AB00013060106930501072328F1068327410940
:100AC0001305010823200106232AF1068327810943
:100AD0002322010623240106232CF1068327C109C2
:100AE000232EF106B707FC3F2326F106EFC0903313
:100AF000032801080326410883268108832CC108A6
:100B00009305010813050109232801092322010582
:100B1000232AC1082320C104232CD108232ED1026B
:100B2000232E9109232001082322010823240108F0
:100B300023260108EFC040768326C1030326010463
:100B4000032841048328810463160500130710005D
:100B50002326E10A13071006970A0100938ACAD5D3
:100B60006316ED00970A0100938ACAD3130EFBFFA8
:100B7000938D0400B7070340930501082322C108A1
:100B80001305010913060107232411052322C105BA
:100B900023200109232EF1062324D10823269109BD
:100BA00023280106232A0106232C0106EFC09027E3
:100BB0000326010983264109130501092320C104E5
:100BC000232ED102EFE0107693050500130A0500ED
:100BD00013050109832C8109032CC109EFF0C00A18
:100BE00083270109032601048326C1032320F1067C
:100BF000832741092328C106930501072322F10613
:100C00008327810913060106130501082324F10631
:100C10008327C109232C9107232E81072326F10660
:100C2000232AD106EFD01024B3854A0183C50500DD
:100C3000032E4104032CC108938D1D00832201085B
:100C4000832F4108032F8108232EC103A38FBDFEEC
:100C50009307F0FF930C0C0083288104630CFE06BD
:100C6000130EFEFF9305010813050109232EE1056C
:100C7000232CF105232A5104232811052326C1051D
:100C80002328510823245104232AF1092322F105A2
:100C9000232CE1092320E105232E810923200108CB
:100CA000232201082324010823260108EFC0C05E87
:100CB000832601040326410403288104032EC10472
:100CC0008328010583224105832F8105032FC10558
:100CD000E31205EAB70CFE3F93050108130501096D
:100CE000232011052328510823265104232AF10922
:100CF0002324F105232CE1092322E105232E810978
:100D00002320010823220108232401082326910916
:100D1000EFC04065832801046346A0048322C10418
:100D2000832F8104032F4104930501081305010952
:100D300023285108232AF109232CE109232E8109B4
:100D400023200108232201082324010823269109D6
:100D5000EFC0805483280104631C0518137A1A001D
:100D600063080A1803C6FA00232EB10B930500038B
:100D70008326C10B9387F6FF232EF10A83C7F6FF64
:100D80006384C714130690036394C71483C7AA002F
:100D9000A38FF6FE138A0D0013077004330A9A40DE
:100DA000832CC10A6392EB2A1307D0FF63C4EC00C3
:100DB000635E9B31130DEDFF1387FCFF2326E10AD1
:100DC0001376FDFD130510049376FD0F93050000C7
:100DD0006318A6009386F60093F6F60F93051000AD
:100DE000230AD10A9307B0026358070013071000C3
:100DF000330797419307D002A30AF10A93079000A3
:100E000063D8E7289307310C9385070013059000FA
:100E10001308A000B36607031386F7FF33470703E1
:100E200093860603A38FD7FE6346E52413070703C3
:100E30009387E7FFA30FE6FE9306610B63E0B724F9
:100E40009307410BB387F6402328F102338B470108
:100E50009307100063C64701937714006386070069
:100E600083274101330BFB001374F4BF9367041015
:100E70002320F102130C0000930B0000930C0000E0
:100E800083278103638607001307D002A303E10AC7
:100E900003240102930A00006F004048232201004E
:100EA0009304C1126FF0DFB92322A1006FF05FB984
:100EB00023220100130B60006FF09FB82322610111
:100EC000130B10006FF0DFB7A38FB6FE6FF05FEA71
:100ED0009387170093F7F70F6FF09FEB130A1A0031
:100EE000A30FEAFEB3074C41E3DA07FE6FF0DFEA37
:100EF0008327C103138A0D0013070003338CFD0001
:100F00006FF05FFE93076004638EFB00930750044D
:100F1000930A1B006384FB00930A0B001306200056
:100F20006F00C000930A0B00130630009307010BFB
:100F30001308C10B1307C10A93860A009305010920
:100F400013850900232011052328C109232EC1037D
:100F5000232AB109232C9109232E4109EF3040396E
:100F60009307700493040500032EC1038328010432
:100F70006396FB00937714006388070A9307600465
:100F8000338C54016392FB0603C7040093070003EC
:100F90006318F704930501081305010923201105BF
:100FA0002328C109232EC103232AB109232C910927
:100FB000232E4109232001082322010823240108AC
:100FC00023260108EFC0402D032EC103832801040E
:100FD0006308050093071000B38A57412326510B7D
:100FE0008327C10A330CFC0093050108130501098E
:100FF000232E11032328C109232AB109232C910987
:10100000232E41092320010823220108232401085B
:1010100023260108EFC040288328C10313070003DB
:10102000631E0500232E810B032AC10B6FF0DFD650
:1010300093861700232ED10A2380E7008327C10B54
:10104000E3E887FF6FF05FFE13076004E396EBD6DB
:101050006352900763160B00137714006302070CAA
:10106000832741013387FC00330BEB00130D60062F
:101070006F004009930706006FF09FD99387170010
:1010800003C7F7FF93861600A38FE6FE6FF01FDB02
:101090009307610B6398050093070003230BF10A84
:1010A0009307710B13070703938617002380E7004C
:1010B0006FF01FD963160B00137714006306070641
:1010C00083274101138717006FF01FFA63C04C0399
:1010D00013771400138B0C0063060700832741016C
:1010E000338BFC00130D70066F00C0018327410194
:1010F000130D7006330BFA006346900133039B41D6
:10110000130B1300937B0440130C0000E38A0BD6EF
:10111000930B0000E35690D79306F00F6F00800307
:10112000138B0C006FF09FF4130D6006130B10006F
:101130006FF05FFD6356970383278100B38CEC400B
:1011400003C717006308070293871700938B1B00E0
:101150002324F1008327810003C70700E31CD7FC89
:101160008327410233878B013307F702330B670173
:101170006FF01FD1130C1C006FF0DFFD13874A00C6
:101180002326E1001377040283A70A006300070205
:101190000327810123A0E7001357F74123A2E700AB
:1011A000832AC100832401016FF08FB213770401F9
:1011B000630807000327810123A0E7006FF05FFEAB
:1011C0001377040463080700035781012390E700A5
:1011D0006FF01FFD13740420E30E04FC034781012C
:1011E0002380E7006FF0DFFB1364040193770402B0
:1011F00063880704938A7A0093FA8AFF83AC0A0013
:1012000003AC4A0093878A002326F1001374F4BFCD
:1012100093070000A303010A1307F0FF630CEB42DE
:1012200013070400B3E68C011374F4F763940642C9
:1012300063020B5A130710006392E7426FF00FDE50
:1012400093874A002326F100937704016386070001
:1012500083AC0A006F0000019377040463880700E1
:1012600083DC0A00130C00006FF05FFA9377042010
:10127000E38007FE83CC0A006FF0DFFE93874A000D
:101280002326F100B787FFFF93C707832314F10AD2
:1012900097F7000093870761232AF10283AC0A00C5
:1012A000130C00001364240093072000130D800723
:1012B0006FF05FF693874A002326F100A303010A2B
:1012C0009307F0FF2320110383A40A006306FB02A7
:1012D00013060B009305000013850400EF40406ADD
:1012E0002322A10083280102630605E4330B954005
:1012F000232201006FF00FE413850400EF50502DFE
:1013000083280102130B050023220100930A000029
:10131000130C0000930B0000930C000023205103DA
:1013200063D46A01232061030347710A630807003D
:1013300083270102938717002320F102937D240065
:1013400063880D0083270102938727002320F10281
:1013500093774408232CF102639807068327C10181
:10136000032701023387E7406350E006930E000134
:1013700017FE0000130E0E50130F70008326810C11
:1013800023A0C8010326C10C93861600938588000C
:1013900063CAEE4623A2E8003307C7002326E10C08
:1013A0002324D10C1307700093880500635ED700D7
:1013B0001306410C9305090013850900EF70501DB9
:1013C000E314056C9308C10E0347710A6308070410
:1013D0001307710A23A0E8001307100023A2E800F6
:1013E0000327C10C93067000938888001307170029
:1013F0002326E10C0327810C130717002324E10C9B
:1014000063DEE6001306410C93050900138509000D
:10141000EF701018E31A05669308C10E63880D0477
:101420001307810A23A0E8001307200023A2E80085
:101430000327C10C930670009388880013072700C8
:101440002326E10C0327810C130717002324E10C4A
:1014500063DEE6001306410C9305090013850900BD
:10146000EF701013E31205629308C10E8327810306
:10147000130700086398E7068327C10103270102C9
:10148000B38DE7406350B007130E000197F70000DB
:101490009387473F930E70000327810C23A0F80029
:1014A0008326C10C13071700138688006348BE3BD0
:1014B00023A2B801B38DDD002326B10D2324E10C56
:1014C000930670009308060063DEE6001306410CE5
:1014D0009305090013850900EF70900BE316055A78
:1014E0009308C10EB38A6A41635050071308000184
:1014F00097FD0000938D0D39130E70000327810CAA
:1015000023A0B8018326C10C130717001386880097
:10151000634E583923A25801B38ADA002326510DAD
:101520002324E10C930670009308060063DEE600B6
:101530001306410C9305090013850900EF7050054F
:10154000E31405549308C10E13770410832DC10CC6
:101550006312073A3303BB0123A0980023A268015A
:101560002326610C8327810C130770009388880061
:10157000938717002324F10C6352F74C1306410C98
:101580009305090013850900EF709000E31E054ED6
:101590009308C10E6F00804A13640401937704021C
:1015A00063820702938A7A0093FA8AFF83AC0A0067
:1015B00003AC4A0093878A002326F10093071000AA
:1015C0006FF05FC593874A002326F10093770401EB
:1015D0006386070083AC0A006F0000019377040460
:1015E0006388070083DC0A00130C00006FF01FFD06
:1015F00093770420E38007FE83CC0A006FF0DFFEC0
:1016000097F700009387072A6FE0DFFA93874A0075
:101610002326F100937704016386070083AC0A0058
:101620006F000001937704046388070083DC0A00DD
:10163000130C00006FE09FFA93770420E38007FE0D
:1016400083CC0A006FF0DFFE13070400930710003D
:101650006FF05FBD13071000638CE79A130720003B
:10166000638EE712930701199316DC0113F77C00D0
:1016700093DC3C0013070703B3EC9601135C3C00BA
:10168000A38FE7FEB3E68C019384F7FF639E060207
:1016900093761400638A0600930600036306D7005E
:1016A000A38FD4FE9384E7FF93070119930A0B00DD
:1016B00023220100338B9740130C0000930B000092
:1016C000930C00006FF09FC5938704006FF0DFF963
:1016D000130A0000930D0119937A0440930B9000B4
:1016E0001306A0009306000013850C0093050C0060
:1016F00023221101EFA0902D13050503A38FADFE4A
:101700009384FDFF130A1A0083284100638E0A04A4
:101710008327810083C707006318FA049307F00F3B
:101720006304FA0463140C0063F09B0583274102F1
:101730008325C10223221101B384F44013860700DC
:1017400013850400EF50806A83278100130A00008C
:101750008328410083C7170063880700832781001F
:10176000938717002324F10013850C0093050C00C8
:101770001306A0009306000023221101EFA0C06110
:10178000138C0500B3E5A500930C050083284100E8
:10179000E38C05F0938D04006FF09FF4930401191E
:1017A0000327410393F7FC009384F4FFB307F7008A
:1017B00083C7070093DC4C002380F4009317CC010F
:1017C000B3EC9701135C4C00B3E78C01E39A07FC80
:1017D0006FF09FED93040119E39807EC137717005E
:1017E000E30407EC93070003A307F1186FF08F835E
:1017F000E30E0D2E2306A113A303010A2326510194
:101800006FE09FFA1306060123A2D8012326C10C1C
:101810002324D10C635EDF021306410C93050900FB
:10182000138509002324E1052322C1052320D105C6
:10183000232EE102EF70C055E3180524032F810425
:10184000032E4104832E01040327C1039305C10E17
:10185000130707FF938805006FF05FB293860601B8
:1018600023A2C8012326D10C2324E10C63DAEE0263
:101870001306410C93050900138509002320D105A7
:10188000232EF102232CC103EF708050E31E051EAE
:10189000832E01048327C103032E81031306C10E87
:1018A000938D0DFF930806006FF01FBF938606010E
:1018B00023A208012326D10C2324E10C6356EE0257
:1018C0001306410C9305090013850900232EC1035B
:1018D000232C0103EF70C04BE318051A032EC1033C
:1018E000032881031306C10E938A0AFF930806009A
:1018F0006FF0DFC0130750066354A7730327010D71
:1019000093050108130501092328E1080327410D68
:10191000232C110323200108232AE1080327810D2A
:101920002322010823240108232CE1080327C10DE9
:1019300023260108232EE108EFB010168328810327
:101940006314051897F70000938747F823A0F80061
:101950009307100023A2F8008327810C938D1D00AC
:101960002326B10D938717002324F10C1307700071
:1019700093888800635EF7001306410C9305090005
:1019800013850900EF70C040E31005109308C10EE5
:101990008327C10A63C64701937714006380070A4F
:1019A00083278102032741019388880023ACF8FE36
:1019B0008327410123AEF8FE8327C10CB387E700DC
:1019C0002326F10C8327810C1307700093871700DF
:1019D0002324F10C635EF7001306410C9305090004
:1019E00013850900EF70C03AE310050A9308C10E91
:1019F0009304FAFF63549004930B000197FA0000DC
:101A0000938A4AE8130C70008327810C23A05801A5
:101A10000327C10C938717009386880063CA9B062F
:101A200023A29800B384E4002326910C2324F10C14
:101A30001307700093880600E342F7B41374440060
:101A40006314047E032DC101832701026354FD004A
:101A5000138D070083278101B387A701232CF10091
:101A60008327C10C638C07001306410C9305090002
:101A700013850900EF70C031E3180500832741008A
:101A80002324010CE39C07049308C10E6FF04FF16F
:101A90001307070123A278012326E10C2324F10C6C
:101AA000635EFC001306410C9305090013850900D1
:101AB000EF70002E631A057C9306C10E938404FF19
:101AC000938806006FF05FF40327C10A6346E016AF
:101AD00097F70000938787DF23A0F8009307100093
:101AE00023A2F8008327810C938D1D002326B10DBE
:101AF000938717002324F10C130770009388880044
:101B0000635EF7001306410C930509001385090075
:101B1000EF700028631A05769308C10E8327C10A67
:101B20006398070063160A0093771400E38807F0B0
:101B300083278102032741019388880023ACF8FEA4
:101B40008327410123AEF8FE8327C10CB387E7004A
:101B50002326F10C8327810C13077000938717004D
:101B60002324F10C635EF7001306410C9305090072
:101B700013850900EF70C021631805709308C10E2A
:101B8000832AC10A63D20A06B30A504113870800A8
:101B9000130C000197FB0000938BCBCE130D70004C
:101BA0008327810C232077018326C10C938717009C
:101BB0009388880063465C0523225701B38ADA00C4
:101BC0002326510D2324F10C13077000635EF700E8
:101BD0001306410C9305090013850900EF70401BA3
:101BE0006314056A9308C10E8327C10C23A09800D3
:101BF00023A24801B38747012326F10C6FF09F967B
:101C000093860601232287012326D10C2324F10C7D
:101C1000635EFD001306410C93050900138509005E
:101C2000EF700017631205669308C10E938A0AFFCE
:101C3000138708006FF0DFF6938A0C0063549A0153
:101C4000930A0A00635250050327810CB38DBA0131
:101C500023A098001307170023A258012326B10DD3
:101C60002324E10C930670009388880063DEE6006D
:101C70001306410C9305090013850900EF7040110C
:101C8000631405609308C10E63D40A00930A000030
:101C9000B38A5C4163505007930D000117FD0000AB
:101CA000130D4DBE130B70000327810C23A0A80158
:101CB0008326C10C130717001386880063C25D1BBF
:101CC00023A25801B38ADA002326510D2324E10C04
:101CD000930670009308060063DEE6001306410CCD
:101CE0009305090013850900EF70800A631E0558EB
:101CF0009308C10E93770440B38A9401638407026A
:101D0000130D7000338B440197FD0000938D8DB748
:101D100063940B1863140C18B387440163F45701E0
:101D2000938A07008327C10A63C64701937714008B
:101D3000638A07048327810203274101938888006F
:101D400023ACF8FE8327410123AEF8FE8327C10CA4
:101D5000B387E7002326F10C8327810C130770005B
:101D6000938717002324F10C635EF7001306410CE0
:101D70009305090013850900EF7080016316055073
:101D80009308C10EB3844401B38754418324C10A2C
:101D9000B3049A4063D4970093840700635490047B
:101DA0008327C10C23A0580123A29800B387F40015
:101DB0002326F10C8327810C130770009388880079
:101DC000938717002324F10C635EF7001306410C80
:101DD0009305090013850900EF60907B6316054A9F
:101DE0009308C10E9387040063D404009307000096
:101DF0008324C10AB3049A40B384F440E35090C4EE
:101E0000930B000197FA0000938ACAA7130C700085
:101E10008327810C23A058010327C10C9387170047
:101E200093868800E3DE9BBE1307070123A2780197
:101E30002326E10C2324F10C635EFC001306410C05
:101E40009305090013850900EF609074631E054235
:101E50009306C10E938404FF938806006FF05FFB26
:101E60009386060123A2B8012326D10C2324E10C7A
:101E7000635EEB001306410C93050900138509000E
:101E8000EF601071631205401306C10E938A0AFFBA
:101E9000930806006FF05FE163020C0E130CFCFF69
:101EA0008327C102032741029388880023ACF8FEF0
:101EB0008327410223AEF8FE8327C10CB387E700D6
:101EC0002326F10C8327810C938717002324F10C20
:101ED000635EFD001306410C93050900138509009C
:101EE000EF60106B6312053A9308C10E83278100DF
:101EF00033075B4183C707006354F700930707006C
:101F00006356F0040327C10C23A0580123A2F80054
:101F10003387E7002326E10C0327810C9388880090
:101F2000130717002324E10C6352ED021306410C42
:101F30009305090013850900232CF102EF60506519
:101F400063140534832781039308C10E13870700A8
:101F500063D40700130700008327810013080001E2
:101F600083C70700B387E7406346F00683278100F5
:101F700083C70700B38AFA006FF09FD983278100D7
:101F8000938BFBFF9387F7FF2324F1006FF05FF142
:101F90009386060123A208012326D10C2324E10CF9
:101FA0006356ED021306410C9305090013850900E1
:101FB000232E0103232CF102EF60905D6316052CA4
:101FC0000328C103832781031306C10E938707FFEC
:101FD000930806000327810C23A0B8018326C10CB7
:101FE0001307170013868800E344F8FA23A2F800C9
:101FF000B387D7002326F10C2324E10C93080600B5
:10200000E356EDF61306410C93050900138509000C
:10201000EF601058631A05269308C10E6FF01FF584
:102020008327810C1307100023A09800938D1D00B7
:1020300093871700938B88006346470193761400BB
:102040006388061C1307100023A2E8002326B10DA5
:102050002324F10C13077000635EF7001306410C94
:102060009305090013850900EF609052631E052057
:10207000930BC10E8327810203274101938B8B00B1
:1020800023ACFBFE8327410123AEFBFE8327C10C5B
:10209000B387E7002326F10C8327810C1307700018
:1020A000938717002324F10C635EF7001306410C9D
:1020B0009305090013850900EF60904D6316051C18
:1020C000930BC10E8327010D930501081305010928
:1020D0002328F1088327410D930AFAFF23200108E2
:1020E000232AF1088327810D2322010823240108D4
:1020F000232CF1088327C10D23260108232EF10884
:10210000EFB08019630605088327C10C0327810CF3
:10211000938414009387F7FFB387470113071700D1
:1021200023A09B0023A25B012326F10C2324E10CB6
:1021300093077000938B8B0063DEE7001306410C5E
:102140009305090013850900EF609044631E051292
:10215000930BC10E9307410B23A0FB0083270103C0
:102160000327010393888B0023A2FB008327C10C64
:10217000B387E7002326F10C8327810C1307700037
:10218000938717002324F10CE35AF78A6FF00FBFEF
:10219000E35250FD130C000197E400009384846E19
:1021A000130D70000327810C23A09B008327C10C13
:1021B0001307170093868B0063405C03B387FA0014
:1021C00023A25B012326F10C2324E10C930770006A
:1021D000938B06006FF05FF69387070123A28B01B4
:1021E0002326F10C2324E10C635EED001306410C61
:1021F0009305090013850900EF60903963160508FF
:102200009306C10E938A0AFF938B06006FF09FF925
:1022100023A2E8002326B10D2324F10C130770003C
:10222000E35AF7F26FF09FF18327C1010327010200
:102230003384E740E3588080930A000197E400006C
:1022400093844463930B70008327810C23A0980030
:102250000327C10C9387170063C68A0423A2880052
:102260003304E4002326810C2324F10C13077000AF
:10227000635AF7FC1306410C930509001385090006
:10228000EF601031630005FC832741006394070071
:102290006FE08FF89385070013850900EF00101198
:1022A0006FE08FF71307070123A258012326E10CE3
:1022B0002324F10C9388880063DEFB001306410C95
:1022C0009305090013850900EF60902CE31E05FAC1
:1022D0009308C10E130404FF6FF01FF7832541001C
:1022E00013850900EF00900C6FF00FFA8327C10CE3
:1022F000639407006FE04FF21306410C9305090049
:1023000013850900EF60D0286FE00FF197070100F7
:10231000938747BF930606001386050093050500C3
:1023200003A507006FE00F8383D7C500130101B831
:10233000232C814693F7D7FF231AF10083A7450684
:1023400013840500232A91462326F10683D7E5004E
:1023500023282147232E1146231BF10083A7C50103
:1023600013090500232001022322F10283A745025D
:10237000930581002326F102930701072324F1002E
:10238000232CF100930700402328F100232EF100B5
:10239000EFD05FFC93040500634C050093058100BA
:1023A00013050900EF004038630405009304F0FFB3
:1023B0008357410193F70704638807008357C400DC
:1023C00093E707042316F4008320C14703248147C1
:1023D0001385040003290147832441471301014861
:1023E00067800000130101FF97070100938787B101
:1023F000232291009304050003A5070023248100F4
:102400002326110013840500630805008327850334
:1024100063940700EF00C04B0317C4009317070134
:1024200093D7070193F68700639E060693F607018C
:10243000639606029307900023A0F4001367070435
:102440002316E4001305F0FF8320C100032481005C
:1024500083244100130101016780000093F74700C6
:10246000638C070283250403638C0500930704042F
:102470006386F50013850400EF00407323280402EF
:102480008357C4002322040093F7B7FD2316F400FA
:10249000832704012320F4008357C40093E78700B7
:1024A0002316F40083270401639007028357C400B6
:1024B0001307002093F707286388E70093050400BB
:1024C00013850400EF20504A8357C40013F7170008
:1024D000630C07028327440123240400B307F04060
:1024E000232CF4008327040113050000E39E07F466
:1024F0008317C40013F70708E30807F493E70704FA
:102500002316F4006FF01FF493F727001307000061
:1025100063940700032744012324E4006FF09FFC29
:102520008397C500130101FE232C81001397070137
:1025300013570701232A9100232E1100232821017C
:102540002326310193768700930405001384050048
:10255000639C06163717000013070780B3E7E700F0
:1025600003A745002396F5006346E00203A7C503D1
:102570006342E002130500008320C10103248101AE
:1025800083244101032901018329C10013010102B0
:102590006780000003278402E30E07FC03A9040000
:1025A0009396370123A004008325C40163D8060C49
:1025B000032604058357C40093F74700638E070082
:1025C000832744003306F64083270403638607000D
:1025D0008327C4033306F640832784028325C4017E
:1025E0009306000013850400E78007009307F0FFBF
:1025F0008356C4006312F50283A704001307D001B9
:10260000636CF70A37074020130717003357F700AA
:10261000137717006302070AB7F7FFFF9387F77F67
:1026200003270401B3F7D7009397070193D7074116
:102630002320E4002316F40023220400139737011B
:10264000635C07009307F0FF6316F50083A704009F
:10265000639407002328A4048325040323A02401F2
:10266000E38A05F0930704046386F50013850400EC
:10267000EF00C053232804026FF0DFEF13060000C1
:102680009306100013850400E70007009307F0FF8E
:1026900013060500E310F5F283A70400E38C07F0AE
:1026A0001307D0016386E700130760016392E70612
:1026B00023A024016FF01FEC93E706042316F40017
:1026C0001305F0FF6FF05FEB83A90501E38409EACE
:1026D00003A905001377370023A0350133093941D9
:1026E000930700006314070083A745012324F40027
:1026F000E35220E9832744028325C401930609009D
:102700001386090013850400E78007006348A000D2
:102710008357C40093E707046FF05FFAB389A900F9
:102720003309A9406FF0DFFC130101FE232C810067
:10273000232E110013040500630C05008327850375
:10274000639807002326B100EF0080188325C1009D
:102750008397C500638C07001305040003248101DF
:102760008320C101130101026FF09FDB8320C101AF
:10277000032481011305000013010102678000009A
:1027800093050500631E050097F7000093874777C0
:1027900003A5070097050000938545F96F00C072F7
:1027A00097F700009387077603A507006FF0DFF720
:1027B0001305000067800000977500009385855D14
:1027C0006F008070130101FF232481002326110074
:1027D000130405002316B5002317C50023200500A8
:1027E00023220500232405002322050623280500B3
:1027F000232A0500232C0500130680009305000002
:102800001305C505EF30001A974700009387472F3F
:102810002320F40297470000938707342322F40211
:10282000974700009387873B2324F40297470000D3
:1028300093874740232E84002326F4028320C1007F
:1028400003248100130101016780000013050000CB
:1028500067800000130101FF232291001306800608
:102860009384F5FFB384C40223202101138905005A
:10287000232481002326110093854407EF20D01DD7
:10288000130405006300050223200500232225010F
:102890001305C5002324A4001386840693050000B5
:1028A000EF304010130504008320C1000324810091
:1028B0008324410003290100130101016780000006
:1028C00097F700009387C76303A507006FF0DFEE5B
:1028D00083278503639E0706130101FF232611004A
:1028E0002324810097070000938747ED232EF502EC
:1028F000930730002322F52E9307C52E13040500FD
:102900002324F52E2320052E032545001306000061
:1029100093054000EFF01FEB032584001306100021
:1029200093059000EFF01FEA0325C4001306200072
:1029300093052001EFF01FE993071000232CF40208
:102940008320C1000324810013010101678000007E
:1029500067800000130101FF97F700009387475A33
:102960002322910083A407002320210123261100A4
:1029700083A78403232481001309050063960700BD
:1029800013850400EFF0DFF49384042E03A4840085
:1029900083A744009387F7FF63DA070083A7040047
:1029A000638E070083A404006FF05FFE0317C4006A
:1029B00063040704130484066FF0DFFD93054000F1
:1029C00013050900EFF01FE923A0A400E31C05FC98
:1029D0009307C0002320F90013040000130504002E
:1029E0008320C100032481008324410003290100C6
:1029F0001301010167800000B707FFFF93871700ED
:102A0000232204062320040023220400232404009C
:102A10002326F40023280400232A0400232C040086
:102A200013068000930500001305C405EF2090777E
:102A300023280402232A0402232204042324040456
:102A40006FF0DFF96780000067800000678000009A
:102A50006780000097F700009387C74A03A5070027
:102A600097050000938505D56F00003C97F700009F
:102A70009387474903A5070097050000938545DD27
:102A80006F00803A130101FD232481022322910269
:102A900023202103232E31012326B10023261102F6
:102AA0001309050097F9000093890905EF20507D6F
:102AB00083A789008325C10083A44700B7170000BE
:102AC0001384F7FE93F4C4FF3304B440330494003A
:102AD0001354C4001304F4FF1314C4006356F40227
:102AE00013050900EF20107A130500008320C102AE
:102AF0000324810283244102032901028329C101A5
:102B0000130101036780000093050000130509000D
:102B1000EF30106183A78900B3879700E312F5FCBB
:102B2000B305804013050900EF30905F9307F0FF75
:102B30006312F5049305000013050900EF30505EA1
:102B400003A789009306F000B307E540E3DAF6F83F
:102B500097F600009386463B83A6060093E717008E
:102B60002322F7003305D54097F6000023ACA63AA0
:102B70006FF01FF783A78900B384844093E41400A7
:102B800023A2970097F700009387C73983A7070010
:102B9000130509003384874097F7000023A4873882
:102BA000EF20506E130510006FF05FF4638C052664
:102BB000130101FF23248100232291001304050047
:102BC0009384050023261100EF20906B83A5C4FF9A
:102BD000938684FF17F50000130505F293F7E5FFD0
:102BE0003386F600032746000328850093F5150079
:102BF0001377C7FF631AC806B387E700639005021F
:102C000003A784FFB386E64003A68600B387E700E8
:102C100003A7C6002326E6002324C70013E71700F6
:102C200023A2E60017F70000232CD7EC17F70000CB
:102C30001307C72D0327070063ECE70097F7000091
:102C40009387C72D83A5070013050400EFF09FE3CA
:102C500013050400032481008320C1008324410064
:102C6000130101016F2010622322E6001308000007
:102C70006396050283A584FF97F80000938848E8CF
:102C8000B386B640B387B70083A58600638C150B67
:102C900083A8C60023A6150123A4B800B305E60047
:102CA00083A5450093F51500639C0502B387E700F3
:102CB00003278600631C080897F50000938545E408
:102CC0006316B70817F600002322D6E417F60000B3
:102CD000232CD6E223A6E60023A4E6001308100066
:102CE00013E7170023A2E6003387F6002320F7003E
:102CF000E31008F61307F01F6362F70693D7370057
:102D000013D62740130710003317C70003264500CA
:102D100093871700939737003367C700B307F50011
:102D200017F60000232CE6DC03A70700138687FFB5
:102D300023A6C60023A4E60023A0D7002326D7009D
:102D40006FF01FF1130810006FF05FF50326C60047
:102D50002326C7002324E6006FF09FF813D69700C0
:102D600013074000636AC70413D76700130787037C
:102D700013061700131636003306C500930586FFA9
:102D8000032606006396C5089307100013572740D3
:102D90003397E700832745003367F70097F7000074
:102DA00023AEE7D423A6B60023A4C60023A4D500EF
:102DB0002326D6006FF0DFE9130740016366C700E2
:102DC0001307B6056FF0DFFA130740056368C70005
:102DD00013D7C7001307E7066FF09FF913074015D5
:102DE0006368C70013D7F700130777076FF05FF822
:102DF000930540551307E007E3ECC5F613D7270109
:102E00001307C7076FF0DFF6032686006388C50047
:102E1000032746001377C7FFE3E8E7FE8325C600D4
:102E20006FF05FF867800000130101FD2324810229
:102E300023202103232C4101232A5101232611029F
:102E400023229102232E31011304052E13090000C1
:102E5000130A1000930AF0FF631604028320C102D4
:102E6000032481021305090083244102032901027E
:102E70008329C101032A8101832A4101130101032E
:102E80006780000083248400832944009389F9FF2C
:102E900063D60900032404006FF01FFC83D7C4002D
:102EA0006370FA028397E400638C57011385040072
:102EB0002326B100E78005008325C1003369A900FE
:102EC000938484066FF09FFC130101FD232481028B
:102ED00023202103232C4101232A510123286101AE
:102EE000232671012326110223229102232E310170
:102EF000130A0500938A05001304052E1309000028
:102F0000130B1000930BF0FF631A04028320C1021D
:102F100003248102130509008324410203290102CD
:102F20008329C101032A8101832A4101032B010165
:102F3000832BC100130101036780000083248400F8
:102F4000832944009389F9FF63D609000324040010
:102F50006FF09FFB83D7C400637EFB008397E40080
:102F6000638A77019385040013050A00E7800A004D
:102F70003369A900938484066FF0DFFC9307450151
:102F800013052500231F05FEE31CF5FE67800000E6
:102F900093074501130525000357E5FF9385250099
:102FA000239FE5FEE398A7FE678000009307A50135
:102FB00013052500231F05FEE31CF5FE67800000B6
:102FC0001307850193870500130525008356E5FF48
:102FD00093872700239FD7FEE318A7FE239C0500B5
:102FE0006780000093074500938545001305A50100
:102FF000938727009385250083D6E7FF03D7E5FF56
:103000006398E600E316F5FE1305000067800000F4
:10301000130510006364D7001305F0FF67800000FC
:1030200093064500930700001305A5013786FFFFAF
:1030300003D70600937517006384050093E7170014
:1030400093F5270013571700639005029397170015
:103050002390E600939707019386260093D70701F4
:10306000E318D5FC678000003367C7006FF01FFED0
:10307000930665011307000083D726001396070106
:103080001356064163540600136717009397170001
:10309000939707011376270093D707016310060261
:1030A000131717002391F600131707019386E6FF05
:1030B00013570701E312D5FC6780000093E7170060
:1030C0006FF01FFE93074500130700001305A501CD
:1030D00083D607009387270013D686003367C7007F
:1030E000239FE7FE13978600131707011357070165
:1030F000E310F5FE678000009307650113070000E9
:1031000083D627009387E7FF139686003367C700AF
:103110002392E70013D78600E314F5FE67800000D2
:1031200093074500130785019387270083D607007F
:10313000239FD7FEE31AF7FE231C050067800000DB
:10314000930785011307A501930645009387E7FFC1
:1031500003D607001307E7FF2310C700E398F6FE26
:103160002312050067800000938585011307650120
:10317000930600008357270003D605001307E7FFD7
:103180009385E5FFB387C700B387D7002391F50088
:1031900093D7070193F61700E31EE5FC6780000054
:1031A00093858501130765019306000083D7050009
:1031B000035627001307E7FF9385E5FFB387C74052
:1031C000B387D7402391F50093D7070193F61700F3
:1031D000E31EE5FC67800000130101FE37030100D8
:1031E00093888501231D0100231E0100938545005E
:1031F0009306C1011303F3FF03D708009386E6FF8C
:103200009388E8FF631C0702239F06FEE39615FFE1
:10321000930740001307A00193054100B385F50013
:1032200083D50500B306F600938727002390B600E8
:10323000E394E7FE13010102678000003307A70251
:1032400003D82600B3776700B387070113D80701B7
:103250002391F6009357070103D70600B387E700D1
:10326000B38707012390F60093D70701239FF6FE4B
:103270006FF0DFF98357250193C7F7FF1397170105
:10328000631C070093072501130525000357E5FF7D
:1032900063180700E39AA7FE13050000678000008B
:1032A0001305100067800000130101FF2324810033
:1032B0002326110013040500EFF0DFFB631E050059
:1032C000031524011355F5018320C1000324810057
:1032D0001301010167800000130500006FF0DFFE9D
:1032E00083172501130101FF2326110023248100E8
:1032F000232291002320210163D807069307F0FFC2
:103300002390F50003572501B78700009387F7FF47
:1033100033F7E7002391E500130905016316F7066B
:103320001384050093040500EFF0DFF46302050445
:1033300093076400231204001385C4FF1309E9FFF7
:103340000357290093872700239FE7FEE318A9FE70
:103350008320C1000324810083244100032901004C
:103360001301010167800000239005006FF09FF9B1
:10337000930744009305A40193872700239F07FE2A
:10338000E39CB7FE6FF0DFFC938765002392050096
:103390001305E5FF1309E9FF035729009387270069
:1033A000239FE7FEE318A9FE239C05006FF05FFA58
:1033B000130101FB2322910423202105232611045C
:1033C000232481041309050093840500EFF09FEA8C
:1033D0006310050E13850400EFF0DFE91304050008
:1033E0006318050C9305810013050900EFF05FEFEA
:1033F0009305410213850400EFF09FEE035781000F
:10340000835741026380E7069307200093068001FB
:10341000130681003306F60003560600631C0602FD
:10342000130641023306F600035606006314060233
:1034300093872700E39ED7FC130504008320C10473
:103440000324810483244104032901041301010599
:103450006780000013041000E30007FE1304F0FF70
:103460006FF09FFD13061000638407001306F0FF42
:103470009307000093058001130781003307F700CD
:1034800083560700130741023307F700035707006D
:103490006398E60093872700E390B7FE6FF0DFF9AB
:1034A00013040600E36AD7F83304C0406FF0DFF876
:1034B0001304E0FF6FF05FF88357250193C7F7FF10
:1034C0001397170163100702130101FF2326110050
:1034D000EFF05FDA8320C1001335150013010101FD
:1034E0006780000013050000678000009307250136
:1034F00013052500231F05FEE31CF5FE8357050079
:10350000378700001307F7FFB3E7E7002310F50044
:1035100067800000130101FE232C81002326310166
:10352000232E1100232A9100232821012324410165
:1035300023225101930905001384050063D205106D
:103540003309B040130A090093040000930AF00005
:1035500063CE4A0313594900930500FFB305B9022E
:10356000130A70003384854013090400634C2A0356
:1035700093553400930780FFB385F50233848500AB
:10358000631E0402333590006F00400983D7890120
:1035900013850900130A0AFFB3E4F400EFF05FBAE1
:1035A0006FF01FFB83C7890113850900130989FF89
:1035B000B3E49700EFF01FB16FF05FFB83D7890191
:1035C000138509001304F4FF93F71700B3E4970081
:1035D000EFF01FA56FF0DFFA13850900EFF05FB47D
:1035E000938404FFE34A99FE93554400930700FF38
:1035F000B385F502130970003304B400930404008A
:103600006346990493553400930780FFB385F50210
:103610003304B40063140404130500008320C101C3
:103620000324810183244101032901018329C1006D
:10363000032A8100832A41001301010267800000F0
:10364000938405001309F0006FF0DFF9138509007A
:10365000EFF09FAA938484FF6FF09FFA138509000F
:10366000EFF01FA11304F4FF6FF0DFFA835745005A
:10367000130101FF2322910023261100232481003E
:103680002320210193040500639207088317650036
:10369000130400001309000A63D80702130504008D
:1036A0008320C100032481008324410003290100F9
:1036B0001301010167800000138504001304040155
:1036C000EFF01FA6E30C24FD83D76400E38607FE1A
:1036D00083D7640093F707F0638207021309000A97
:1036E00083976400E3CC07FA1385040013041400E5
:1036F000EFF01F98E35689FE6FF05FFA1385040020
:10370000EFF09F9F130484006FF09FFC93F707F086
:103710001304000063860700EFF0DF9A130480FFB4
:10372000130900F76F004001138504001304F4FF30
:10373000EFF01F8FE34424F783D74400E39607FE9E
:103740006FF0DFF59307050113052500231F05FE24
:10375000E31CF5FEB7C7FFFF2310F500B787FFFF97
:1037600093C7F7FF2311F5006780000013070500DA
:1037700083560700138505008357270063860600DC
:10378000B786FFFFB3E7D7002319F50003562700DC
:10379000B78600009386F6FF93076700631ED60086
:1037A0001307A70183D607006398060293872700B3
:1037B000E39AE7FE6FF09FD3130505011307870116
:1037C0009387270083D6E7FF1305E5FF2311D50074
:1037D000E398E7FE678000006FF0DFF6130101FD5C
:1037E0002322910293040500130541002324810242
:1037F0002326110213840500EFF04FFB03D7E400EA
:103800009317070193D7074163C2070423120100EE
:10381000B78600009386F6FF3377D7009387E400DE
:10382000631CD706138704008356070063860602CD
:1038300013050400EFF01FF18320C102032481026D
:103840008324410213010103678000009307F0FF06
:103850002312F1006FF0DFFB13072700E396E7FC6C
:1038600013050400EFF08FF113050400EFF01FC8FB
:103870008397E400E3D207FC13050400EFF09F9F59
:10388000E31C05FA835724013787FFFFB3C7E7001E
:103890002319F4006FF05FFA2313E100930641004F
:1038A0009387E7FF03D60700938626002392C6007E
:1038B000E398F4FE631C0700231401009305040041
:1038C00013054100EFF09FEA6FF01FF79307100018
:1038D0009305F0FF130541002314F100EFF09FC39F
:1038E0006FF0DFFD130101FE232C8100232A9100DC
:1038F00023282101232631012324410123225101C0
:103900001389060013840700232E11009304050079
:1039100093890500130A0600930A0700EFF01FD5EC
:10392000930700093309A94063D4A704B7870000AF
:103930009387E7FF63C6272D938724009384A40110
:1039400093872700239F07FEE39C97FE8320C101F6
:103950000324810183244101032901018329C1003A
:10396000032A8100832A41001301010267800000BD
:10397000635E0900930700F7634CF9129305090091
:1039800013850400EFF01FB96310051463860A2243
:1039900003274400832704006306F7061305A401E8
:1039A000EFF0CFE08327440013078003638EE71610
:1039B0006340F712130780016386E71A1307500369
:1039C0006382E7181307C0002324E400370701804F
:1039D0001307F7FF232AE40013071000231CE40059
:1039E0001307B0002326E4000327C4008356840194
:1039F00013078700131717003307E4002315D700B8
:103A00002320F400634220030327440093070009A6
:103A1000630CF70083D784011385040093F7170024
:103A2000B3E9F900EFF0CFDF8326840003564401A9
:103A300083254400139716003387E400835707005B
:103A4000B3F7C7001306F008634AB6009386160062
:103A5000130607009305C00063DAD51083564401AE
:103A60000356070093C6F6FFB3F6C6002310D7002F
:103A700003576401B376F700638A06106312F702F6
:103A8000639409108327C400035784019397170098
:103A9000B387F40083D70700B3F7E7006388070E06
:103AA000938504001305A401EFF00FEC6F00000EE6
:103AB000938724009384A40193872700239F07FE04
:103AC000E39C97FE6FF09FE8930910006FF01FECE6
:103AD000130700046388E70213071007E394E7EE77
:103AE000378700401307F7FF9306A000232AE4005E
:103AF0002324D4003787FFFF231CE4002326D400AF
:103B00006FF09FEE130770002324E4003707018055
:103B10001307F7FF232AE40013071000231CE40017
:103B2000130760006FF01FEC9306600037078000FA
:103B30001307F70F232AE4002324D40013070010EF
:103B40006FF09FFB370700041307F77F93066000B1
:103B5000232AE400371700002324D400130707802A
:103B60006FF09FF9930640006FF05FFC035526004D
:103B70006304050093E717002311060093861600DF
:103B8000130626006FF05FEDE30C0AF0634C200192
:103B900003274400930700096306F7001385040018
:103BA000EFF00FCD83D7440063880700138504002E
:103BB000EFF00FC713091900B7870000239C04001A
:103BC0009387E7FF63D42703B787FFFF93C7F7FF08
:103BD0002391F40093874400938484012390070089
:103BE00093872700E39CF4FE6FF05FD663560900CD
:103BF000239104006FF09FD5239124016FF01FD50E
:103C0000E3980AD8239C04006FF01FFC130101FE07
:103C100023244101035A2500232C8100138405002D
:103C2000232E1100232A9100232821012322510150
:103C30002320610113090600130B460323263101DB
:103C4000930A0500EFF09FA283542400330AAA4090
:103C500013050400EFF09FA1B384A44013050B00EB
:103C6000EFF0CFB463D244051305040003248101AF
:103C70008320C1018329C100032A8100832A4100D6
:103C8000032B010093070900938604000329010117
:103C90008324410113070000130600009305000070
:103CA000130101026FF01FC49305040013850A007D
:103CB000EFF04FB393090000634AA000930504009E
:103CC00013850A00EFF0CFCD9309100013050B0008
:103CD000EFF00FBA8357C904130504009384F4FF6F
:103CE000B3E9F90023163905EFF08FB86FF09FF7AD
:103CF000130101F72324810823229108232021099D
:103D0000232E310723261108232C4107232A51078C
:103D10002328610723267107232481072322910783
:103D20009304050013840500130906009389060017
:103D3000EFF04FD4630205049305090013850400D6
:103D4000EFF00FA58320C1080324810883244108D4
:103D5000032901088329C107032A8107832A410710
:103D6000032B0107832BC106032C8106832C4106FC
:103D7000130101096780000013050400EFF08FCFE5
:103D80006308050093050900130504006FF05FFB4D
:103D900013850400EFF04FF26314050613050400C9
:103DA000EFF08FF1630C050097D50000938545B2C5
:103DB00013850400EFF0CFDF630E050413850400C4
:103DC000EFF08FEF6318050013050400EFF0CFEE5E
:103DD000630C050413850400EFF00FCD9304050078
:103DE00013050400EFF04FCC638CA402B787FFFFEC
:103DF0002319F90013050900EFF04FEF6FF09FF45E
:103E000097D500009385C5AC13050400EFF04FDA99
:103E1000E31605F813050900EFF0DF926FF09FF24B
:103E2000231909006FF01FFD138504009305C100DD
:103E3000EFF00FCB1305040093058102EFF04FCA9A
:103E40000354E1008354A1026314040293070000A9
:103E5000130760019306C100B386F60083D62600DF
:103E6000638A06101305C100EFF05F803304A040A1
:103E70008357A102138C04006392070213076001A9
:103E800093068102B386F60083D62600638E060E63
:103E900013058102EFF08FFD338CA440835781021C
:103EA000938B490393848903239AF9028357A102D0
:103EB000138A0B00239BF9029387E90423900400E3
:103EC00093842400E39C97FE930A0000130B0000E8
:103ED000930CC0FE9307C100B387570103D5870138
:103EE000630E05009305810213064104EFF0CFAE87
:103EF00093850B0013054104EFF00FA783D7C90486
:103F000013850B00938AEAFF336BFB00EFF04FA39E
:103F1000E3929AFD9307810203570A00130A2A00CD
:103F200093872700239FE7FEE3189AFEB7C6FFFF9B
:103F30003304840193862600938709001307000445
:103F4000B306D4001306000093050B00130581028D
:103F5000EFF05F990357C10083578102631CF7029A
:103F6000231401029305090013058102EFF01F805D
:103F70006FF05FDD93872700E39EE7EC13050900F0
:103F8000EFE0DFFF6FF01FDC93872700E39AE7EE97
:103F90006FF0DFFE9307F0FF2314F1026FF09FFC38
:103FA000130101F7232481082322910823202109EA
:103FB000232A510723261108232E3107232C4107DA
:103FC00023286107232671072324810723229107D1
:103FD0002320A1079304050013840500130906009C
:103FE000938A0600EFF00FA9630405049305090006
:103FF00013850400EFE0DFF98320C1080324810862
:1040000083244108032901088329C107032A810762
:10401000832A4107032B0107832BC106032C81064A
:10402000832C4106032D010613010109678000005E
:1040300013050400EFF00FA46308050093050900C1
:10404000130504006FF01FFB97D50000938545888A
:1040500013850400EFF0CFB56306051E1385040039
:10406000EFF08FC59309050013050400EFF0CFC4EE
:10407000639A091E63100520138504009305C1008F
:10408000EFF00FA61305040093058102EFF04FA592
:104090008354A1020354E1006394040293070000D7
:1040A0001307600193068102B386F60083D62600CB
:1040B0006388061E13058102EFF04FDBB304A040B6
:1040C0008357E100930B040063920702130760011A
:1040D0009306C100B386F60083D626006388061CCB
:1040E0001305C100EFF08FD8B30BA44083578102B2
:1040F0000357A10293894A03239AFA0293878A03FA
:10410000239BEA02138A07001387EA049387270098
:10411000239F07FEE39CE7FE13058102EFE05FF0BB
:10412000035C2101370B0100130BFBFF330D6C0304
:10413000938CA9018357C1020354E10293970701AD
:10414000B387870013040B006368FD0033D4870333
:1041500013140401135404019305C1001305040052
:1041600013064104EFF04F879305810213054104C4
:10417000EFE05FE76356A002930541041305C10019
:10418000EFF00F829305810213054104EFE09FE5F4
:10419000634CA0121304F4FF13140401135404011C
:1041A0009305810213054104EFE09FFF130581028F
:1041B00023108A00130A2A00EFE09FF6E31C9AF707
:1041C0009307000093050000130760019306810226
:1041D000B386F60083D6460093872700B3E5D50063
:1041E000E396E7FEB335B0009307810203D70900D9
:1041F0009389290093872700239FE7FEE3183AFF5E
:10420000B7460000B38474419386F6FF93870A0093
:1042100013070004B386D4001306000013058102BF
:10422000EFF04FEC0357C10083578102631CF70A7C
:10423000231401029305090013058102EFF00FD347
:104240006FF09FDB97C50000938585681305040018
:10425000EFF00F96E31405E013050900EFF08FCEA1
:104260006FF09FD9E31A05FE13050900EFE01FD197
:104270006FF09FD813850400EFF00F8393040500BF
:1042800013050400EFF04F82638CA402B787FFFF91
:104290002319F90013050900EFF04FA56FF0DFD5E2
:1042A00093872700E390E7E06FF01FFC93872700D8
:1042B000E390E7E20357C10083578102E318F7FC5C
:1042C000231909006FF01FFD1304E4FF1314040108
:1042D000930541041305C10013540401EFE05FECA2
:1042E0006FF01FEC9307F0FF2314F1026FF09FF4BF
:1042F00003AE050003A3450083A8850083A5C50080
:10430000130101E2232C811C2326B1021384070030
:10431000832505049307F0FF2328F1149307000970
:104320002328211D2326311D2324411D232E711BEB
:10433000232E111C232A911C2322511D2320611D91
:10434000232C811B232A911B2328A11B2326B11B6D
:10435000232601012320C103232261022324110308
:10436000232AF11413090500130A06009389060095
:10437000930B070063800502832745041307100091
:104380003317F70023A2F50023A4E500EF10407ACD
:10439000232009041305010293050105EFF00FC462
:1043A00013050105EFE05FF0630E05189307100099
:1043B0002320F40093073000630AFA1893044001A5
:1043C000630A0A009384F9FF9307A00263D497005D
:1043D0009304A00283274115130501052328F1004A
:1043E000EFE05FE91304050097C50000938585732E
:1043F000E3140528930700099305C1061305010579
:10440000232AF114EFE0DFB88357E107930A000095
:104410001397070113570741635E070037870000B2
:104420001307F7FFB3F7E700B70A0100231FF106F0
:10443000938AFAFF9305810817C500001305854A82
:10444000EFE01FB50357E107E31807201307C10684
:1044500093070000930690000356070063140610AC
:104460009387170013072700E398D7FE9305010CE5
:1044700013058108EFE0DFE6930581081305010CC1
:10448000EFE01FB49305010C1305C106EFE05FE5F3
:104490009305C1061305010CEFE09FB21306011549
:1044A0009305C10613058108EFF04FF6035BC119B0
:1044B00017CC0000130CCC41631A0B0093050C00C1
:1044C0001305C106EFE0DFEE631E056A9307D00215
:1044D00063940A0093070002230AF1109307300047
:1044E000138C04006318FA00338C84009307A00235
:1044F000E3CE87219307A000631CFB6C9307100396
:10450000A30AF1109307E002230BF110130B7111B2
:10451000635A800193070003A30BF110130CFCFFF7
:10452000130B811113041400635E0C6A130604005C
:1045300097C500009385456113050B00EF2080545B
:104540006F009014232004006FF0DFE693840900CD
:104550006FF09FE78317C10797C500009385855EBD
:10456000E3DC07109305C10617C500001305853766
:10457000EFE01FE4E30C05EE635805469305410A9E
:104580001305C106EFE0DFA0B74700009387E708F7
:10459000231BF10AB78700009387F7FF232AF10056
:1045A000B7C7FFFF93872700130C0000930C00018F
:1045B000232CF10097C700009387073E33858701BE
:1045C00093060115130681089305410AEFF05F9DDC
:1045D0009305C10313058108EFE09F9B83274101E9
:1045E000035BE1043377FB00832781013307F70086
:1045F000634EE0041305010CEFE05F98131B0B0101
:10460000135B0B4163500B12930700001307C103A8
:104610003307F700835607001307010C3307F70031
:1046200003570700638AE63A17C500001305852B78
:10463000EFE05FC4630805089305010C17C500008F
:104640001305452AEFE0DF946F00C00D93070009C2
:10465000338DE7409305010C1305C103EFE05F9331
:104660006352A00D9306010C93070D001306F00092
:104670006342F60493574D00130600FF939617000C
:10468000B387C7021307010CB306D70017C7000092
:1046900013070724B387A70193971700B307F70001
:1046A00083D7C71203D70600B3F7E7002390F600BD
:1046B0006FF0DFF423900600938707FF93862600B0
:1046C0006FF01FFB1305010CEFE0DFBA6308050074
:1046D0009305010C138505006FF0DFF617C5000088
:1046E00013054520EFE05FDD130D05001305010CF8
:1046F000EFE09FDC130B0500630C0D146302051241
:1047000017C500001305051EEFE01FBA130B0500C7
:104710001305010CEFE05FB96314AB101305010C36
:10472000EFF04F8293070000130781083307F7006B
:10473000835607001307010C3307F70003570700E0
:104740006390E6029387270013072001E39EE7FCAE
:104750009305410A13058108EFE09F833304940118
:10476000130C4C019307400693DC1C00E314FCE49B
:104770008357610B0357E1079305C1061305410AEF
:10478000B387E70037C7FFFF130727F7B387E700B3
:10479000231BF10AEFE0CFFF9305810817C5000046
:1047A00013054514EFE0CFFE130B0000B71C00000B
:1047B000930D401097C70000938707149305410A93
:1047C00017C5000013054522338C6701EFE05FBE7B
:1047D000E34EA0C89305410A13050C00EFE05FBD4E
:1047E0006348A0021306410A9305060093060115CB
:1047F00013050C00EFF0CFFA13068108930601159C
:104800009305060013050C00EFF08FCE33049401DE
:10481000130B4B0193DC1C00E31EBBF96FF01FC5AB
:1048200017C500001305050C9305010CEFE04FF6CA
:104830001305010CEFE01FA4E31605EE8357210DCD
:104840003787FFFFB3C7E7002319F10C6FF09FED27
:10485000E31005E89305C10D17C500001305850891
:10486000EFE01FA89305810F1305010CEFE05FA790
:104870000357C10D835DA10F8357E10D1347F7FF68
:10488000131D0701135D0D01231EA10DB387B74151
:104890006354F008930541111305810F232EF10095
:1048A000EFE00FF29305810F1305C10DEFE04FF11B
:1048B0009305C10D13054111EFE08FF08327C1016E
:1048C000835DA10FB307F0401307F0F663C6E70856
:1048D000938507001305C10DEFE0DFC3130D05003D
:1048E0000357C10D8357810F9305810F1305C10D28
:1048F000631EF70CEFE05F879307011513070004B1
:1049000093860D0013060B0093050D001305810F10
:10491000EFE05FFD6F004004E39807FA9305810F15
:104920001305C10DEFE00FEC631805068357810FE7
:104930006388A7011305010CEFE04FE46FF09FDEE1
:1049400063940D020317E10F930700006340070211
:104950001305810FEFE0CFF19305010C1305810FD3
:10496000EFE0DFE06FF01FDC93070000130760014A
:104970009306810F3386F60003562600630806006F
:10498000938D1D00231DB10F6FF01FFD938727002E
:10499000E390E7FE6FF01FFF130D0000E352A0F459
:1049A000930541111305810FEFE08FE19305810F0E
:1049B0001305C10DEFE0CFE09305C10D13054111C3
:1049C000EFE00FE0130D0B006FF09FF1EFE04FFDF4
:1049D000130B10006FF05FF293872700130720017D
:1049E000E396E7C26FF01FD48357E10717CB0000AF
:1049F000130B8BFF6388070A9305010C1305C1068F
:104A0000374B0000EFE0DF8D130BEBFF130C50FD75
:104A10008357810D93F77700639207069305410A48
:104A20001305010CEFE0CFD91305410AEFE04FDF8A
:104A30001305410AEFE0CFDE9305410A1305010C8F
:104A4000EFE08FF28357610A938737002313F10A4F
:104A50008357810A639E07108357C10B6390070237
:104A60008357610A636CFB009305010C1305410A2F
:104A70001304F4FFEFE0CFD4E31C84F99305C106DF
:104A80001305010CEFE09FCE6F0040021306C10634
:104A9000930601159305060013050B00EFF04FA5D3
:104AA0001304F4FF8317C107E3D207FE9305010C3B
:104AB0001305C106EFE0CFCD9305810817C50000AF
:104AC000130545E2EFE0CFCC930C000037FBFFFF6E
:104AD000130D2000930D401097C700009387C7E186
:104AE000338C970197C70000938787F3338797012B
:104AF0009305010C17C500001305C5DE232AE1004C
:104B0000EFE01F8B032741016356A0049305010CBE
:104B100013050700EFE0DF89634805021306010C67
:104B2000930506009306011513050C00EFF04F9C4A
:104B300013068108930601159305060013050C0062
:104B4000EFF00F9B33046401938C4C01334BAB03A8
:104B5000E394BCF9130681089306011597C500007C
:104B6000938545D813050600EFF08FC36FF01F90B3
:104B70001305410AEFE0CFCA8357610A93871700F4
:104B80006FF0DFEC1305C106EFE08FCE9305410A0D
:104B90001305C106EFE0CFC21305410AEFE04FCD88
:104BA0001305410AEFE0CFCC9305C1061305410A76
:104BB000EFE08FDB130601159305C106130581088D
:104BC000EFF0CF841304F4FF035BC1196FF0DF8EA5
:104BD000130B0B039307E002A30A6111230BF110DF
:104BE000130B7111930A0B00B3876A416356FC04DF
:104BF0008357C11913074000138BFAFFE358F7924C
:104C0000130750006384E70893070B001306E002C4
:104C100093058003930600039387F7FF03C70700FC
:104C20001377F70763580C0A130710032380E70074
:104C3000130414006FF09F8F1305C106EFE04FC3FC
:104C40009305410A1305C106EFE08FB71305410A2A
:104C5000EFE00FC21305410AEFE08FC19305C106D3
:104C60001305410AEFE04FD0130601159305C10665
:104C700013058108EFE09FF98347C119938A1A0051
:104C800093870703A38FFAFE6FF01FF69305810841
:104C90001305C106EFE09FAD97C50000938545C39E
:104CA00013058108EFE0CFF0E31005F6E3400C8830
:104CB00083C7EAFF938727FD93B7170093C7F7FFD2
:104CC000B307FB0083C7070093F71700E38007864D
:104CD0006FF09FF36314C70203C7F7FF93068003C7
:104CE00063E8E60013071700A38FE7FE6FF01F8449
:104CF00013041400130710036FF01FFF63E8E500AF
:104D0000130717002380E7006FF05F822380D7002E
:104D10006FF09FF01304140023A08B0093870A0008
:104D20009306E00203C70700631607001307500449
:104D30006F00C002630CD700938717006FF09FFECF
:104D400003C7170093871700A38FE7FE03C7070069
:104D5000E31807FE6FF09FFD9387F7FF83C60700F8
:104D60006384E600E3EAFAFE238007006F00001583
:104D7000938717006F004015138406006F00C0155D
:104D80001304F4FF230004000347F4FF6316D70065
:104D900033075441E3C6E7FE9307300013879900B9
:104DA0006314FA0283270116B384F40063D8040065
:104DB000230A011023A00B0013840A0083A70B0011
:104DC000B389F900138739002322090493074000AF
:104DD00093864701832549046378D70613050900A4
:104DE000EF00904A2320A90493850A00930405004C
:104DF000EF10507C8327C1006388070033045441BF
:104E00003384840023A087008320C11D0324811DD7
:104E1000138504000329011D8324411D8329C11C1E
:104E2000032A811C832A411C032B011C832BC11BD9
:104E3000032C811B832C411B032D011B832DC11AC5
:104E40001301011E67800000938515002322B90419
:104E5000939717006FF0DFF7B78700009387F7FF8E
:104E6000631AF7EE97C50000938505CD63860A00A7
:104E700097C50000938585CB1305411137240000A9
:104E8000EF1050401304F47083270101130501054E
:104E900023208116232AF114EFE00FE2930A411137
:104EA0006318050013050105EFE0CFBCE30405E638
:104EB000B72700009387F77023A0FB0093870A00B1
:104EC000130600029306D00203C70700E302C7EAF5
:104ED000E300D7EA13840A009387170003C7F7FF9C
:104EE00093061400A38FE6FEE31807E813072000DB
:104EF000930710006308EA008327011663D4970024
:104F000093870400930600036FF01FE89307A00047
:104F1000130CA002E31EFBCA93071003A30AF110AF
:104F20009307E002230BF110130CA0026FF08FDE49
:104F300083270500130101FC930541012320F100A3
:104F400083274500232E11022322F10083278500A9
:104F50002324F1008327C500130501002326F10057
:104F6000EFE0DF87835761021305000093C7F7FF67
:104F700013971701631A070013054101EFE08FAF84
:104F800013351500130515008320C1031301010417
:104F9000678000001305050F6780000097D70000A9
:104FA000938747F683A7070003A547036316050009
:104FB00017D500001305859D1305050F67800000B8
:104FC00097D70000938707F483A7070003A547033B
:104FD0006316050017D500001305459B1305050F43
:104FE0006780000063080606130101FF97C50000F3
:104FF000938505B61305060023248100232611009E
:1050000013040600EF1050436308050297C5000023
:105010009385C5B313050400EF101042630E05001D
:1050200097B500009385056E13050400EF10D0407E
:10503000930700006316050097C70000938707B128
:105040008320C1000324810013850700130101019F
:105050006780000097C70000938747AF138507005C
:105060006780000097D700009387C7E983A70700F0
:1050700083A747036396070097D70000938707919C
:1050800003C58712678000000325C50E67800000F6
:1050900097D70000938707E783A7070083A74703F5
:1050A0006396070097D700009387478E03A5C70E26
:1050B0006780000097D700009387C7E41386050038
:1050C0009305050003A507006FF0DFF1130101FA56
:1050D000232A9104938405008395E500232C810401
:1050E000232E11041304060063DE050083D7C400D9
:1050F00023A0060093F7070863980704930700406E
:105100006F00C004130641012326D100EF40107147
:105110008326C100E34C05FC03278101B7F700009B
:1051200037150000B3F7E70037E7FFFFB387E70065
:1051300093B7170023A0F600930700402320F40044
:10514000130505806F000001930700042320F4007D
:10515000130500008320C105032481058324410534
:10516000130101066780000083D7C500130101FE0B
:10517000232C8100232E1100232A910023282101B2
:1051800093F727001384050063880702930734040C
:105190002320F4002328F40093071000232AF400AE
:1051A0008320C101032481018324410103290101DA
:1051B00013010102678000009306C10013068100FD
:1051C00093040500EFF09FF083258100130905008B
:1051D00013850400EF004008631005028317C40024
:1051E00013F70720E31E07FA93F7C7FF93E727009B
:1051F0002316F4006FF09FF997D7FFFF9387075CA2
:1052000023AEF4028357C4002320A4002328A40063
:1052100093E707082316F40083278100232AF4006C
:105220008327C100638207028315E400138504000D
:10523000EF50C029630A05008357C40093F7C7FFE6
:1052400093E717002316F4008357C4003369F9006D
:10525000231624016FF0DFF4130101FD2326110250
:10526000232481022322910223202103232E3101B2
:10527000232C4101232A5101232861012326710196
:10528000232481019387B500130760016374F70439
:1052900093F487FF63D204049307C0002320F50032
:1052A000130500008320C1020324810283244102EC
:1052B000032901028329C101032A8101832A4101B3
:1052C000032B0101832BC100032C81001301010377
:1052D0006780000093040001E3E0B4FC13090500BB
:1052E000EF00007A9307701F97D900009389C98057
:1052F00063EA9704138784003387E9000324470097
:10530000930687FF93D734006318D4000324C700A3
:105310009387270063008708832744000327C4007E
:105320008326840093F7C7FFB307F40023A6E600A3
:105330002324D70003A747001367170023A2E70021
:105340006F00C00A13D794009307F003630A0700A5
:105350009307400063E4E70A93D7640093878703C9
:1053600013871700131737003387E900032447001A
:10537000930587FF1305F000630CB4000327440076
:105380001377C7FF330697406352C50C9387F7FF27
:105390009387170003A4090197C5000093854576FC
:1053A0006302B414032744009306F0001377C7FF89
:1053B0003306974063DEC60A93E714002322F40005
:1053C000B306940097C7000023A2D77497C70000C4
:1053D00023ACD7729367160023A6B60023A4B600A9
:1053E00023A2F6003307E4002320C70013050900B9
:1053F000EF004069130584006FF0DFEA9307400176
:1054000063E6E7009307B7056FF09FF59307400544
:1054100063E8E70093D7C4009387E7066FF05FF473
:105420009307401563E8E70093D7F4009387770765
:105430006FF01FF3930640559307E007E3E2E6F2AF
:1054400093D724019387C7076FF09FF18326C40089
:10545000634C06008327840023A6D70023A4F6000C
:10546000B307E4006FF01FED138406006FF0DFF068
:1054700097C6000023ACB66897C6000023A6B6689E
:10548000634C06003307E4008327470093E71700C7
:105490002322F7006FF09FF59306F01F03A8490041
:1054A00063E2E61A1357370013562740930610009D
:1054B00013071700B396C600131737003387E900A8
:1054C000B3E6060117C60000232AD662832607002A
:1054D000130687FF2326C4002324D400232087003B
:1054E00023A6860013D72740130310003313E300CD
:1054F00003A74900636C6706B3766700639C0600E8
:1055000093F7C7FF13131300B37667009387470021
:10551000E38A06FE130EF00093963700B386D90097
:1055200013880600138507000324C800631E041DAA
:10553000130515001377350013088800E31607FEDE
:1055400013F737006314072403A749009347F3FFB9
:10555000B377F70017C700002322F75A03A74900C3
:1055600013131300636467006316032483AB89007D
:1055700003A44B00937AC4FF63E89A0033879A40F0
:105580009307F00063C0E73697D700009387079929
:1055900003A4070097D700009387079783A6070007
:1055A0001307F0FF33848400138A07006398E62012
:1055B000130404019305040013050900EF1040369D
:1055C0009307F0FF130B05006302F52AB3875B0115
:1055D0006374F500639C3B2917DC0000130C8C946A
:1055E00003270C003307E40097D6000023ACE692B3
:1055F0006392671F93964701639E061C83A78900E9
:1056000033848A001364140023A2870017D7000094
:105610001307879083270C00032707006376F700A2
:1056200017D70000232AF78E17D700001307878E9D
:1056300003270700637CF72217D70000232CF78C81
:105640006F00C022135697009306400063E8C6041B
:10565000935667009386860313861600131636004A
:105660003386C900130586FF032606006314C508A8
:105670001307100093D62640B316D700B3E60601F1
:1056800017C70000232CD7462326A4002324C400D8
:1056900023248500232686006FF0DFE49306400173
:1056A00063E6C6009306B6056FF01FFB9306400540
:1056B00063E8C6009356C7009386E6066FF0DFF9ED
:1056C0009306401563E8C6009356F7009386760765
:1056D0006FF09FF8130540559306E007E36EC5F69B
:1056E000935627019386C6076FF01FF7032686009F
:1056F0006308C5008326460093F6C6FFE368D7FE1D
:105700000325C6006FF05FF8032744000326C4009A
:105710001377C7FFB308974063541E0593E714003F
:105720002322F40083278400B30694003307E400A7
:1057300023A6C7002324F60097C7000023A8D73C60
:1057400097C7000023A2D73C93E7180023A6B60012
:1057500023A4B60023A2F600232017016FF01FC96F
:1057600063C208023307E4008327470093E717006A
:105770002322F7008327840023A6C7002324F600F2
:105780006FF0DFC6130406006FF05FDA138786FF41
:1057900083A606009387F7FFE384E6DA6FF01FDC49
:1057A0009387470013131300B3766700E38A06FE5E
:1057B0006FF09FD6930705006FF01FFFB71700002B
:1057C0009387F7003304F400B7F7FFFF3374F40056
:1057D0006FF05FDE03260A009306F0FF631CD60A13
:1057E00097C7000023A2677393757B006388050049
:1057F00093078000B385B740330BBB00B717000099
:10580000B385F50033048B009387F7FF3374F400FE
:10581000338A854093050A0013050900EF104010F4
:105820009307F0FF6316F50013050B00130A000041
:1058300083270C0033056541B3874701330A4501CF
:1058400017C700002320F76E136A1A0097C70000DD
:1058500023A8672B23224B01E38A3BDB1307F000CD
:1058600063645705930710002322FB0083A7890078
:1058700083A7470093F7C7FF3387974063E69700F6
:105880009307F00063C0E70613050900EF00801FCF
:105890006FF01FA1B307FB40B387E70017C70000F5
:1058A0002322F7686FF05FF483A74B0013844AFF4D
:1058B000137484FF93F71700B3E7870023A2FB005C
:1058C00093065000B3878B0023A2D70023A4D700F0
:1058D000E37E87D293858B0013050900EFD00FADCF
:1058E0006FF0DFD203A4890093E714002322F400B1
:1058F000B307940097C6000023A4F6206FF0DFA33F
:1059000097C700009387076083A7070083A7470313
:105910006396070097C700009387470703A3470EC6
:1059200067000300639A0502130101FF9305C1009C
:1059300013050000630E06001305E0FF638A0600EE
:105940008347060023A0F500034506003335A00079
:1059500013010101678000001305000063000602C7
:105960001305E0FF638C06008347060023A0F500C3
:10597000034506003335A000678000006780000003
:1059800093F5F50F3306C5006316C5001305000037
:105990006780000083470500E38CB7FE1305150000
:1059A0006FF09FFE1303F00013070500637EC30230
:1059B0009377F7006390070A63920508937606FFD2
:1059C0001376F600B386E6002320B7002322B70043
:1059D0002324B7002326B70013070701E366D7FE89
:1059E0006314060067800000B306C3409396260048
:1059F00097020000B38656006780C6002307B700F1
:105A0000A306B7002306B700A305B7002305B70018
:105A1000A304B7002304B700A303B7002303B70010
:105A2000A302B7002302B700A301B7002301B70008
:105A3000A300B7002300B7006780000093F5F50FBF
:105A400093968500B3E5D50093960501B3E5D5009F
:105A50006FF0DFF69396270097020000B38656009A
:105A600093820000E78006FA93800200938707FF85
:105A70003307F7403306F600E378C3F66FF0DFF341
:105A800067800000678000008327C504130101FFC1
:105A900023229100232021012326110023248100A9
:105AA00093040500138905006382070403A7C40457
:105AB00093172900B307F70003A507006310050635
:105AC0001304100033142401130654001316260087
:105AD0009305100013850400EF40001D63020502CA
:105AE00023222501232485006F00C0031306100222
:105AF00093054000EF40401B23A6A404E31805FAD9
:105B0000130500008320C100032481008324410089
:105B1000032901001301010167800000032705002C
:105B200023A0E70023280500232605006FF09FFD32
:105B30006380050283A74500139727008327C504C8
:105B4000B387E70003A7070023A0E50023A0B70061
:105B500067800000130101FD232E31019309050028
:105B600037050100232481022322910213840500BA
:105B700083A40501232611022320210393854501D7
:105B8000130800001305F5FF83A705009385450062
:105B90001308180033F7A7003307C70293D707018C
:105BA000B387C7023307D700935607013377A7009F
:105BB000B387D70093D6070193970701B387E70010
:105BC00023AEF5FEE34298FC638406068327840037
:105BD00063C4F40483254400138509002326D100FF
:105BE00093851500EFF05FEA032604019305C400D6
:105BF0001309050013062600131626001305C50019
:105C0000EF40D0169305040013850900EFF05FF212
:105C10008326C1001304090093874400939727004B
:105C2000B307F40023A2D700938414002328940020
:105C3000130504008320C10203248102832441024E
:105C4000032901028329C1011301010367800000B8
:105C5000130101FD93878600232A5101938A0600D0
:105C6000930690002324810223229102232C4101D8
:105C700013840500B3C7D702232611022320210372
:105C8000232E3101130A0500930406009306100029
:105C90009305000063C6F60813050A002326E100F9
:105CA000EFF09FDE0327C100930710002328F500C3
:105CB000232AE5009307900063DA970613099400FE
:105CC00093090900330494009389190083C6F9FFEE
:105CD000930505001306A000938606FD13050A0030
:105CE000EFF05FE7E39289FE33049900130484FF29
:105CF000B3848440B307940063C057058320C10276
:105D00000324810283244102032901028329C10162
:105D1000032A8101832A41011301010367800000E6
:105D200093961600938515006FF0DFF61304A40018
:105D3000930490006FF0DFFB130414008346F4FF1C
:105D4000930505001306A000938606FD13050A00BF
:105D5000EFF05FE06FF01FFA3707FFFF3377E500E2
:105D600093070500130500006316070093970701CA
:105D700013050001370700FF33F7E700631607003C
:105D80001305850093978700370700F033F7E70086
:105D9000631607001305450093974700370700C0B7
:105DA00033F7E700631607001305250093972700D4
:105DB00063CC0700139717006356070013051500FF
:105DC000678000001305000267800000832705003C
:105DD00013F77700630E070293F61700130700000E
:105DE000639C060013F72700630C070093D7170086
:105DF0002320F5001307100013050700678000003B
:105E000093D727002320F500130720006FF0DFFE53
:105E10009396070193D606011307000063960600C8
:105E200093D707011307000193F6F70F6396060057
:105E30001307870093D7870093F6F7006396060051
:105E40001307470093D7470093F637006396060081
:105E50001307270093D7270093F6170063980600CF
:105E600093D7170063880700130717002320F50056
:105E70006FF09FF8130700026FF01FF8130101FF86
:105E800023248100138405009305100023261100AC
:105E9000EFF09FBF232A85008320C10003248100E7
:105EA000130710002328E50013010101678000009B
:105EB00003A7050183270601130101FD2322910297
:105EC000232611022324810223202103232E3101C2
:105ED000938405006356F7009304060013860500BB
:105EE00083A904010329060183A7840083A5440034
:105EF0003384290163D48700938515002326C100CC
:105F0000EFF09FB80326C1001308450113132400C6
:105F1000330368009307080063EC6704938544012A
:105F20009398290013064601131E2900B7060100A5
:105F3000B3881501330EC6019386F6FF6360C6056C
:105F4000635880001303C3FF83270300638607128F
:105F5000232885008320C102032481028324410277
:105F6000032901028329C101130101036780000095
:105F700023A00700938747006FF01FFA032F060046
:105F8000337FDF0063040F06930F08009382050040
:105F90009304000003A7020083A30F009382420032
:105FA000B37ED700B38EEE03B3F7D30093D30301D0
:105FB000B38EFE0093570701B387E703B38E9E00AD
:105FC00013D70E01B3FEDE00B3877700B387E70077
:105FD00093D407019397070113874F00B3E7D701C5
:105FE000232EF7FE63E2120923A29F0083522600AC
:105FF0006386020683270800930E0800138F0500AE
:10600000930F000003270F0083D32E00B3F7D700B0
:106010003377D70033075702130F4F00330777004A
:106020003307F701931F0701B3E7FF0093834E0087
:1060300023AEF3FE8357EFFF83AF4E0013570701E4
:10604000B3875702B3FFDF00B387F701B387E700D9
:1060500093DF0701636E1F0123A2FE0013064600B3
:10606000130848006FF09FED930F07006FF09FF249
:10607000938E03006FF01FF91304F4FF6FF05FECD1
:10608000130101FE232A9100232821012326310137
:10609000232E1100232C8100232441019377360005
:1060A0001309050093040600938905006384070221
:1060B0009387F7FF17B70000130747AA93972700A6
:1060C000B307F70003A6070093060000EFF09FA8B0
:1060D0009309050093D424406380040803248904B1
:1060E000631E04009305102713050900EFF01FD964
:1060F0002324A904130405002320050093F71400AA
:106100006384070293850900130604001305090040
:10611000EFF01FDA130A0500938509001305090043
:10612000EFF01FA193090A0093D414406386040280
:1061300003250400631E05001306040093050400F4
:1061400013050900EFF0DFD62320A400232005006B
:10615000130405006FF09FFA8320C101032481011D
:106160001385090083244101032901018329C1000A
:10617000032A81001301010267800000130101FD61
:106180002322910293840500232E310183A9040167
:106190002324810283A545001354564083A784001D
:1061A000B309340123202103232A5101232611029C
:1061B000232C4101930A05001389190063C6270D9A
:1061C00013850A002326C100EFF01F8C0326C100AF
:1061D00093074501130A0500938607001307000083
:1061E000938646006348870A635404001304000042
:1061F00083A6040113142400338787009396260096
:10620000938744011376F601B386D700630E060820
:10621000130800023308C8409305000003A50700D7
:1062200093084700938747003315C500B365B50051
:1062300023AEB8FE83A5C7FFB3D5050163E2D70639
:106240002322B70063840500138929001309F9FF8D
:1062500023282A0113850A0093850400EFF05F8D3F
:106260008320C1020324810213050A008324410212
:10627000032901028329C101032A8101832A4101E3
:1062800013010103678000009385150093971700A1
:106290006FF0DFF223AE06FE130717006FF05FF416
:1062A000138708006FF09FF79387470003A6C7FF87
:1062B00013074700232EC7FEE3E8D7FE6FF01FF950
:1062C0008327050103A70501B387E740639C070205
:1062D000131727001305450193854501B306E50013
:1062E000B385E5009386C6FF9385C5FF03A6060028
:1062F00003A70500630CE6009307F0FF6364E60064
:10630000930710001385070067800000E36CD5FC3D
:106310006FF05FFF130101FE232A910093840500B3
:106320002326310193050600930905001385040017
:10633000232C8100232E11002328210113040600A1
:10634000EFF01FF8631C0502930500001385090098
:10635000EFF08FF3930710002328F500232A0500A0
:106360008320C10103248101832441010329010108
:106370008329C10013010102678000001309100086
:10638000634A050093070400130900001384040006
:10639000938407008325440013850900EFF0CFEEB6
:1063A0000323040183A8040113064401131E2300E0
:1063B0001388440193982800B70E01002326250175
:1063C000330EC601B308180193064501130F0000F0
:1063D000938EFEFF03270600832F08009386460056
:1063E000B375D701B3F7DF01B385E501B385F54098
:1063F00093DF0F0193570701B387F74113D7054187
:10640000B387E70013DF0741B3F5D5019397070181
:10641000B3E7B7001308480023AEF6FE13064600A4
:10642000E36A18FBB70501009385F5FF636CC601AD
:106430009386C6FF83A706006382070423286500AE
:106440006FF01FF28327060093864600130646006E
:1064500033F7B7003307E7011358074193D7070114
:10646000B387070113DF07413377B700939707011D
:10647000B3E7E70023AEF6FE6FF05FFB1303F3FF15
:106480006FF01FFBB707F07FB3F5B700B707C0FC8D
:10649000B385F5006358B00093070000138507002B
:1064A00067800000B305B04093D745411307300122
:1064B0006348F700B7050800B3D5F5406FF0DFFD7E
:1064C0009387C7FE9306E0019305000013071000B1
:1064D00063C6F60093C7F7FF3317F700930707006B
:1064E0006FF0DFFB130101FD2322910283240501DC
:1064F000232E31019309450193942400B38499001C
:106500002324810203A4C4FF232021032326B100F6
:106510001305040023261102EFF01F848325C10018
:1065200093070002B387A74023A0F5009307A000BC
:106530001389C4FF63CCA7049307B000B387A740B7
:106540003707F03FB356F400B3E6E6001307000048
:1065500063F4290103A784FF130555013315A40033
:10656000B357F700B367F5008320C102032481020B
:1065700083244102032901028329C10113850700F5
:106580009385060013010103678000009307000054
:1065900063F6290183A784FF138984FF130555FF40
:1065A000630E0502130700023306A7403314A4004C
:1065B0003707F03F3364E400B3D6C700B366D400B6
:1065C0001307000063F429010327C9FFB397A7004D
:1065D0003357C700B3E7E7006FF01FF9B706F03F86
:1065E000B366D4006FF05FF8130101FD232481022C
:1065F0001384050093051000232291022320210318
:1066000093040600232E3101232C410113090700B6
:1066100023261102138A0600EFF00FC73707100078
:106620009307F7FFB3F7970093D4440193F4F47FF3
:1066300093090500639A04082326F100630E0408F9
:106640001305810023248100EFF04FF88326810099
:10665000630005080327C10093070002B387A74022
:10666000B317F700B3E7D7003357A70023AAF90001
:106670002326E1000324C10023AC890033348000C9
:106680001304140023A88900638A04069384D4BCED
:10669000B384A4009307500323209A003385A740B6
:1066A0002320A9008320C10203248102138509004D
:1066B00083244102032901028329C101032A8101A4
:1066C0001301010367800000B3E7E7006FF0DFF616
:1066D00023AAD9006FF01FFA1305C100EFF00FEFE6
:1066E0008327C100130505021304100023AAF90033
:1066F0009307100023A8F9006FF01FF993172400E7
:106700001305E5BCB387F9002320AA0003A5070100
:1067100013145400EFF04FE43304A4402320890005
:106720006FF05FF8130101FD232021031389050099
:106730009305810023261102232481022322910242
:10674000232E3101232C4101130A0500EFF09FD9BC
:1067500093090500938405001384050013050900BF
:106760009305C100EFF01FD88327090103270A0111
:10677000832681003307F7408327C1001317570092
:10678000B386F640B307D7006354F00493974701EC
:106790001386050033849700130706009305040051
:1067A000130605009306070013850900EF501063D8
:1067B0008320C102032481028324410203290102B0
:1067C0008329C101032A81011301010367800000AD
:1067D0003707F0FFB387E7023386B7006FF0DFFBC0
:1067E000130101FF2324810023261100232221010C
:1067F00023203101930770011304050063CAA70227
:106800001314350097A7000093874735338487001A
:1068100003250401832544018320C1000324810052
:106820000329410083290100130101016780000051
:1068300097B70000938707BB03A5070083A5470010
:1068400097B70000938787BA03A9070083A9470079
:1068500013060900938609001304F4FFEF60004655
:10686000E31804FE6FF05FFB9387F5FF0327060133
:1068700093D75740938717009397270093064601B5
:1068800013172700B307F5003387E60063E6E60039
:10689000636EF500678000009386460003A6C6FF7E
:1068A00013054500232EC5FE6FF05FFE130545005E
:1068B000232E05FE6FF0DFFD8326050193D755409B
:1068C0001307450163C0F60463D4D70293F5F501BD
:1068D0006380050293962700B306D70003A606003F
:1068E00013051000B356B600B395B6006318B60290
:1068F00093972700B307F700636AF70013050000BA
:1069000067800000938706006FF09FFE9387C7FFA4
:1069100083A60700E38206FE1305100067800000CF
:10692000130101FF232481001304050013850500D2
:1069300097B7000023AC076023261100EF90D041E9
:106940009307F0FF631CF50097B70000938707607B
:1069500083A70700638407002320F4008320C1007D
:10696000032481001301010167800000130101FF6E
:1069700023229100B70400802324810023261100E4
:1069800093C4F4FF33F7B400232006003708F07FE8
:106990009306050093870500130406006354070758
:1069A0003368A70063000806B707100013860500C8
:1069B0006356F70297B700009387C7A303A60700A3
:1069C00083A64700EF60802F9307A0FC9306050085
:1069D0001386050033F7B4002320F4008327040056
:1069E00013574741130727C03387E700B7071080C5
:1069F0009387F7FF3376F600B707E03F2320E400E4
:106A0000B367F6008320C100032481008324410082
:106A100013850600938507001301010167800000BC
:106A2000130101F6232AF108B707008093C7F7FF87
:106A3000232EF1002328F100B707FFFF2326D108FA
:106A40002324B100232CB100938787209306C1082B
:106A500093058100232E1106232AF1002328E10843
:106A6000232C0109232E11092322D100EF00803CA1
:106A700083278100238007008320C1071301010AB7
:106A800067800000130101F6232AF108B707008090
:106A900093C7F7FF232EF1002328F100B707FFFF6C
:106AA000938787202324C1082326D1082328E108BF
:106AB000232C0109232E1109232AF10097B7000086
:106AC000938747442324A100232CA10003A507009A
:106AD000930681081386050093058100232E110675
:106AE0002322D100EF000035832781002380070097
:106AF0008320C1071301010A67800000130101FF11
:106B000023248100138405008395E50023261100CA
:106B1000EF3090396340050283270405B387A7004F
:106B20002328F4048320C100032481001301010100
:106B3000678000008357C40037F7FFFF1307F7FF94
:106B4000B3F7E7002316F4006FF0DFFD1305000034
:106B50006780000083D7C500130101FE232C81004C
:106B6000232A91002328210123263101232E1100FD
:106B700093F707109304050013840500130906001A
:106B800093890600638A07008395E5009306200039
:106B900013060000EF3050188357C40037F7FFFF8B
:106BA0001307F7FFB3F7E7002316F4008315E4009B
:106BB000032481018320C101938609001306090083
:106BC0008329C100032901011385040083244101A5
:106BD000130101026F300008130101FF232481001B
:106BE000138405008395E50023261100EF30D012B1
:106BF0009307F0FF0357C4006312F502B7F7FFFFD6
:106C00009387F7FFB3F7E7002316F4008320C10052
:106C1000032481001301010167800000B717000001
:106C2000B367F7002316F4002328A4046FF01FFEB7
:106C30008395E5006F3000113367B5009303F0FFD3
:106C40001377370063100710B7877F7F9387F7F7B5
:106C50000326050083A60500B372F6003363F60031
:106C6000B382F200B3E26200639272106316D60838
:106C70000326450083A64500B372F6003363F60091
:106C8000B382F200B3E26200639E720C6316D60612
:106C90000326850083A68500B372F6003363F600F1
:106CA000B382F200B3E262006398720C6316D604FA
:106CB0000326C50083A6C500B372F6003363F60051
:106CC000B382F200B3E262006392720C6316D602E2
:106CD0000326050183A60501B372F6003363F600AF
:106CE000B382F200B3E26200639C720A13054501AD
:106CF00093854501E30ED6F4131706019397060119
:106D0000631EF7001357060193D706013305F740BA
:106D10009375F50F63900502678000001357070114
:106D200093D707013305F7409375F50F639405007A
:106D3000678000001377F70F93F7F70F3305F740DD
:106D4000678000000346050083C605001305150093
:106D5000938515006314D600E31606FE3305D6406E
:106D6000678000001305450093854500E31CD6FCB1
:106D700013050000678000001305850093858500DA
:106D8000E312D6FC13050000678000001305C50060
:106D90009385C500E318D6FA13050000678000004C
:106DA0001305050193850501E31ED6F813050000C0
:106DB000678000009307050003C70500938717004D
:106DC00093851500A38FE7FEE31807FE6780000098
:106DD000930705009387170003C7F7FFE31C07FE1F
:106DE0003385A7401305F5FF6780000013070500F2
:106DF00063140600678000009385150083C6F5FFC5
:106E0000930717001308F6FFA38FD7FE63980600B9
:106E10003307C700639AE700678000001387070005
:106E2000130608006FF0DFFC93871700A38F07FE9F
:106E30006FF05FFE130101E32326111C2322911C36
:106E40002320211D232E311B232A511B938905004A
:106E500093040600938A06002324811C232C411BE3
:106E60002328611B2326711B2324811B2322911BB2
:106E70002320A11B232EB11913090500EFE00F9267
:106E800083270500138507002324F102EFF05FF448
:106E900083D7C900232AA1002328010C232A010C2F
:106EA000232C010C232E010C93F7070863800704A1
:106EB00083A70901639C07029305000413050900D9
:106EC000EFE08FB923A0A90023A8A900631C050047
:106ED0009307C0002320F9009307F0FF232CF10053
:106EE0006F00C0589307000423AAF9009308C10E4D
:106EF0002322110D2326010C2324010C130A000068
:106F0000232A010223280102232401002322010253
:106F100023260102232C01001384040013075002CE
:106F200083470400638407006392E70C330B9440AB
:106F3000630A0B048327C10C23A0980023A26801D5
:106F4000B38767012326F10C8327810C1307700098
:106F500093888800938717002324F10C635EF70061
:106F60001306410C9385090013050900EF305063A7
:106F70006318054E9308C10E83278101B38767010B
:106F8000232CF10083470400639407006F10505EC8
:106F9000930714002328F100A303010A130BF0FF49
:106FA000232E010013040000930B90009306A0050C
:106FB0001306A0028327010103CD07009387170062
:106FC0002328F10093070DFE63F4F6006F10802A6A
:106FD00017A70000130707CB93972700B387E70095
:106FE00083A70700B387E700678007001304140036
:106FF0006FF01FF397A700009387078C232AF102F5
:1070000093770402639407006F108008938A7A00D4
:1070100093FA8AFF03AC0A0083AC4A0093878A0084
:107020002326F10093771400638E0700B3679C0159
:10703000638A0700930700032304F10AA304A10B4A
:10704000136424001374F4BF930720006F00D0442E
:107050001305090023221101EFD05FF483274500B7
:10706000138507002326F102EFF09FD62322A10209
:1070700013050900EFD09FF2832785008328410084
:107080002324F10083274102E38207F28327810052
:10709000E38E07F083C70700E38A07F01364044018
:1070A0006FF0DFF08347710AE39207F09307000265
:1070B000A303F10A6FF09FEF136414006FF01FEF4A
:1070C00083A70A00938A4A00232EF100E3D007EE3B
:1070D000B307F040232EF100136444006FF01FED5E
:1070E0009307B0026FF0DFFC032701018327010142
:1070F000034D0700938717006310CD0403AB0A000C
:1071000013874A0063540B00130BF0FF930A070028
:107110002328F1006FF09FE99305A0003303BB0221
:107120009387170003CDF7FF330BE30013070DFD23
:10713000E3F4EBFE6FF0DFE8130B00006FF01FFFCE
:10714000136404086FF09FE683270101232E0100DA
:107150000327C1019305A000130D0DFD3307B702EE
:10716000938717003307ED0003CDF7FF232EE100CF
:1071700013070DFDE3FEEBFC6FF09FE41364840046
:107180006FF0DFE28327010103C707009307800642
:10719000631CF70083270101136404209387170001
:1071A0002328F1006FF09FE0136404046FF01FE0E8
:1071B0008327010103C707009307C006631CF7007C
:1071C00083270101938717002328F1001364040229
:1071D0006FF0DFDD136404016FF05FDD93874A0019
:1071E0002326F10083A70A00A303010A2306F11254
:1071F00023220100130B1000930D0000130C00005C
:10720000930B0000930C00009304C1126F005039DF
:107210001364040193770402638E0704938A7A004F
:1072200093FA8AFF03AC0A0083AC4A0093878A0072
:107230002326F10063DE0C00330C8041B33780015C
:10724000B30C9041B38CFC409307D002A303F10A26
:107250009307F0FFE31CFB66E39E0C6E9307900020
:10726000E3EA876F130C0C03A30781199304F11849
:107270006F00D06B93874A002326F10093770401B7
:107280006388070003AC0A00935CFC416FF09FFA2F
:107290009377040403AC0A0063880700131C0C01F5
:1072A000135C0C416FF05FFE93770420E38E07FCC4
:1072B000131C8C01135C8C416FF01FFD93778400CD
:1072C0006382070C93874A002326F10083A70A00F4
:1072D00003A6070083A6470003A7870083A7C7006C
:1072E0002328C10C232AD10C232CE10C232EF10CD2
:1072F0001305010D23221101EFD09FC32326A10AFC
:1073000093072000832841006314F50C8327010DA7
:1073100093050108130501092328F1088327410D6E
:107320002320010823220108232AF1088327810D45
:107330002324010823260108232CF1088327C10DEB
:10734000232EF108EF6000188328410063560500E2
:107350009307D002A303F10A9307700497940000E7
:107360009384845363C6A701979400009384845246
:107370001374F4F723220100130B3000930D000067
:107380006F00D05B938A7A0093FA8AFF83A50A0084
:1073900003A64A0093878A001305010923221101DD
:1073A0002326F100EF80502683270109832841001E
:1073B0002328F10C83274109232AF10C8327810913
:1073C000232CF10C8327C109232EF10C6FF05FF2FF
:1073D000930710006318F5028327C10D63D60700D9
:1073E0009307D002A303F10A930770049794000057
:1073F0009384044BE3CEA7F7979400009384044A48
:107400006FF01FF7937BFDFD930710046390FB0A59
:10741000930700032304F10A13071006930780055E
:107420006314ED0093078007A304F10A9307300665
:107430001364240063D6674F93051B0013050900EE
:1074400023221101EFD05FE193040500832841005E
:10745000631E054C83D7C90093E707042396F90000
:1074600083D7C90093F70704E39807A68320C11CBC
:107470000324811C032581018324411C0329011C51
:107480008329C11B032A811B832A411B032B011B58
:10749000832BC11A032C811A832C411A032D011A44
:1074A000832DC1191301011D678000009307F0FFB0
:1074B0006302FB4893077004232201006394FB00DE
:1074C00063000B48832AC10D936704102320F10247
:1074D000232C0102032E010D832D410D832C810DE0
:1074E00063DA0A00B7070080B3CA57019307D002D6
:1074F000232CF102930710046398FB48130501093C
:10750000232411052328C109232C9109232AB10919
:10751000232E5109EF8090311306C10AEFF00FC5F9
:10752000138605009305050013050109EF80D00DB2
:107530008327010913060106930501072328F10695
:10754000832741091305010823200106232AF10698
:10755000832781092322010623240106232CF10617
:107560008327C109232EF106B707FC3F2326F10626
:10757000EF60400B03280108032641088326810899
:10758000832CC1089305010813050109232801096B
:1075900023220105232AC1082320C104232CD1085A
:1075A000232ED102232E9109232001082322010832
:1075B0002324010823260108EF50104E8326C1031F
:1075C000032601040328410483288104631605006F
:1075D000130710002326E10A13071006979A0000EC
:1075E000938A8A2D6316ED00979A0000938A8A2B5E
:1075F000130EFBFF938D0400B707034093050108AA
:107600002322C108130501091306010723241105CC
:107610002322C10523200109232EF1062324D108AA
:107620002326910923280106232A0106232C01067B
:10763000EF50507F032601098326410913050109F4
:107640002320C104232ED102EF80C04D93050500F5
:10765000130A050013050109832C8109032CC109B4
:10766000EF80806283270109032601048326C1037A
:107670002320F106832741092328C106930501072A
:107680002322F10683278109130601061305010849
:107690002324F1068327C109232C9107232E810778
:1076A0002326F106232AD106EF60D07BB3854A0159
:1076B00083C50500032E4104032CC108938D1D00D2
:1076C00083220108832F4108032F8108232EC10341
:1076D000A38FBDFE9307F0FF930C0C008328810459
:1076E000630CFE06130EFEFF930501081305010946
:1076F000232EE105232CF105232A5104232811050B
:107700002326C1052328510823245104232AF109E3
:107710002322F105232CE1092320E105232E8109F1
:10772000232001082322010823240108232601081D
:10773000EF50903683260104032641040328810478
:10774000032EC1048328010583224105832F81056F
:10775000032FC105E31205EAB70CFE3F93050108AC
:10776000130501092320110523285108232651045C
:10777000232AF1092324F105232CE1092322E10521
:10778000232E810923200108232201082324010834
:1077900023269109EF50103D832801046346A0047D
:1077A0008322C104832F8104032F41049305010820
:1077B0001305010923285108232AF109232CE10983
:1077C000232E8109232001082322010823240108F4
:1077D00023269109EF50502C83280104631C0518BF
:1077E000137A1A0063080A1803C6FA00232EB10B95
:1077F000930500038326C10B9387F6FF232EF10A1E
:1078000083C7F6FF6384C714130690036394C714F9
:1078100083C7AA00A38FF6FE138A0D001307700416
:10782000330A9A40832CC10A6392EB2A1307D0FFD4
:1078300063C4EC00635E9B31130DEDFF1387FCFF07
:107840002326E10A1376FDFD130510049376FD0F40
:10785000930500006318A6009386F60093F6F60FD2
:1078600093051000230AD10A9307B002635807005A
:1078700013071000330797419307D002A30AF10AB8
:107880009307900063D8E7289307310C938507008E
:10789000130590001308A000B36607031386F7FFD3
:1078A0003347070393860603A38FD7FE6346E52479
:1078B000130707039387E7FFA30FE6FE9306610B09
:1078C00063E0B7249307410BB387F6402328F10206
:1078D000338B47019307100063C647019377140069
:1078E0006386070083274101330BFB001374F4BF49
:1078F000936704102320F102130C0000930B000087
:10790000930C000083278103638607001307D002CE
:10791000A303E10A03240102930D00006F00404815
:10792000232201009304C1126FF0DFB92322A100CA
:107930006FF05FB923220100130B60006FF09FB856
:1079400023226101130B10006FF0DFB7A38FB6FE87
:107950006FF05FEA9387170093F7F70F6FF09FEBD5
:10796000130A1A00A30FEAFEB3074C41E3DA07FE3D
:107970006FF0DFEA8327C103138A0D0013070003AA
:10798000338CFD006FF05FFE93076004638EFB0095
:1079900093075004130C1B006384FB00130C0B00B3
:1079A000130620006F00C000130C0B0013063000FC
:1079B0009307010B1308C10B1307C10A93060C00B0
:1079C0009305010913050900232011052328C10986
:1079D000232EC103232AB109232C9109232E5109F7
:1079E000EFC01F919307700493040500032EC10399
:1079F000832801046396FB00937714006388070AC9
:107A000093076004338A84016392FB0603C7040072
:107A1000930700036318F704930501081305010990
:107A2000232011052328C109232EC103232AB109CC
:107A3000232C9109232E5109232001082322010818
:107A40002324010823260108EF501005032EC1034B
:107A5000832801046308050093071000338C8741D5
:107A60002326810B8327C10A330AFA0093050108F4
:107A700013050109232E11032328C109232AB10963
:107A8000232C9109232E51092320010823220108C8
:107A90002324010823260108EF5010008328C10386
:107AA00013070003631E0500232E410B032AC10B9D
:107AB0006FF0DFD693861700232ED10A2380E700CC
:107AC0008327C10BE3E847FF6FF05FFE13076004F5
:107AD000E396EBD66352900763160B0013771400FE
:107AE0006302070C832741013387FC00330BEB0053
:107AF000130D60066F004009930706006FF09FD9D1
:107B00009387170003C7F7FF93861600A38FE6FE3F
:107B10006FF01FDB9307610B639805009307000369
:107B2000230BF10A9307710B1307070393861700C2
:107B30002380E7006FF01FD963160B001377140042
:107B40006306070683274101138717006FF01FFAAA
:107B500063C04C0313771400138B0C0063060700FB
:107B600083274101338BFC00130D70066F00C001A9
:107B700083274101130D7006330BFA006346900111
:107B800033039B41130B1300937B0440130C000041
:107B9000E38A0BD6930B0000E35690D79306F00FC1
:107BA0006F008003138B0C006FF09FF4130D6006C1
:107BB000130B10006FF05FFD63569703832781005E
:107BC000B38CEC4003C717006308070293871700C4
:107BD000938B1B002324F1008327810003C7070038
:107BE000E31CD7FC8327410233878B013307F7025D
:107BF000330B67016FF01FD1130C1C006FF0DFFD1A
:107C000013874A002326E1001377040283A70A00A2
:107C1000630007020327810123A0E7001357F74100
:107C200023A2E700832AC100832401016FF0CFAEB5
:107C300013770401630807000327810123A0E700ED
:107C40006FF05FFE13770404630807000357810198
:107C50002390E7006FF01FFD13740420E30E04FC73
:107C6000034781012380E7006FF0DFFB1364040109
:107C70009377040263880704938A7A0093FA8AFF51
:107C800003AC0A0083AC4A0093878A002326F100E4
:107C90001374F4BF93070000A303010A1307F0FF56
:107CA000630CEB4213070400B3669C011374F4F7F2
:107CB0006394064263020B5A130710006392E74273
:107CC0006FF04FDA93874A002326F100937704017F
:107CD0006386070003AC0A006F0000019377040479
:107CE0006388070003DC0A00930C00006FF05FFA62
:107CF00093770420E38007FE03CC0A006FF0DFFED9
:107D000093874A002326F100B787FFFF93C70783B5
:107D10002314F10A979700009387C7B8232AF1022A
:107D200003AC0A00930C00001364240093072000A6
:107D3000130D80076FF05FF693874A002326F1004A
:107D4000A303010A9307F0FF2320110383A40A0071
:107D50006306FB0213060B00930500001385040065
:107D6000EFD01FC22322A10083280102630805E08F
:107D7000330B9540232201006FF04FE01385040080
:107D8000EFF00F8583280102130B05002322010069
:107D9000930D0000130C0000930B0000930C0000E7
:107DA0002320B10363D46D01232061030347710ACB
:107DB0006308070083270102938717002320F1023D
:107DC00093772400232CF1026388070083270102A4
:107DD000938727002320F102937A440863980A06C8
:107DE0008327C10103270102338EE7406350C00798
:107DF000130F0001979E0000938E8EFF930F70006B
:107E00008326810C23A0D8010327C10C938616007A
:107E100013868800634ACF473307EE0023A2C801C8
:107E20002326E10C2324D10C1307700093080600CD
:107E3000635ED7001306410C938509001305090002
:107E4000EF201076E314056C9308C10E0347710A06
:107E5000630807041307710A23A0E8001307100042
:107E600023A2E8000327C10C9306700093888800C2
:107E7000130717002326E10C0327810C13071700B3
:107E80002324E10C63DEE6001306410C9385090010
:107E900013050900EF20D070E31A05669308C10EA0
:107EA00083278103638807041307810A23A0E8005E
:107EB0001307200023A2E8000327C10C93067000DB
:107EC00093888800130727002326E10C0327810CE1
:107ED000130717002324E10C63DEE6001306410CB0
:107EE0009385090013050900EF20906BE3100562EC
:107EF0009308C10E130700086398EA068327C1019F
:107F000003270102B38AE74063505007130E0001B4
:107F1000979700009387C7EE930E70008326810C1D
:107F200023A0F8000327C10C93861600138688004F
:107F300063485E3B3387EA0023A258012326E10C05
:107F40002324D10C1307700093080600635ED7004A
:107F50001306410C9385090013050900EF205064B6
:107F6000E316055A9308C10EB38A6D41635050075A
:107F700013080001979D0000938D8DE8130E70008B
:107F80000327810C23A0B8018326C10C1307170017
:107F900013868800634E583923A25801B38ADA0049
:107FA0002326510D2324E10C93067000930806004C
:107FB00063DEE6001306410C9385090013050900F2
:107FC000EF20105EE31405549308C10E13770410DC
:107FD000832DC10C6312073A3303BB0123A0980021
:107FE00023A268012326610C8327810C13077000EC
:107FF00093888800938717002324F10C6352F74C71
:108000001306410C9385090013050900EF20505910
:10801000E31E054E9308C10E6F00804A13640401ED
:108020009377040263820702938A7A0093FA8AFFA5
:1080300003AC0A0083AC4A0093878A002326F10030
:10804000930710006FF05FC593874A002326F10065
:10805000937704016386070003AC0A006F000001F8
:10806000937704046388070003DC0A00930C000084
:108070006FF01FFD93770420E38007FE03CC0A0016
:108080006FF0DFFE979700009387C7816FE01FF7BF
:1080900093874A002326F100937704016386070043
:1080A00003AC0A006F0000019377040463880700A3
:1080B00003DC0A00930C00006FE0DFF693770420E6
:1080C000E38007FE03CC0A006FF0DFFE1307040015
:1080D000930710006FF05FBD13071000638EE796E3
:1080E00013072000638EE712930701199396DC01B2
:1080F00013777C00135C3C001307070333EC860105
:1081000093DC3C00A38FE7FEB3669C019384F7FFEA
:10811000639E060293761400638A060093060003AA
:108120006306D700A38FD4FE9384E7FF930701195A
:10813000930D0B0023220100338B9740130C00009A
:10814000930B0000930C00006FF09FC59387040011
:108150006FF0DFF9130A0000930D0119937A0440C0
:10816000930B90001306A0009306000013050C006B
:1081700093850C0023221101EF40400513050503F0
:10818000A38FADFE9384FDFF130A1A0083284100DC
:10819000638E0A048327810083C707006318FA04EB
:1081A0009307F00F6304FA0463940C0063F08B05EB
:1081B000832741028325C10223221101B384F440A5
:1081C0001386070013850400EFE05FC28327810058
:1081D000130A00008328410083C717006388070043
:1081E00083278100938717002324F10013050C00D7
:1081F00093850C001306A0009306000023221101B2
:10820000EF309039938C0500B3E5A500130C050001
:1082100083284100E38C05F0938D04006FF09FF4F8
:1082200093040119032741039377FC009384F4FF1F
:10823000B307F70083C70700135C4C002380F400EA
:108240009397CC0133EC870193DC4C00B3679C011E
:10825000E39A07FC6FF09FED93040119E39807EC94
:1082600013771700E30407EC93070003A307F11843
:108270006FE0DFFFE30E0D2E2306A113A303010A17
:10828000232651016FE0DFF61307070123A2E8015F
:108290002326E10C2324D10C63DEDF021306410CFC
:1082A00093850900130509002324F1052322D10534
:1082B0002320E105232EC103EF20902EE31805248F
:1082C000832F8104832E4104032F0104032EC10355
:1082D0001306C10E130E0EFF930806006FF05FB277
:1082E0001307070123A2C8012326E10C2324D10C84
:1082F00063DADE021306410C9385090013050900B9
:108300002320D105232EF102232CC103EF20502975
:10831000E31E051E832E01048327C103032E810360
:108320001306C10E938A0AFF930806006FF01FBF61
:108330009386060123A208012326D10C2324E10CF5
:108340006356EE021306410C9385090013050900DC
:10835000232EC103232C0103EF209024E318051AD8
:10836000032EC103032881031306C10E938A0AFF5B
:10837000930806006FF0DFC0130750066354A7731D
:108380000327010D93050108130501092328E108BE
:108390000327410D232C110323200108232AE10880
:1083A0000327810D2322010823240108232CE1083F
:1083B0000327C10D23260108232EE108EF40D06DCD
:1083C000832881036314051897870000938707505B
:1083D00023A0F8009307100023A2F8008327810C44
:1083E000938D1D002326B10D938717002324F10CD4
:1083F0001307700093888800635EF7001306410C32
:108400009385090013050900EF209019E31005106A
:108410009308C10E8327C10A63C6470193771400EE
:108420006380070A8327810203274101938888001C
:1084300023ACF8FE8327410123AEF8FE8327C10C4D
:10844000B387E7002326F10C8327810C1307700004
:10845000938717002324F10C635EF7001306410C89
:108460009385090013050900EF209013E310050A16
:108470009308C10E9304FAFF63549004930B000118
:10848000979A0000938ACA97130C70008327810C77
:1084900023A058010327C10C9387170093868800F7
:1084A00063CA9B0623A29800B384E4002326910CA0
:1084B0002324F10C1307700093880600E342F7B4FD
:1084C000137444006314047E032DC1018327010249
:1084D0006354FD00138D070083278101B387A70133
:1084E000232CF1008327C10C638C07001306410C79
:1084F0009385090013050900EF20900AE318050091
:10850000832741002324010CE39C07049308C10E38
:108510006FF04FF11307070123A278012326E10C26
:108520002324F10C635EFC001306410C93850900C3
:1085300013050900EF20D006631A057C9306C10ECF
:10854000938404FF938806006FF05FF40327C10A49
:108550006346E016978700009387473723A0F8000B
:108560009307100023A2F8008327810C938D1D0030
:108570002326B10D938717002324F10C13077000F5
:1085800093888800635EF7001306410C9385090009
:1085900013050900EF20D000631A05769308C10E79
:1085A0008327C10A6398070063160A0093771400B3
:1085B000E38807F08327810203274101938888001D
:1085C00023ACF8FE8327410123AEF8FE8327C10CBC
:1085D000B387E7002326F10C8327810C1307700073
:1085E000938717002324F10C635EF7001306410CF8
:1085F0009385090013050900EF20807A6318057040
:108600009308C10E832AC10A63D20A06B30A5041F5
:1086100013870800130C0001978B0000938B4B7E8F
:10862000130D70008327810C232077018326C10C52
:10863000938717009388880063465C0523225701BF
:10864000B38ADA002326510D2324F10C130770009E
:10865000635EF7001306410C9385090013050900BA
:10866000EF2000746314056A9308C10E8327C10CC0
:1086700023A0980023A24801B38747012326F10CC9
:108680006FF09F9693860601232287012326D10C43
:108690002324F10C635EFD001306410C9385090051
:1086A00013050900EF20C06F631205669308C10E21
:1086B000938A0AFF138708006FF0DFF6938A0C0095
:1086C00063549A01930A0A00635250050327810CF0
:1086D000B38DBA0123A098001307170023A25801F5
:1086E0002326B10D2324E10C9306700093888800A3
:1086F00063DEE6001306410C9385090013050900AB
:10870000EF20006A631405609308C10E63D40A0069
:10871000930A0000B38A5C4163505007930D000137
:10872000178D0000130DCD6D130B70000327810C06
:1087300023A0A8018326C10C130717001386880005
:1087400063C25D1B23A25801B38ADA002326510DB0
:108750002324E10C930670009308060063DEE60014
:108760001306410C9385090013050900EF204063AF
:10877000631E05589308C10E93770440B38A940191
:1087800063840702130D7000338B4401978D000042
:10879000938D0D6763940B1863140C18B387440111
:1087A00063F45701938A07008327C10A63C6470110
:1087B00093771400638A070483278102032741010A
:1087C0009388880023ACF8FE8327410123AEF8FE8E
:1087D0008327C10CB387E7002326F10C8327810C84
:1087E00013077000938717002324F10C635EF700D2
:1087F0001306410C9385090013050900EF20405A28
:10880000631605509308C10EB3844401B3875441E5
:108810008324C10AB3049A4063D497009384070069
:10882000635490048327C10C23A0580123A298000D
:10883000B387F4002326F10C8327810C1307700003
:1088400093888800938717002324F10C635EF70058
:108850001306410C9385090013050900EF204054CD
:108860006316054A9308C10E9387040063D404007D
:10887000930700008324C10AB3049A40B384F440F0
:10888000E35090C4930B0001978A0000938A4A57E3
:10889000130C70008327810C23A058010327C10CFF
:1088A0009387170093868800E3DE9BBE13070701BA
:1088B00023A278012326E10C2324F10C635EFC0043
:1088C0001306410C9385090013050900EF20404D64
:1088D000631E05429306C10E938404FF938806002D
:1088E0006FF05FFB9386060123A2B8012326D10C0B
:1088F0002324E10C635EEB001306410C9385090011
:1089000013050900EF20C049631205401306C10E8C
:10891000938A0AFF930806006FF05FE163020C0E72
:10892000130CFCFF8327C1020327410293888800B0
:1089300023ACF8FE8327410223AEF8FE8327C10C47
:10894000B387E7002326F10C8327810C9387170058
:108950002324F10C635EFD001306410C938509008E
:1089600013050900EF20C0436312053A9308C10EB6
:108970008327810033075B4183C707006354F700F7
:10898000930707006356F0040327C10C23A0580186
:1089900023A2F8003387E7002326E10C0327810C8C
:1089A00093888800130717002324E10C6352ED021B
:1089B0001306410C9385090013050900232CF102CD
:1089C000EF20003E63140534832781039308C10E12
:1089D0001387070063D40700130700008327810073
:1089E0001308000183C70700B387E7406346F0061A
:1089F0008327810083C70700B38AFA006FF09FD9ED
:108A000083278100938BFBFF9387F7FF2324F100DB
:108A10006FF05FF19386060123A208012326D10C93
:108A20002324E10C6356ED021306410C93850900E3
:108A300013050900232E0103232CF102EF204036F9
:108A40006316052C0328C103832781031306C10E77
:108A5000938707FF930806000327810C23A0B80122
:108A60008326C10C1307170013868800E344F8FA25
:108A700023A2F800B387D7002326F10C2324E10CAE
:108A800093080600E356EDF61306410C93850900A2
:108A900013050900EF20C030631A05269308C10EA4
:108AA0006FF01FF58327810C1307100023A0980097
:108AB000938D1D0093871700938B880063464701B1
:108AC000937614006388061C1307100023A2E800A5
:108AD0002326B10D2324F10C13077000635EF70009
:108AE0001306410C9385090013050900EF20402B64
:108AF000631E0520930BC10E8327810203274101CA
:108B0000938B8B0023ACFBFE8327410123AEFBFE3E
:108B10008327C10CB387E7002326F10C8327810C40
:108B200013077000938717002324F10C635EF7008E
:108B30001306410C9385090013050900EF20402618
:108B40006316051C930BC10E8327010D93050108C5
:108B5000130501092328F1088327410D930AFAFF21
:108B600023200108232AF1088327810D23220108ED
:108B700023240108232CF1088327C10D2326010893
:108B8000232EF108EF404071630605088327C10CCE
:108B90000327810C938414009387F7FFB387470161
:108BA0001307170023A09B0023A25B012326F10CCF
:108BB0002324E10C93077000938B8B0063DEE700A6
:108BC0001306410C9385090013050900EF20401D91
:108BD000631E0512930BC10E9307410B23A0FB00EC
:108BE000832701030327010393888B0023A2FB0043
:108BF0008327C10CB387E7002326F10C8327810C60
:108C000013077000938717002324F10CE35AF78AA7
:108C10006FF00FBFE35250FD130C0001978400006A
:108C20009384041E130D70000327810C23A09B0066
:108C30008327C10C1307170093868B0063405C03E6
:108C4000B387FA0023A25B012326F10C2324E10C55
:108C500093077000938B06006FF05FF69387070110
:108C600023A28B012326F10C2324E10C635EED008B
:108C70001306410C9385090013050900EF204012EB
:108C8000631605089306C10E938A0AFF938B0600AC
:108C90006FF09FF923A2E8002326B10D2324F10CE5
:108CA00013077000E35AF7F26FF09FF18327C101B9
:108CB000032701023384E740E3588080930A0001D0
:108CC000978400009384C412930B70008327810C57
:108CD00023A098000327C10C9387170063C68A045A
:108CE00023A288003304E4002326810C2324F10C02
:108CF00013077000635AF7FC1306410C93850900B3
:108D000013050900EF20C009630005FC832741001B
:108D1000639407006FE0CFF4938507001305090003
:108D2000EF90DFE86FE0CFF31307070123A25801AC
:108D30002326E10C2324F10C9388880063DEFB00DA
:108D40001306410C9385090013050900EF20400527
:108D5000E31E05FA9308C10E130404FF6FF01FF71A
:108D60008325410013050900EF905FE46FF00FFACF
:108D70008327C10C639407006FE08FEE1306410C4C
:108D80009385090013050900EF2080016FE04FED86
:108D900083278600130101FD23248102232611026B
:108DA0002322910223202103232E3101232C410170
:108DB000232A5101232861012326710123248101E3
:108DC00013040600639E0702232206001305000019
:108DD0008320C1020324810283244102032901026A
:108DE0008329C101032A8101832A4101032B010147
:108DF000832BC100032C8100130101036780000055
:108E000083A745061389050013972701635A0706B0
:108E100083240600130A0500930BF0FF83278400C8
:108E2000639A070013050000232404002322040092
:108E30006FF01FFA83A9440003AB0400930A0000FB
:108E400013DC290063CE8A018327840093F9C9FFCC
:108E500093848400B3893741232434016FF01FFCCD
:108E600083250B001306090013050A00EF1080127A
:108E7000130B4B00630A7501938A1A006FF09FFC75
:108E8000EF10C01E6FF05FFA1305F0FF6FF0DFF90F
:108E9000130101ED2324811223202113232E3111EC
:108EA000232C41112326111223229112232A51111E
:108EB000232861112326711123248111232291116A
:108EC0002320A111232EB10F93090500138405005F
:108ED000130A06001389060063080500832785032B
:108EE00063940700EF90DF9E8317C4001397270158
:108EF00063420702B726000003274406B3E7D70002
:108F00002316F400B7E7FFFF9387F7FFB377F70067
:108F10002322F4068357C40093F78700638E070665
:108F200083270401638A07068357C4001307A00040
:108F300093F7A701639EE7068317E40063CA070659
:108F40009306090013060A0093050400138509001F
:108F5000EF00503F930B05008320C11203248112C0
:108F600013850B0083244112032901128329C111A7
:108F7000032A8111832A4111032B0111832BC11074
:108F8000032C8110832C4110032D0110832DC10F60
:108F90001301011367800000930504001385090085
:108FA000EF904FC4E30205F8930BF0FF6FF0DFFA88
:108FB000130BC1042320610523240104232201048F
:108FC00013070B002328010023260100232A010098
:108FD000232C0100930B000093040A009306500217
:108FE00083C70400638407006394D70AB38A4441AB
:108FF00063860A0483278104232047012322570123
:10900000B38757012324F10483274104930670009A
:1090100013078700938717002322F10463DEF6000D
:10902000130601049305040013850900EFF05FD6D1
:10903000E31A052813070B00B38B5B0183C70400F9
:10904000E386072C138A1400A30D01029304F0FF9A
:10905000930A0000130D0000130C90001305A005E7
:109060001308A00203460A00130A1A00930606FE1C
:10907000E36AD50E97870000938787D993962600D9
:10908000B386F60083A60600B386F6006780060066
:10909000938414006FF0DFF4978700009387C781F3
:1090A0002328F10093760D026388066C130979007A
:1090B000137989FF83280900832C4900130C890048
:1090C00093761D00638E0600B3E69801638A06005E
:1090D00093060003230ED102A30EC102136D2D00CF
:1090E000137DFDBF6F004032138509002324E1008A
:1090F000EFB0DFEA8327450013850700232CF1003A
:10910000EFD01FCD232AA10013850900EFB01FE97E
:1091100083278500032781002326F100832741014F
:10912000E38E07F28327C100E38A07F283C60700B4
:10913000E38606F2136D0D406FF05FF28346B103D4
:10914000E39E06F093060002A30DD1026FF01FF11B
:10915000136D1D006FF09FF0832A09001309490069
:10916000E3DE0AEEB30A5041136D4D006FF01FEFBE
:109170009306B0026FF05FFD03460A0093061A00E3
:1091800063120605832409001306490063D4040012
:109190009304F0FF13090600138A06006FF01FEC1A
:1091A0009307A000B384F4029386160003C6F6FF6B
:1091B000B384B400930506FDE374BCFE138A060075
:1091C0006FF0DFEA930400006FF0DFFE136D0D080F
:1091D0006FF0DFE893060A00930A00009307A000EF
:1091E000B38AFA02130606FD93861600B30A5601E7
:1091F00003C6F6FF930506FDE372BCFE6FF01FFC8D
:1092000003460A00930680066318D600130A1A0064
:10921000136D0D206FF09FE4136D0D046FF01FE4CC
:1092200003460A009306C0066318D600130A1A0004
:10923000136D0D026FF09FE2136D0D016FF01FE2D1
:1092400083260900130C4900A30D01022306D1084F
:1092500093041000930C00001309C1086F00C01E96
:10926000136D0D0193760D02638C060413097900CA
:10927000137989FF83280900832C4900130C890086
:1092800063DE0C00B3081041B33610013303904184
:10929000B30CD3409306D002A30DD1029306F0FF86
:1092A0006398D45063920C589306900063EE16575F
:1092B00093880803A307110F1309F10E6F0040559F
:1092C00093760D01130C490063880600832809007A
:1092D00093DCF8416FF0DFFA93760D0483280900E0
:1092E000638806009398080193D808416FF05FFEE9
:1092F00093760D20E38E06FC9398880193D88841DD
:109300006FF01FFD13760D02832609001309490033
:10931000630A060093D7FB4123A0760123A2F6003F
:109320006FF09FCB13760D016306060023A0760134
:109330006FF09FCA13760D04630606002390760132
:109340006FF09FC993770D20E38207FE238076019B
:109350006FF09FC8136D0D0193760D0263860604AE
:1093600013097900137989FF83280900832C4900A8
:10937000130C8900137DFDBF93060000A30D0102AD
:109380001306F0FF638CC44213060D00B3E5980189
:10939000137DFDF7639405426388045A1306100099
:1093A0006392C6426FF0DFF093760D01130C490013
:1093B00063860600832809006F00000193760D0480
:1093C0006388060083580900930C00006FF09FFA31
:1093D00093760D20E38006FE834809006FF0DFFEE0
:1093E000B786FFFF8328090093C60683977700009E
:1093F0009387474B130C4900930C0000136D2D000D
:10940000231ED1022328F100930620006FF01FF7DE
:10941000A30D01029306F0FF2324E100130C490081
:10942000032909006388D42C1386040093050000E7
:1094300013050900EFC0CFD4930C0000032781006F
:1094400063040500B30425412324910163D49C00E7
:10945000232491008346B10363880600832781009B
:10946000938717002324F100937D2D0063880D005E
:1094700083278100938727002324F10093774D08E9
:10948000232EF1006396070683278100B386FA40F6
:109490006350D0069308000117880000130808AE37
:1094A0001303700003264104232007018325810450
:1094B000130616001305870063C0D84C2322D7007B
:1094C000B386B6002324D1042322C104930670007E
:1094D0001307050063DEC6001306010493050400AC
:1094E00013850900EFF0DF8A631E055C13070B008C
:1094F0008346B103638806041306B1032320C70023
:1095000013061000832641042322C700032681048A
:10951000938616002322D104130616002324C104C7
:109520001306700013078700635ED600130601045C
:109530009305040013850900EFF09F856314055817
:1095400013070B0063880D041306C1032320C70013
:1095500013062000832641042322C700032681042A
:10956000938616002322D104130626002324C10467
:109570001306700013078700635ED600130601040C
:109580009305040013850900EFF09F80631C0552CA
:1095900013070B008327C101930600086396D706C3
:1095A00083278100B38DFA406350B0079308000110
:1095B000178800001308889D130370008326410458
:1095C0002320070103268104938616009305870054
:1095D00063C0B8412322B701B38DCD002324B10568
:1095E0002322D1041306700013870500635ED600A2
:1095F000130601049305040013850900EFF04FF9E9
:109600006312054C13070B00B38C9C40635090070A
:1096100013080001978D0000938D4D9793087000FB
:10962000832641042320B701032681049386160074
:10963000930587006346983F23229701B38CCC00A3
:10964000232491052322D1041306700013870500FB
:10965000635ED60013060104930504001385090018
:10966000EFF00FF36310054613070B008326810408
:109670002322970023202701B384960083264104E8
:109680002324910413067000938616002322D1042C
:1096900013078700635ED6001306010493050400D8
:1096A00013850900EFF0CFEE631E054013070B0092
:1096B00093774D00639A073A8327810063D4FA00B9
:1096C000938A070083278104B38B5B01638C0700B7
:1096D000130601049305040013850900EFF04FEB16
:1096E0006312053E2322010413090C0013070B002B
:1096F0006FF09F8E13050900EFD08FED93040500E6
:10970000930C0000032781006FF01FD4136D0D012F
:1097100093760D026380060213097900137989FF9D
:1097200083280900832C4900130C8900930610003C
:109730006FF0DFC493760D01130C490063860600B9
:10974000832809006F00000193760D0463880600EA
:1097500083580900930C00006FF05FFD93760D2095
:10976000E38006FE834809006FF0DFFE9777000074
:10977000938747136FF0DF9293760D01130C490026
:1097800063860600832809006F00000193760D04AC
:109790006388060083580900930C00006FF05F9205
:1097A00093760D20E38006FE834809006FF0DFFE0C
:1097B00013060D00930610006FF05FBD1306100036
:1097C000E382C6AE130620006384C6149306010F1D
:1097D0009395DC0113F6780093D83800130606033E
:1097E000B3E8150193DC3C00A38FC6FEB3E59801F6
:1097F0001389F6FF6396050293751D00638A0500C1
:10980000930500036306B600A30FB9FE1389E6FFB4
:109810009307010F938C0400B38427416FF0DFC2DC
:10982000930609006FF0DFFA93770D40930D000067
:10983000130E010F2324F100138508001306A00066
:109840009306000093850C002322E1021309FEFF1A
:109850002320C103232E1101EF205017032E0102F4
:109860008327810013050503A30FAEFE938D1D0012
:109870008328C10103274102638207068327C100B1
:1098800083C60700639CB6059307F00F6388FD0449
:1098900063960C009307900063F21705832741013C
:1098A00083258101232011033309F9401386070022
:1098B00013050900232EE100EFD04FD38327C10009
:1098C000930D00000327C10183C6170083280102FE
:1098D00063860600938717002326F100138508008E
:1098E00093850C001306A00093060000232EE100D0
:1098F000EF20804A938C0500B3E5A500930805008E
:109900000327C101E38605F0130E09006FF0DFF2B3
:109910001309010F8327010193F6F8001309F9FFDA
:10992000B386D70083C6060093D848002300D90029
:109930009396CC01B3E8160193DC4C00B3E6980192
:10994000E39A06FC6FF0DFEC1309010FE39206ECDB
:1099500013761600E30E06EA93060003A307D10E62
:109960006FF09F956304061A2306C108A30D010238
:10997000130C09006FF0DF8D938505012322170179
:109980002324B1042322C104635EC302130601042D
:109990009305040013850900232661022324010393
:1099A000232211032320D102EFF08FBE631C051088
:1099B0000323C10203288102832841028326010276
:1099C00013050B00938606FF130705006FF09FAD8C
:1099D00013060601232217012324C1042322D104E4
:1099E000635AD3021306010493050400138509008A
:1099F0002322610223200103232E1101EFF04FB92E
:109A00006312050C03234102032801028328C101CC
:109A100093050B00938D0DFF138705006FF01FBAA0
:109A200013060601232207012324C1042322D104A3
:109A300063D6D802130601049305040013850900B8
:109A400023201103232E0101EFF08FB4631C0506C0
:109A5000832801020328C10193050B00938C0CFF9E
:109A6000138705006FF0DFBB83278100B384FA40C2
:109A7000E35490C4930C00011779000013090950B6
:109A8000930D70008327410423202701832681043E
:109A90009387170063C09C0423229700B384D400EB
:109AA000232491042322F10413077000E356F7C026
:109AB000130601049305040013850900EFF04FAD70
:109AC000E30C05BE8357C40093F70704638607C8F9
:109AD0006FF08FCD93860601232297012324D104B2
:109AE0002322F1041307870063DEFD00130601043F
:109AF0009305040013850900EFF08FA9E31405FC1A
:109B000013070B00938404FF6FF0DFF783278104B2
:109B1000E38A07FA1306010493050400138509007C
:109B2000EFF00FA76FF01FFA978700009387873D2C
:109B300093060600138605009305050003A507009C
:109B40006FF00FB583D7C500130101B8232C8146F0
:109B500093F7D7FF231AF10083A745061384050066
:109B6000232A91462326F10683D7E500232821479F
:109B7000232E1146231BF10083A7C50113090500FD
:109B8000232001022322F10283A7450293058100CD
:109B90002326F102930701072324F100232CF1006F
:109BA000930700402328F100232EF100EFF04FAE81
:109BB00093040500634C050093058100130509001B
:109BC000EF809FB6630405009304F0FF83574101C3
:109BD00093F70704638807008357C40093E70704DB
:109BE0002316F4008320C147032481471385040012
:109BF000032901478324414713010148678000007E
:109C0000978700009387073083A7070083A7470340
:109C10006396070097870000938747D703A3070E33
:109C200067000300638405029307F00F63FAC7001F
:109C30009307A0082320F5001305F0FF67800000BC
:109C40002380C50013051000678000001305000085
:109C500067800000130101FF232481001304050025
:109C600013850500930506001386060097870000FC
:109C700023AE072C23261100EF60901B9307F0FF03
:109C8000631CF500978700009387472C83A7070084
:109C9000638407002320F4008320C1000324810093
:109CA0001301010167800000B385C502130101FFA4
:109CB0002324810023261100EFB00FDA13040500DE
:109CC000630205040326C5FF130740021376C6FF8F
:109CD0001306C6FF6362C7069306300193070500AB
:109CE00063FCC60023200500232205009307B00172
:109CF00063E4C7029307850023A0070023A207009F
:109D000023A40700130504008320C100032481005D
:109D100013010101678000002324050023260500AC
:109D200093070501E31AE6FC232805009307850144
:109D3000232A05006FF05FFC93050000EFB09FC67B
:109D40006FF05FFC130101FF232481001304050061
:109D5000138505009787000023AA071E23261100FC
:109D6000EF6000679307F0FF631CF5009787000022
:109D70009387C71D83A70700638407002320F4008F
:109D80008320C100032481001301010167800000CA
:109D9000130101FF232611002324810023229100B7
:109DA0002320210163920502130900008320C100D2
:109DB00003248100130509008324410003290100C5
:109DC000130101016780000093040500138405005E
:109DD000630805008327850363940700EF805FAF66
:109DE0008317C400E38207FC930504001385040075
:109DF000EF800FF38327C40213090500638C07006B
:109E00008325C40113850400E7800700635405001F
:109E10001309F0FF8357C40093F70708638807000E
:109E20008325040113850400EF805FD88325040394
:109E3000638C0500930704046386F5001385040012
:109E4000EF80DFD6232804028325440463880500BD
:109E500013850400EF809FD523220404EF809FBE6A
:109E600023160400EF805FBE6FF05FF49787000059
:109E7000938747099305050003A507006FF05FF17D
:109E8000130101FD2324810223229102232C41018D
:109E90002326110223202103232E3101232A5101DD
:109EA00023286101130A05009384050013040600AA
:109EB000EFB04F9B93071000631AF5049387F4FFEC
:109EC0001307E00F6364F704230691009309100061
:109ED00013090000930AF0FF130BA0006312390767
:109EE000138504008320C1020324810283244102DC
:109EF000032901028329C101032A8101832A410127
:109F0000032B010113010103678000009306C405C0
:109F1000138604009305C10013050A00EF10105DBD
:109F20009307F0FF93090500E314F5FA8357C40083
:109F300093E707042316F4001305F0FF6FF09FFA70
:109F40009307C100B387270183C5070083278400D7
:109F50009387F7FF2324F40063D8070003278401C5
:109F600063C0E702638E650183270400138717002F
:109F70002320E4002380B700130919006FF01FF6B7
:109F80001306040013050A00EF10D041E31655FF35
:109F90006FF09FFA8317C6001397270163400702EB
:109FA00003274606B7260000B3E7D7002316F600BE
:109FB000B7270000B367F7002322F6066FF05FECC7
:109FC000130101FE978700009387C7F3232C8100BC
:109FD00003A40700232A9100232E110093040500F7
:109FE00013860500630E040083278403639A070029
:109FF000130504002326B100EF809F8D0326C100C6
:10A0000013050400032481018320C101938504000A
:10A0100083244101130101026FF0DFF7130101FFF7
:10A020002324810013040500138505009305060011
:10A030009787000023AC07F023261100EF60803ED5
:10A040009307F0FF631CF50097870000938707F0E4
:10A0500083A70700638407002320F4008320C10046
:10A06000032481001301010167800000832786001B
:10A0700063980700930700001385070067800000BE
:10A0800083D7C500130101FB23248104232021056C
:10A09000232A51032326110423229104232E310362
:10A0A000232C4103232861032326710323248103E6
:10A0B000232291032320A103232EB10193F78700CC
:10A0C000930A060013840500130905006382070E36
:10A0D00083A70501638E070C8357C40003AA0A00F7
:10A0E00013F72700631A071693F7170063840720F6
:10A0F000930B000013050000130B000093090000F0
:10A100006384093663120502138609009305A000D3
:10A1100013050B00EFB0DF86938B19006306050073
:10A1200013051500B30B6541138C0B0063F4790123
:10A13000138C0900032504008327040183264401AE
:10A1400063FEA73283248400B384960063D88433EB
:10A1500093050B0013860400EF00C04F8327040013
:10A160009305040013050900B38797002320F4002A
:10A17000EF808FDB63160516B38B9B401305100031
:10A18000639A0B009305040013050900EF80CFD9F3
:10A190006318051483A78A00330B9B00B389994089
:10A1A000B384974023A49A00E39C04F46F008006D4
:10A1B0009305040013050900EF80CFA29307F0FF79
:10A1C000E30C05F06F00400583290A0083244A0050
:10A1D000130A8A00E38A04FE9386040063749B00DA
:10A1E00093060B00832744028325C40113860900CC
:10A1F00013050900E78007006354A00E83A78A00B7
:10A20000B389A900B384A4403385A74023A4AA003E
:10A21000E31205FC930700008320C104032481049A
:10A2200083244104032901048329C103032A8103F0
:10A23000832A4103032B0103832BC102032C8102D8
:10A24000832C4102032D0102832DC10113850700D8
:10A250001301010567800000370B0080930900009F
:10A2600093040000134B0BC06FF0DFF6032B0A00C2
:10A2700083244A00130A8A00E38A04FE0357C400B9
:10A28000832784000325040093760720638806143F
:10A2900063E2F40C93760748638E060A832D44012B
:10A2A00083250401B38DBC03B309B540938719001E
:10A2B000B3879700B3CDAD0363F4FD00938D070022
:10A2C000137707406304070E93850D0013050900FB
:10A2D000EFA09FF8631005049307C0002320F90046
:10A2E0008357C40093E707042316F4009307F0FF95
:10A2F0006FF09FF2B70B008013CCEBFF130B000045
:10A300009304000093CBFBFF930C3000130D20004F
:10A310006FF09FF683250401138609002326A10010
:10A32000EF00C0240357C4008327C1001377F7B799
:10A33000136707082316E4002328F400232AB40136
:10A34000B3873701B38D3D412320F4002324B401AA
:10A35000938704009389040063F4F4009387040056
:10A36000032504001386070093050B002326F10044
:10A37000EF00402E032784008327C1003307F740F6
:10A380002324E40003270400B307F7002320F4008C
:10A3900083A78A00330B3B01B3843441B38937412F
:10A3A00023A43A01E39A09EC6FF0DFE613860D006F
:10A3B00013050900EF00803493070500E31E05F63E
:10A3C0008325040113050900EF804FFE8357C40065
:10A3D00093F7F7F72316F4006FF01FF0032704013B
:10A3E0006366A7008326440163F6D40493890700BB
:10A3F00063F4F400938904001386090093050B00AD
:10A40000EF0040258327840003270400B3873741EA
:10A41000330737012324F4002320E400E39A07F6EE
:10A420009305040013050900EF800FB0E30205F661
:10A430006FF01FEB93870B0063649C00938704000D
:10A44000B3C7D702032744028325C40113060B00B8
:10A4500013050900B386D702E7000700930905003A
:10A46000E348A0F26FF0DFE7032B0A0083294A00DC
:10A4700013050000130A8A006FF09FC86342DC02D4
:10A48000832744028325C40113060B00130509002A
:10A49000E780070093040500E340A0CE6FF05FE47F
:10A4A00013060C0093050B00EF00C01A83278400ED
:10A4B00093040C00B38787412324F400832704000E
:10A4C000B38787012320F4006FF01FCB130101FF36
:10A4D00023248100130405001385050097870000DD
:10A4E00023A607A623261100EF50907A9307F0FFCA
:10A4F000631CF50097870000938747A583A7070093
:10A50000638407002320F4008320C100032481001A
:10A510001301010167800000130101FF2324810062
:10A520001304050013850500930506001386060035
:10A530009787000023AC07A023261100EF50507826
:10A540009307F0FF631CF50097870000938707A02F
:10A5500083A70700638407002320F4008320C10041
:10A56000032481001301010167800000B3C7A50027
:10A5700093F737003307C500639607009307300051
:10A5800063E4C70293070500636CE5006780000081
:10A5900083C605009387170093851500A38FD7FE08
:10A5A000E3E8E7FE678000009377350063920708D1
:10A5B000930705009376C7FF138606FE63F6C70868
:10A5C00083A3050083A2450083AF850003AFC500C8
:10A5D00083AE050103AE450103A3850183A8C50130
:10A5E000938545029387470203A8C5FF23AE77FCF6
:10A5F00023A057FE23A2F7FF23A4E7FF23A6D7FF3C
:10A6000023A8C7FF23AA67FE23AC17FF23AE07FFCB
:10A610006FF0DFFA83C60500938717009385150056
:10A62000A38FD7FE93F63700E39606FE6FF09FF8F0
:10A63000930705006FF01FFF03A6050093874700EF
:10A640009385450023AEC7FEE3E8D7FEE3EAE7F4CF
:10A65000678000003307C50063E8A5009307050085
:10A66000639AE70267800000B387C5003306F640AF
:10A67000E376F5FEB386C7006394060067800000AA
:10A680009387F7FF83C607001307F7FF2300D70060
:10A690006FF05FFE9385150083C6F5FF9387170063
:10A6A000A38FD7FE6FF0DFFB130101FF232481008E
:10A6B00013040500138505009305060013860600A4
:10A6C0009787000023A4078823261100EF50106409
:10A6D0009307F0FF631CF5009787000093870787B7
:10A6E00083A70700638407002320F4008320C100B0
:10A6F000032481001301010167800000130101FCA4
:10A70000232C8102232E110213840500232A910297
:10A710002328210323263103232441032322510329
:10A7200023206103232E71019305060063180402A0
:10A73000032481038320C1038324410303290103EC
:10A740008329C102032A8102832A4102032B0102C9
:10A75000832BC101130101046FA01FB0930A0500F0
:10A760002326C100EFB0CFB18325C1008326C4FFEB
:10A77000930760019389B500930B84FF13F9C6FF1B
:10A7800063F4370513FB89FF63520B049307C00082
:10A7900023A0FA00130A00008320C10303248103CD
:10A7A00013050A0083244103032901038329C102FD
:10A7B000032A8102832A4102032B0102832BC10158
:10A7C0001301010467800000130B0001E360BBFC70
:10A7D000635E694517770000130707320326870079
:10A7E000B3872B0103A74700630CF6001375E7FF3F
:10A7F0003385A7000325450013751500631C050A62
:10A800001377C7FFB309E9006312F60413050B01C0
:10A8100063C6A90AB38B6B01B389694197770000BE
:10A8200023A0772F93E9190023A23B018329C4FFBA
:10A8300013850A00130A040093F91900B3E96901AA
:10A84000232E34FFEFB00FA46FF01FF563C8690724
:10A8500003A7C70083A7870023A6E7002324F700E8
:10A8600003A74B00B38669411306F0001377170066
:10A87000B3873B016370D63CB369EB0023A23B0175
:10A88000B3856B0193E6160023A2D50003A747000A
:10A890009385850013850A001367170023A2E7003C
:10A8A000EF80CFB013850A00EFB0CF9D138A8B00E5
:10A8B0006FF09FEE130700009307000093F6160059
:10A8C00063940628832484FFB3849B4003AA440036
:10A8D000137ACAFF330A2A01638E071AB3094701A4
:10A8E0006318F60E93070B0163C6F91A03A78400D9
:10A8F00083A7C4001306C9FF138A84002326F70028
:10A9000023A4E70013074002636CC70A93063001D3
:10A9100093070A0063F2C6028327040023A4F4000D
:10A920008327440023A6F4009307B00163ECC70417
:10A9300013048400938704010327040023A0E70085
:10A940000327440023A2E7000327840023A4E70091
:10A95000B3876401B3896941177700002322F71A8E
:10A9600093E9190023A2370183A7440093F7170046
:10A97000B3E9670123A2340113850A00EFB08F9079
:10A980006FF09FE18327840023A8F4008327C4008D
:10A9900023AAF4006308E6001304040193878401EA
:10A9A0006FF09FF9832704011304840123ACF400A2
:10A9B0000327C4FF9387040223AEE4006FF0DFF7A0
:10A9C0009305040013050A00EFF0DFC86FF05FF88D
:10A9D00063C2690D03A7C70083A787001306C9FFD9
:10A9E0001385840023A6E7002324F70003A784002F
:10A9F00083A7C4002326F70023A4E700930740029F
:10AA000063E4C708130730016372C7020327040019
:10AA100023A4E4000327440023A6E4001307B001A5
:10AA20006366C702130484001385040183270400AE
:10AA30002320F500832744002322F5008327840088
:10AA40002324F500938B04006FF09FE1032784001B
:10AA500023A8E4000327C40023AAE4006308F60047
:10AA600013040401138584016FF05FFC8327040144
:10AA7000138504021304840123ACF4008327C4FF6C
:10AA800023AEF4006FF09FFA93050400EFF09FBC33
:10AA90006FF05FFB634A6A0B83A7C40003A78400BF
:10AAA0001306C9FF138584002326F70023A4E700BB
:10AAB0009307400263E4C708130730016372C702BB
:10AAC0000327040023A4E4000327440023A6E40092
:10AAD0001307B0016366C7021304840013850401E1
:10AAE000832704002320F500832744002322F50058
:10AAF000832784002324F50093090A006FF09FF454
:10AB00000327840023A8E4000327C40023AAE40049
:10AB10006308F60013040401138584016FF05FFCE1
:10AB200083270401138504021304840123ACF40079
:10AB30008327C4FF23AEF4006FF09FFA930504004F
:10AB4000EFF05FB16FF05FFB13850A00EFA0CFF06D
:10AB5000130A0500E30205E28327C4FF130785FFFC
:10AB600093F7E7FFB387FB00639AE7008329C5FFEC
:10AB700093F9C9FFB38929016FF09FCE1306C9FF6E
:10AB80009307400263EEC708130730016374C708D8
:10AB9000032704002320E500032744002322E500C7
:10ABA0001307B001636AC702130784009307850087
:10ABB0008326070023A0D7008326470023A2D700BF
:10ABC0000327870023A4E7009305040013850A00E8
:10ABD000EF70DFFD6FF05FDA032784002324E500C8
:10ABE0000327C4002326E5006308F60013070401C9
:10ABF000930705016FF0DFFB83270401130784012E
:10AC00002328F5008326440193078501232AD500D4
:10AC10006FF01FFA93070500130704006FF05FF948
:10AC200093050400EFF01FA36FF01FFA93090900CA
:10AC30006FF01FC3B3E9E90023A23B0103A747005C
:10AC40001367170023A2E7006FF0DFC5130101FFB0
:10AC5000232481001384050083A50500232291008D
:10AC6000232611009304050063840500EFF01FFE06
:10AC700093050400032481008320C1001385040090
:10AC800083244100130101016F705FF29777000088
:10AC90009387472783A707006382A7108327C504EC
:10ACA000130101FE232C8100232A91002328210176
:10ACB000232E110023263101130405009304000004
:10ACC00013090008639407048325040463860500C0
:10ACD00013050400EF709FED83258414638C050435
:10ACE0009304C4146388950403A9050013050400A4
:10ACF000EF70DFEB930509006FF0DFFEB385950081
:10AD000083A50500639E0500938444008325C40445
:10AD1000E39624FF13050400EF705FE96FF0DFFA9C
:10AD200083A9050013050400EF705FE8938509000F
:10AD30006FF05FFD8325440563860500130504005D
:10AD4000EF70DFE683278403638C07028327C40345
:10AD500013050400E78007008325042E63820502A3
:10AD600013050400032481018320C10183244101D0
:10AD7000032901018329C100130101026FF01FEDB6
:10AD80008320C1010324810183244101032901019E
:10AD90008329C10013010102678000006780000061
:10ADA00083278600130101FD232E31012326110282
:10ADB000232481022322910223202103232C4101F9
:10ADC000232A5101232861012326710123248101B3
:10ADD000232291012320A101930906006384071215
:10ADE000832A0600130A050013840500130B0000D4
:10ADF00013090000930B3000130C200063000908B6
:10AE0000032D84006360A90D8357C40013F707481E
:10AE1000630A070A8324040083250401B38CB44029
:10AE20008324440113871C0033072701B3849B024A
:10AE3000B3C4840363F4E4009304070093F707406A
:10AE4000638207109385040013050A00EFA0CFC0AA
:10AE5000130D0500631C05029307C0002320FA00B0
:10AE60008357C4001305F0FF93E707042316F4008B
:10AE700023A4090023A209006F00400903AB0A00C4
:10AE800003A94A00938A8A006FF05FF783250401C3
:10AE900013860C00EFF08FED8357C40093F7F7B7DC
:10AEA00093E707082316F4002328A401232A94001B
:10AEB000330D9D01B38494412320A40123249400E5
:10AEC000130D09006374A901130D09000325040083
:10AED00013060D0093050B00EFF0CFF783278400D6
:10AEE000B387A7412324F40083270400338DA701EF
:10AEF00083A789002320A4013389274123A42901A2
:10AF0000E31E09F623A20900130500008320C102F5
:10AF10000324810283244102032901028329C10100
:10AF2000032A8101832A4101032B0101832BC100E4
:10AF3000032C8100832C4100032D01001301010328
:10AF4000678000001386040013050A00EFF00FFB72
:10AF5000130D0500E31A05F48325040113050A0007
:10AF6000EF70DFC46FF05FEF83D7C500130101ED11
:10AF70002322911223202113232E3111232A511130
:10AF80002326111223248112232C4111232861111D
:10AF90002326711123248111232291112320A11131
:10AFA000232EB10F93F70708930A050013890500B4
:10AFB0009309060093840600638C070283A70501AA
:10AFC0006398070293050004EFA00FA92320A900AE
:10AFD0002328A900631A05009307C00023A0FA00E4
:10AFE000930BF0FF6F00D03293070004232AF9007F
:10AFF000130BC1042320610523240104232201042F
:10B0000013070B002328010023260100232A010037
:10B01000232C0100930B00001384090093065002B7
:10B0200083470400638407006394D70A330A3441DA
:10B0300063060A0483278104232037012322470162
:10B04000B38747012324F10483274104930670004A
:10B0500013078700938717002322F10463DEF600AD
:10B06000130601049305090013850A00EFF05FD36E
:10B07000E31A052813070B00B38B4B018347040029
:10B08000E384073093091400A30D01021304F0FFB9
:10B09000130A0000130D0000130C90001305A00507
:10B0A0001308A00203C6090093891900930606FE3F
:10B0B000E36AD50E97670000938787FE9396260074
:10B0C000B386F60083A60600B386F6006780060006
:10B0D000130414006FF0DFF4975700009387C77DC7
:10B0E0002328F10093760D026388066C9384740024
:10B0F00093F484FF83A8040083AC4400138C840081
:10B1000093761D00638E0600B3E69801638A0600FD
:10B1100093060003230ED102A30EC102136D2D006E
:10B12000137DFDBF6F00403213850A002324E10028
:10B13000EF90DFE68327450013850700232CF100FD
:10B14000EFB01FC9232AA10013850A00EF901FE565
:10B1500083278500032781002326F10083274101EF
:10B16000E38E07F28327C100E38A07F283C6070054
:10B17000E38606F2136D0D406FF05FF28346B10374
:10B18000E39E06F093060002A30DD1026FF01FF1BB
:10B19000136D1D006FF09FF003AA04009384440018
:10B1A000E35E0AEE330A4041136D4D006FF01FEF6E
:10B1B0009306B0026FF05FFD03C609009386190085
:10B1C0006312060503A404001386440063540400BC
:10B1D0001304F0FF93040600938906006FF01FEC40
:10B1E0009307A0003304F4029386160003C6F6FF0B
:10B1F0003304B400930506FDE374BCFE9389060096
:10B200006FF0DFEA130400006FF0DFFE136D0D082E
:10B210006FF0DFE893860900130A00009307A0008F
:10B22000330AFA02130606FD93861600330A460116
:10B2300003C6F6FF930506FDE372BCFE6FF01FFC2C
:10B2400003C60900930680066318D6009389190087
:10B25000136D0D206FF09FE4136D0D046FF01FE46C
:10B2600003C609009306C0066318D6009389190027
:10B27000136D0D026FF09FE2136D0D016FF01FE271
:10B2800083A60400138C4400A30D01022306D108F9
:10B2900013041000930C00009304C1086F00C01E3B
:10B2A000136D0D0193760D02638C06049384740074
:10B2B00093F484FF83A8040083AC4400138C8400BF
:10B2C00063DE0C00B3081041B33610013303904124
:10B2D000B30CD3409306D002A30DD1029306F0FF26
:10B2E0006318D45063920C589306900063EE16577F
:10B2F00093880803A307110F9304F10E6F004055C4
:10B3000093760D01138C44006388060083A8040023
:10B3100093DCF8416FF0DFFA93760D0483A8040004
:10B32000638806009398080193D808416FF05FFE88
:10B3300093760D20E38E06FC9398880193D888417C
:10B340006FF01FFD13760D0283A604009384440062
:10B35000630A060093D7FB4123A0760123A2F600DF
:10B360006FF09FCB13760D016306060023A07601D4
:10B370006FF09FCA13760D046306060023907601D2
:10B380006FF09FC993770D20E38207FE238076013B
:10B390006FF09FC8136D0D0193760D02638606044E
:10B3A0009384740093F484FF83A8040083AC440066
:10B3B000138C8400137DFDBF93060000A30D0102D2
:10B3C0001306F0FF630CC44213060D00B3E59801A9
:10B3D000137DFDF7639405426308045A13061000B9
:10B3E0006392C6426FF0DFF093760D01138C440038
:10B3F0006386060083A804006F00000193760D04A5
:10B400006388060083D80400930C00006FF09FFA55
:10B4100093760D20E38006FE83C804006FF0DFFE04
:10B42000B786FFFF83A8040093C6068397570000E2
:10B4300093874747138C4400930C0000136D2D0035
:10B44000231ED1022328F100930620006FF01FF77E
:10B45000A30D01029306F0FF2324E100138C4400A6
:10B4600083A404006308D42C130604009305000091
:10B4700013850400EFA0CFD0930C000003278100B8
:10B4800063040500330495402324910163D48C00A8
:10B49000232481008346B10363880600832781004B
:10B4A000938717002324F100937D2D0063880D00FE
:10B4B00083278100938727002324F10093774D0889
:10B4C000232EF1006396070683278100B306FA4016
:10B4D0006350D0069308000117680000130808D3D2
:10B4E00013037000032641042320070183258104F0
:10B4F000130616001305870063C0D84C2322D7001B
:10B50000B386B6002324D1042322C104930670001D
:10B510001307050063DEC600130601049305090046
:10B5200013850A00EFF0DF87631E055C13070B002D
:10B530008346B103638806041306B1032320C700C2
:10B5400013061000832641042322C700032681042A
:10B55000938616002322D104130616002324C10467
:10B560001306700013078700635ED60013060104FC
:10B570009305090013850A00EFF09F8263140558B4
:10B5800013070B0063880D041306C1032320C700B3
:10B5900013062000832641042322C70003268104CA
:10B5A000938616002322D104130626002324C10407
:10B5B0001306700013078700635ED60013060104AC
:10B5C0009305090013850A00EFF08FFD631C0552F7
:10B5D00013070B008327C101930600086396D70663
:10B5E00083278100B30DFA406350B0079308000130
:10B5F00017680000130888C21303700083264104F3
:10B6000023200701032681049386160093058700F3
:10B6100063C0B8412322B701B38DCD002324B10507
:10B620002322D1041306700013870500635ED60041
:10B63000130601049305090013850A00EFF04FF685
:10B640006312054C13070B00B38C8C4063509007BA
:10B6500013080001976D0000938D4DBC9308700096
:10B66000832641042320B701032681049386160014
:10B67000930587006346983F23229701B38CCC0043
:10B68000232491052322D10413067000138705009B
:10B69000635ED600130601049305090013850A00B2
:10B6A000EFF00FF06310054613070B0083268104AB
:10B6B00023228700232097003384860083264104B9
:10B6C0002324810413067000938616002322D104DC
:10B6D00013078700635ED600130601049305090073
:10B6E00013850A00EFF0CFEB631E054013070B0034
:10B6F00093774D00639A073A832781006354FA00D9
:10B70000138A070083278104B38B4B01638C0700E6
:10B71000130601049305090013850A00EFF04FE8B2
:10B720006312053E2322010493040C0013070B004F
:10B730006FF09F8E13850400EFB08FE913040500AE
:10B74000930C0000032781006FF01FD4136D0D01CF
:10B7500093760D02638006029384740093F484FF51
:10B7600083A8040083AC4400138C8400930610006B
:10B770006FF0DFC493760D01138C440063860600DE
:10B7800083A804006F00000193760D04638806000F
:10B7900083D80400930C00006FF05FFD93760D20BA
:10B7A000E38006FE83C804006FF0DFFE97570000B9
:10B7B0009387470F6FF0DF9293760D01138C44004F
:10B7C0006386060083A804006F00000193760D04D1
:10B7D0006388060083D80400930C00006FF05F922A
:10B7E00093760D20E38006FE83C804006FF0DFFE31
:10B7F00013060D00930610006FF05FBD13061000D6
:10B80000E382C6AE130620006384C6149306010FBC
:10B810009395DC0113F6780093D8380013060603DD
:10B82000B3E8150193DC3C00A38FC6FEB3E5980195
:10B830009384F6FF6396050293751D00638A0500E5
:10B84000930500036306B600A38FB4FE9384E6FF5E
:10B850009307010F930C0400338497406FF0DFC20D
:10B86000938604006FF0DFFA93770D40930D00008C
:10B87000130E010F2324F100138508001306A00006
:10B880009306000093850C002322E1029304FEFF3F
:10B890002320C103232E1101EF005013032E0102B8
:10B8A0008327810013050503A30FAEFE938D1D00B2
:10B8B0008328C10103274102638207068327C10051
:10B8C00083C60700639CB6059307F00F6388FD04E9
:10B8D00063960C009307900063F2170583274101DC
:10B8E0008325810123201103B384F44013860700CC
:10B8F00013850400232EE100EFB04FCF8327C10052
:10B90000930D00000327C10183C61700832801029D
:10B9100063860600938717002326F100138508002D
:10B9200093850C001306A00093060000232EE1006F
:10B93000EF008046938C0500B3E5A5009308050051
:10B940000327C101E38605F0138E04006FF0DFF2D8
:10B950009304010F8327010193F6F8009384F4FF09
:10B96000B386D70083C6060093D848002380D4004E
:10B970009396CC01B3E8160193DC4C00B3E6980132
:10B98000E39A06FC6FF0DFEC9304010FE39206EC00
:10B9900013761600E30E06EA93060003A307D10E02
:10B9A0006FF09F956302061E2306C108A30D0102D6
:10B9B000138C04006FF0DF8D93850501232217019E
:10B9C0002324B1042322C104635EC30213060104CD
:10B9D0009305090013850A0023266102232401032D
:10B9E000232211032320D102EFF08FBB631C05102B
:10B9F0000323C10203288102832841028326010216
:10BA000013050B00938606FF130705006FF09FAD2B
:10BA100013060601232217012324C1042322D10483
:10BA2000635AD302130601049305090013850A0023
:10BA30002322610223200103232E1101EFF04FB6D0
:10BA40006312050C03234102032801028328C1016C
:10BA500093050B00938D0DFF138705006FF01FBA40
:10BA600013060601232207012324C1042322D10443
:10BA700063D6D802130601049305090013850A0052
:10BA800023201103232E0101EFF08FB1631C050663
:10BA9000832801020328C10193050B00938C0CFF3E
:10BAA000138705006FF0DFBB832781003304FA4062
:10BAB000E35480C4930C00019754000093840475F0
:10BAC000930D70008327410423209700832681046F
:10BAD0009387170063CE8C06232287003304D4009B
:10BAE000232481042322F10413077000E356F7C0D6
:10BAF000130601049305090013850A00EFF04FAA0D
:10BB0000E30C05BE8357C90093F70704639A07CC7B
:10BB10008320C1120324811213850B008324411258
:10BB2000032901128329C111032A8111832A41119A
:10BB3000032B0111832BC110032C8110832C411086
:10BB4000032D0110832DC10F130101136780000025
:10BB500093860601232297012324D1042322F10492
:10BB60001307870063DEFD00130601049305090037
:10BB700013850A00EFF0CFA2E31605F813070B00B8
:10BB8000130404FF6FF01FF483278104E38C07F68E
:10BB9000130601049305090013850A00EFF04FA076
:10BBA0006FF05FF6130101FE232C8100232A910020
:10BBB00023282101232E110023263101130905001A
:10BBC000938405001304060063080500832785039A
:10BBD00063940700EF60DFCF832784012324F40000
:10BBE0008357C40093F78700638A070883270401FB
:10BBF000638607088317C40093F9F40F93F4F40FD6
:10BC0000139727016356070A8327040103250400BD
:10BC10003305F54083274401634AF500930504008A
:10BC200013050900EF605FB06312050683278400E7
:10BC3000130515009387F7FF2324F40083270400DE
:10BC4000138717002320E400238037018327440152
:10BC5000638CA7008357C40093F71700638A070219
:10BC60009307A0006396F4029305040013050900EE
:10BC7000EF609FAB630E05006F0040019305040069
:10BC800013050900EF600FF6E30605F69304F0FFD5
:10BC90008320C101032481011385040003290101CC
:10BCA000832441018329C100130101026780000040
:10BCB00037270000B3E7E7002316F4008327440684
:10BCC00037E7FFFF1307F7FFB3F7E7002322F40678
:10BCD0006FF09FF3976700009387C72213860500D4
:10BCE0009305050003A507006FF0DFEB97670000E1
:10BCF0009387472183A70700130101FE232C8100AE
:10BD0000232A9100232E11001304050093840600BA
:10BD100083A74703639805046396070097670000AD
:10BD20009387C7C683A7070E9386040013060000F7
:10BD30009305410013050400E78007009307F0FF17
:10BD40006318F50023A004009307A0082320F40043
:10BD50008320C101032481018324410113010102D5
:10BD6000678000006396070097670000938707C20B
:10BD700083A7070E938604006FF0DFFB9767000030
:10BD80009387471893060600138605009305050060
:10BD900003A507006FF09FF59387050013080600C1
:10BDA00013870600130305006396062897580000C2
:10BDB0009388085363F6C50E370701006378E60CD5
:10BDC0001307F00F3337C70013173700B356E600D9
:10BDD000B388D80083C608003387E60093060002C4
:10BDE000B386E640638C0600B397D7003357E5006F
:10BDF0003318D600B365F7003313D5001355080187
:10BE0000B3D7A50213160801135606019356030172
:10BE100033F7A502B305F60213170701B366D7007F
:10BE20001387070063FEB600B38606011387F7FF8A
:10BE300063E8060163F6B6001387E7FFB3860601E1
:10BE4000B386B640B3F7A6021313030113530301DD
:10BE5000B3D6A6029397070133E36700B305D60272
:10BE600013850600637CB300330368001385F6FF77
:10BE7000636603016374B3001385E6FF13170701BC
:10BE80003367A700930500006F00400EB70600015E
:10BE900013070001E36CD6F2130780016FF01FF364
:10BEA000631606009306100033D8C602B7060100D9
:10BEB0006372D80C9306F00F63F406011307800039
:10BEC000B356E800B388D80083C60800B386E600FE
:10BED000130700023307D7406318070AB3870741E7
:10BEE00093051000135608019318080193D8080110
:10BEF0009356030133F7C702B3D7C70213170701DD
:10BF0000B366D7003385F8021387070063FEA600E7
:10BF1000B38606011387F7FF63E8060163F6A60000
:10BF20001387E7FFB3860601B386A640B3F7C602C0
:10BF30001313030113530301B3D6C60293970701EA
:10BF400033E36700B388D80213850600637C1301CE
:10BF5000330368001385F6FF6366030163741301FE
:10BF60001385E6FF131707013367A70013050700C2
:10BF700067800000B706000113070001E362D8F4F0
:10BF8000130780016FF0DFF33318E800B3D5D70053
:10BF90003313E500B356D50013550801B397E700F6
:10BFA00033F7A502B3E8F6009317080193D707010A
:10BFB00013D60801B3D5A502131707013367C700CD
:10BFC000B386B70213860500637ED70033070701E7
:10BFD0001386F5FF636807016376D7001386E5FFD4
:10BFE00033070701B306D74033F7A6029398080139
:10BFF00093D80801B3D6A60213170701B385D70259
:10C00000B36717011387060063FEB700B387070104
:10C010001387F6FF63E8070163F6B7001387E6FFAF
:10C02000B3870701B387B74093150601B3E5E50071
:10C030006FF05FEB63E6D5183707010063F4E604A1
:10C040001308F00F3337D8001317370033D8E60042
:10C05000975500009385C528B385050103C80500E1
:10C06000930500023308E800B38505416396050295
:10C0700013071000E3ECF6EE3335C5001347150047
:10C080006FF0DFEEB705000113070001E3E0B6FC37
:10C09000130780016FF09FFB33570601B396B6007C
:10C0A000B366D70093DE060133D70701B378D70311
:10C0B000B397B700335805013363F800939706012F
:10C0C00093D70701135803013316B6003357D7032C
:10C0D0009398080133E80801338FE702130E070035
:10C0E000637EE8013308D800130EF7FF6368D800B9
:10C0F0006376E801130EE7FF3308D8003308E84100
:10C10000B378D8033358D80393980801B38E070344
:10C110009317030193D70701B3E7F800130708004B
:10C1200063FED701B387D7001307F8FF63E8D70092
:10C1300063F6D7011307E8FFB387D700131E0E017C
:10C14000B387D741B70E01003367EE001388FEFFB7
:10C15000337307019358070133780601135606011C
:10C16000330E03033388080393560E013303C302CF
:10C1700033030301B3866600B388C80263F4060183
:10C18000B388D80113D60601B308160163E6170376
:10C19000E39A17CFB70701009387F7FFB3F6F600CE
:10C1A00093960601337EFE003315B500B386C601B3
:10C1B00093050000E37CD5DA1307F7FF6FF09FCCFF
:10C1C00093050000130700006FF05FDA9308060084
:10C1D000138706009307050013880500639C062259
:10C1E000975600009386C60F63FCC50C3703010009
:10C1F000637E660A1303F00F6374C30013078000A5
:10C200003353E600B386660003CE06001303000234
:10C21000330EEE003303C341630C0300B395650096
:10C22000335EC501B31866003368BE00B3176500FE
:10C2300013D608013377C802139508011355050179
:10C2400093D607013358C80213170701B366D70006
:10C250003308050363FA0601B386160163E6160187
:10C2600063F40601B3861601B386064133F7C602AE
:10C270009397070193D70701B3D6C602B306D50239
:10C2800013150701B367F50063FAD700B3871701E9
:10C2900063E6170163F4D700B3871701B387D7406C
:10C2A00033D5670093050000678000003703000165
:10C2B00013070001E36666F4130780016FF05FF473
:10C2C0006316060013061000B35816033706010064
:10C2D00063F2C80A1306F00F637416011307800097
:10C2E00033D6E800B386C60003CE0600130300026F
:10C2F000330EEE003303C34163180308B3851541C1
:10C3000013D70801139508011355050113D607012A
:10C31000B3F6E502B3D5E50293960601B3E6C6008F
:10C32000B305B50263FAB600B386160163E61601DB
:10C3300063F4B600B3861601B385B640B3F6E502E2
:10C340009397070193D70701B3D5E502B305B5026B
:10C3500013950601B367F50063FAB700B3871701B9
:10C3600063E6170163F4B700B3871701B387B740DB
:10C370006FF01FF33706000113070001E3E2C8F670
:10C38000130780016FF0DFF5B398680033D7C5015C
:10C39000B3176500335EC50113D50801B376A70254
:10C3A000B3956500336EBE009395080193D50501E2
:10C3B00013560E013357A70293960601B3E6C60043
:10C3C0003387E50263FAE600B386160163E61601D9
:10C3D00063F4E600B38616013386E640B376A60220
:10C3E000131E0E01135E0E013356A602939606012C
:10C3F0003386C502B3E5C60163FAC500B3851501EE
:10C4000063E6150163F4C500B3851501B385C54026
:10C410006FF01FEFE3EAD5E83707010063FCE6049D
:10C42000930EF00F33B7DE001317370033D3E60057
:10C43000975800009388C8EAB388680083CE080044
:10C44000130E0002B38EEE00330EDE41631E0E02A9
:10C4500063E4B600636AC500B307C540B385D54041
:10C460003335F5003388A540138507009305080090
:10C470006FF09FE3B708000113070001E3E816FB24
:10C48000130780016FF09FFA3357D601B396C601A8
:10C49000B366D700B357D50133D7D501B395C501DE
:10C4A000B3E7B70093D506013373B702139F0601B4
:10C4B000135F0F0193D807013316C6013315C50169
:10C4C0003357B70213130301B36813013308EF02A4
:10C4D0001303070063FE0801B388D8001303F7FFB6
:10C4E00063E8D80063F608011303E7FFB388D800B8
:10C4F000B3880841B3FFB802B3D8B802939F0F01C5
:10C50000B3051F03139F0701135F0F0133EFEF0103
:10C5100013870800637EBF00330FDF001387F8FF27
:10C520006368DF006376BF001387E8FF330FDF0027
:10C5300013130301B70801003363E3009387F8FF87
:10C5400013580601330FBF40B375F30013530301B3
:10C55000B377F6003387F502B307F302B38505031B
:10C5600033030303B385F500135807013308B800FC
:10C570006374F80033031301B70701009387F7FFD3
:10C58000935508013378F800131808013377F70042
:10C59000B38565003307E8006366BF00631EBF0014
:10C5A000637CE5003306C7403337C700B385D54009
:10C5B000B385E540130706003307E5403335E50052
:10C5C000B305BF40B385A540B397D5013357C70125
:10C5D00033E5E700B3D5C5016FF01FCD130101FDB1
:10C5E00023248102232291022328610113040500E0
:10C5F000130B0500B704100013D5450123202103B8
:10C60000232E3101232671019384F4FF2326110286
:10C61000232C4101232A51011375F57F930B06004A
:10C6200093890600B3F4B40013D9F5016306050A33
:10C630009307F07F6306F51093943400B7068000EB
:10C64000B3E4D400935ADB01B3EA9A0013143B001D
:10C65000130A15C0130B000013D54901B7041000CD
:10C660009384F4FF1375F57FB3F43401938F0B00BB
:10C6700093D9F901630205109307F07F6302F51661
:10C68000B707800093943400B3E4F40093D7DB0140
:10C69000B3E79700939F3B00130515C013070000F5
:10C6A00093162B00B3E6E6009386F6FF9305E000B1
:10C6B000334639013305AA4063E0D516975500008B
:10C6C0009385C5B693962600B386B60083A606006A
:10C6D000B386B60067800600B3EA6401638E0A067B
:10C6E0006380040413850400EF30D049930755FF9D
:10C6F0001307C001634EF702930AD001130485FFAC
:10C70000B38AFA40B3948400B35A5B01B3EA9A0047
:10C7100033148B00130AD0C0330AAA406FF09FF382
:10C7200013050B00EF301046130505026FF01FFCD8
:10C73000930485FDB31A9B00130400006FF09FFD66
:10C74000B3EA640163820A02938A0400130AF07F49
:10C75000130B30006FF05FF013040000130A0000A9
:10C76000130B10006FF05FEF13040000130AF07F4B
:10C77000130B20006FF05FEEB3E77401638E0706C2
:10C780006380040413850400EF30D03F130755FF86
:10C790009307C00163CEE7029307D001930F85FF93
:10C7A000B387E740B394F401B3D7FB00B3E7970036
:10C7B000B39FFB011306D0C03305A6406FF01FEEF8
:10C7C00013850B00EF30103C130505026FF01FFCC2
:10C7D000930785FDB397FB00930F00006FF09FFD5B
:10C7E000B3E7740163820702938704001305F07FA7
:10C7F000130730006FF0DFEA930F0000130500000D
:10C80000130710006FF0DFE9930F00001305F07FAE
:10C81000130720006FF0DFE863E657016390FA36F4
:10C82000636EF4359395FA01935614001317F401CF
:10C8300093DA1A0033E4D5009397870013D88F0159
:10C840003368F800935E0801B3D5DA03131E0801BC
:10C85000135E0E019356040193988F00B3F4DA032C
:10C86000938F0500B307BE0293940401B3E69600CC
:10C8700063FEF600B3860601938FF5FF63E80601B9
:10C8800063F6F600938FE5FFB3860601B386F640A4
:10C8900033D3D6031314040113540401B3F6D6039F
:10C8A00093070300B3056E0293960601B366D400A6
:10C8B00063FEB600B38606019307F3FF63E8060143
:10C8C00063F6B6009307E3FFB38606013384B640F0
:10C8D000939F0F01B7050100B3EFFF001383F5FF2E
:10C8E00093D60F01B3F76F0013DF080133F368002D
:10C8F000B3836702B3846602B307FF02B382E60321
:10C90000B386970093D70301B387D70063F49700EA
:10C91000B382B20093D60701B3865600B702010076
:10C920009382F2FFB3F5570093950501B3F35300DB
:10C93000B38575006368D40093870F006314D40433
:10C940006372B70433071701B3321701B3820201D0
:10C95000330454009387FFFF6366880063148802E2
:10C96000636217036366D400639E8600637CB7002E
:10C97000330717019387EFFFB33F1701B38F0F0101
:10C980003304F401B305B7403304D4403337B70060
:10C990003304E440930FF0FF63048812B352D403CE
:10C9A00093D605013374D40313870200B30F5E02DC
:10C9B0001314040133E48600637EF401330404019C
:10C9C0001387F2FF636804016376F4011387E2FFC3
:10C9D000330404013304F441B356D40393950501A1
:10C9E00093D505013374D403330EDE02131404010E
:10C9F00033E4850093850600637EC401330404019B
:10CA00009385F6FF636804016376C4019385E6FFAE
:10CA10003304040113170701B365B7001397050129
:10CA2000135707013304C44113DE0501B30E670237
:10CA300033036E02330ECF03330FEF0213D70E0111
:10CA4000330F6F003307E70163766700B706010015
:10CA5000330EDE00135307013303C301370E010009
:10CA6000130EFEFFB376C70193960601B3FECE0107
:10CA7000B386D60163686400938F05006310640475
:10CA80006380060433048800938FF5FF6364040316
:10CA9000636664006314640263F0D802139718009D
:10CAA000B338170133880801938FE5FF330404017D
:10CAB00093080700631464006384160193EF1F005A
:10CAC0009306F53F635AD01013F77F006300070207
:10CAD00013F7FF0093054000630AB70093854F00EA
:10CAE000B3BFF501B387F701938F05001397770064
:10CAF000635A0700370700FF1307F7FFB3F7E70094
:10CB0000930605401307E07F634AD7181397D701B0
:10CB100093DF3F003367F70193D73700B705100065
:10CB20009385F5FFB3F7B700B70510809385F5FF40
:10CB300093F6F67F93964601B3F7B7008320C102C0
:10CB4000032481021316F601B3E7D700B3E6C7004A
:10CB500083244102032901028329C101032A81019F
:10CB6000832A4101032B0101832BC1001305070018
:10CB70009385060013010103678000001305F5FF8C
:10CB8000130700006FF05FCB1306090093870A00BC
:10CB9000930F040013070B00930620006300D710C7
:10CBA000930630006302D70E93061000E31AD7F005
:10CBB00093070000130700006F0040091386090067
:10CBC0006FF09FFDB7070800930F000013060000E9
:10CBD000130730006FF05FFC93051000B385D5405C
:10CBE00013078003E346B7FC1307F0016344B7065D
:10CBF0001305E5413397A700B3D6BF003395AF00C7
:10CC00003367D7003335A0003367A700B3D7B70029
:10CC100093767700638006029376F70093054000D1
:10CC2000638AB6009306470033B7E600B387E70090
:10CC3000138706009396870063CA06069396D7016A
:10CC40001357370033E7E60093D737009306000009
:10CC50006FF0DFEC130710FE3307D7401308000214
:10CC600033D7E70093060000638605011305E5430B
:10CC7000B396A70033E5F6013335A0003367A7006C
:10CC8000930700006FF0DFF8B707080013070000F4
:10CC90009306F07F130600006FF05FE89307000033
:10CCA000130700009306F07F6FF05FE79307000023
:10CCB00013070000930610006FF05FE6130101FDFB
:10CCC00023202103232A51013709100093DA45015B
:10CCD000232E3101232C41012328610123267101D8
:10CCE0001309F9FF23261102232481022322910232
:10CCF00093FAFA7F130B0500930B0600138A0600C4
:10CD00003379B90093D9F50163880A0A9307F07F54
:10CD10006386FA10370480001319390033698900DB
:10CD20001354D5013364240193143500938A1AC037
:10CD3000130B000013554A01370910001309F9FFBE
:10CD40001375F57F3379490113870B00135AFA01E4
:10CD5000630405109307F07F6304F516B70780009E
:10CD6000131939003369F90093D7DB01B3E72701C1
:10CD700013973B00130515C09306000093152B0075
:10CD8000B3E5D5003385AA009385F5FF9308E0004D
:10CD900033C649011308150063E0B81617450000B3
:10CDA0001305854C93952500B385A50083A5050043
:10CDB000B385A500678005003364A900630E0406EF
:10CDC0006300090413050900EF30C05B930755FFAA
:10CDD0001307C001634CF7021304D001930485FFCD
:10CDE0003304F4403319990033548B003364240125
:10CDF000B3149B00930AD0C0B38AAA406FF05FF3CC
:10CE0000EF304058130505026FF05FFC130485FDF9
:10CE100033148B00930400006FF0DFFD3364A9002E
:10CE2000630404029304050013040900930AF07FCD
:10CE3000130B30006FF01FF093040000930A000002
:10CE4000130B10006FF01FEF93040000930AF07FA4
:10CE5000130B20006FF01FEEB3677901638E070696
:10CE60006300090413050900EF30C051930655FF14
:10CE70009307C00163CED7029307D001130785FF44
:10CE8000B387D7403319E900B3D7FB00B3E72701D5
:10CE90003397EB009306D0C03385A6406FF0DFEDEB
:10CEA00013850B00EF30004E130505026FF01FFCD9
:10CEB000930785FDB397FB00130700006FF09FFDFC
:10CEC000B367790163820702930709001305F07FB6
:10CED000930630006FF09FEA13070000130500006F
:10CEE000930610006FF09FE9130700001305F07F11
:10CEF000930620006FF09FE8B70F0100138FFFFF2C
:10CF000093D6040113530701B3F4E4013377E70127
:10CF1000B3089302B3059702B382E602338E58003A
:10CF200093D80501B388C801B38E660263F4580034
:10CF3000B38EFE0113D90801B3F8E80193DF0701AE
:10CF4000B3F5E501B3F3E70193980801B388B8009E
:10CF5000B3877602B3859302B3849F02338EF400C5
:10CF600093D40501B384C401B386F60363F6F400D9
:10CF7000B7070100B386F60013DF0401B70901000B
:10CF8000330FDF009386F9FFB3F4D400B3F5D50077
:10CF900093570401939404013374D400B384B40010
:10CFA000B306870233099900338EE702B305830283
:10CFB0003307F3023383C50193D50601B3856500BA
:10CFC00063F4C5013307370113D30501B709010025
:10CFD000B302E3001387F9FFB3F5E500B3F6E6000B
:10CFE0003383830293950501B385D5003387770298
:10CFF00033848F02338EFF023304E400935703011E
:10D00000338487006374E400330E3E01B7070100E8
:10D010009387F7FFB376F4003373F300939606011A
:10D02000B38E2E01B3866600B3B49E00B386E601CC
:10D03000B3879600B38EBE00B3B5BE0033835700EE
:10D04000B30FB300B3B6E601B3B79700B3E7F6008A
:10D050001354040133335300B3B5BF00B3878700C3
:10D06000B365B300B387B700B387C70113D77F0198
:10D0700093979700B3E7E70013979E003367170174
:10D080003337E00093DE7E0193969F003367D7012C
:10D090003367D7009396770063DA0610935617002C
:10D0A0001377170033E7E6009396F7013367D7004D
:10D0B00093D717009305F83F635EB00E9376770021
:10D0C000638006029376F70013054000638AA6008A
:10D0D0009306470033B7E600B387E70013870600DF
:10D0E0009396770063DA0600B70600FF9386F6FF93
:10D0F000B3F7D700930508409306E07F63CEB616DA
:10D10000935637001397D7013367D70093D737006B
:10D11000B70610009386F6FFB3F7D70093F6F57FB6
:10D12000B70510809385F5FF93964601B3F7B700D6
:10D130008320C102032481021316F601B3E7D7004E
:10D14000B3E6C70083244102032901028329C101F8
:10D15000032A8101832A4101032B0101832BC10092
:10D160001305070093850600130101036780000083
:10D1700013860900930704001387040093060B002D
:10D1800093052000638AB60E93053000638CB60CBD
:10D1900093051000E390B6F2930700001307000018
:10D1A0006F00800813060A006FF09FFD130805004A
:10D1B0006FF05FF0130510003305B5409306800350
:10D1C000E3CCA6FC9306F00163C4A6061308E8416D
:10D1D000B3960701B355A70033170701B3E6B600AE
:10D1E0003337E00033E7E600B3D7A7009376770044
:10D1F000638006029376F70093054000638AB600C9
:10D200009306470033B7E600B387E70013870600AD
:10D210009396870063CA06069396D7011357370083
:10D2200033E7E60093D73700930500006FF05FEE19
:10D23000930610FEB386B64093080002B3D6D7001B
:10D2400093050000630615011308E843B395070131
:10D2500033E7E5003337E00033E7E60093070000EB
:10D260006FF0DFF8B7070800130700009305F07FA1
:10D27000130600006FF0DFE99307000013070000BA
:10D280009305F07F6FF0DFE89307000013070000BD
:10D29000930510006FF0DFE78327C50003AF05009B
:10D2A00083AF450083A2850083A5C50037870000B2
:10D2B00093D607011307F7FF13980701939E050103
:10D2C00013D6F701B3F6E60093D70501130101FF6A
:10D2D0008328050003234500032E85001358080109
:10D2E00093DE0E01B3F7E70093D5F5016390E602F4
:10D2F00033E768003367C701336707011305100080
:10D30000631A07046398D7046F008000639CE700EA
:10D310003367FF01336757003367D70113051000E8
:10D32000631A0702130510006396D7026394E8039B
:10D330006312F30363105E02631ED8016300B6023A
:10D34000639A070033E568003365C501336505015D
:10D350003335A000130101016780000013050000B0
:10D360006FF05FFF8327C50083A8C500032F05006A
:10D3700003264500032885003785000013D70701E1
:10D380001305F5FF939E080193D6080183A20500BB
:10D3900003A3450003AE85003377A70093950701EB
:10D3A000130101FF93D5050193D7F70193DE0E0119
:10D3B000B3F6A60093D8F8016310A702B36FCF00AD
:10D3C000B3EF0F01B3EFBF001305E0FF63800F0E53
:10D3D00013010101678000006398A602B3EF6200A9
:10D3E000B3EFCF01B3EFDF011305E0FFE3920FFED0
:10D3F000631207043365CF00336505013365B5005B
:10D40000133515006F00C0026314070A3365CF009F
:10D41000336505013365B50013351500639A0600C1
:10D42000B3EF6200B3EFCF01B3EFDF01638C0F0600
:10D43000631A0500638E170113051000E38A07F8CD
:10D440006F008000E39608F81305F0FF6FF05FF8B7
:10D45000E3C4E6FE635AD7001305F0FFE38A07F63C
:10D46000130510006FF0DFF6E3E8BEFC6396D5030A
:10D47000E3640EFD6314C805E360C3FC6314660037
:10D48000E3ECE2FBE36A66FC13050000E31266F4DA
:10D49000E3645FFC6FF0DFF3E3E0D5FD130500000C
:10D4A0006FF01FF3E31C05FE6FF01FF9E388E6F24F
:10D4B00013050000E38606F66FF0DFF7E36EC8F9A8
:10D4C0006FF0DFFD8327C50083A8C500032F05008B
:10D4D00003264500032885003785000013D7070180
:10D4E0001305F5FF939E080193D6080183A205005A
:10D4F00003A3450003AE85003377A700939507018A
:10D50000130101FF93D5050193D7F70193DE0E01B7
:10D51000B3F6A60093D8F8016310A702B36FCF004B
:10D52000B3EF0F01B3EFBF001305200063800F0EB0
:10D5300013010101678000006398A602B3EF620047
:10D54000B3EFCF01B3EFDF0113052000E3920FFE2D
:10D55000631207043365CF00336505013365B500F9
:10D56000133515006F00C0026314070A3365CF003E
:10D57000336505013365B50013351500639A060060
:10D58000B3EF6200B3EFCF01B3EFDF01638C0F069F
:10D59000631A0500638E170113051000E38A07F86C
:10D5A0006F008000E39608F81305F0FF6FF05FF856
:10D5B000E3C4E6FE635AD7001305F0FFE38A07F6DB
:10D5C000130510006FF0DFF6E3E8BEFC6396D503A9
:10D5D000E3640EFD6314C805E360C3FC63146600D6
:10D5E000E3ECE2FBE36A66FC13050000E31266F479
:10D5F000E3645FFC6FF0DFF3E3E0D5FD13050000AB
:10D600006FF01FF3E31C05FE6FF01FF9E388E6F2ED
:10D6100013050000E38606F66FF0DFF7E36EC8F946
:10D620006FF0DFFD130101F42326310B83A9C50040
:10D6300083A6050083A745002326A10003A5850036
:10D64000139709012328210B2324410B2322510B7B
:10D650002320610B032A0600032B4600832A860041
:10D660000329C60037860000232A910A13570701B1
:10D6700093D409011306F6FF23263107232E110A3E
:10D68000232C810A232E7109232C8109232A910935
:10D690002328A1092326B1092320D1062322F1063C
:10D6A0002324A1062328D102232AF102232CA1023C
:10D6B000232EE102B3F4C40093D9F901638A041262
:10D6C000638AC424B7070100B367F700232EF10271
:10D6D000130601039307C10303A7070083A6C7FF2F
:10D6E0009387C7FF1317370093D6D6013367D70048
:10D6F00023A2E700E312F6FE8327010337C5FFFFED
:10D7000013051500939737002328F102B384A40072
:10D71000930B000093170901378700001355090187
:10D7200093D707011307F7FF23262107232041077B
:10D730002322610723245107232041052322610569
:10D74000232451052326F1043375E5001359F9010B
:10D750006306051E6308E530B70A0100B3EA570106
:10D7600023265105130601049307C10403A70700EC
:10D7700083A6C7FF9387C7FF1317370093D6D60139
:10D780003367D70023A2E700E312F6FE83270104E4
:10D79000939737002320F104B7C7FFFF9387170043
:10D7A0003305F50013070000B3C729012328F10052
:10D7B000B30795002320F10293871700232EF10071
:10D7C00093972B00B3E7E7009387F7FF9306E000FA
:10D7D00063EEF62A974600009386C6AC939727001F
:10D7E000B387D70083A70700B387D70067800700F8
:10D7F00033E6D7003366A6003366E600630A0612F6
:10D80000630E070413050700EF20D037130745FF09
:10D81000935757401377F701630C07069306C0FF31
:10D82000B386D7021308000293952700130E00FF5A
:10D830003308E8409386C6FF6394C609930601083F
:10D84000B385B600832601039387F7FF3397E6007D
:10D8500023A8E5FA9306F0FF6F00800A630805002D
:10D86000EF205032130505026FF05FFA638A07005C
:10D8700013850700EF201031130505046FF01FF921
:10D8800013850600EF201030130505066FF01FF812
:10D890001306C0FF3386C702130701039306300047
:10D8A000B305C70083A5C5009386F6FF1307C7FF1E
:10D8B0002328B700E3D6F6FE9387F7FF6FF09FF9B2
:10D8C000130601033303D600B388D500B30816014D
:10D8D0000326C30003230301335606013313E30079
:10D8E0003366660023A8C8006FF0DFF413972700A3
:10D8F000130601033307E600232007009387F7FF91
:10D90000E396D7FEB7C4FFFF93841401B384A44009
:10D910006FF01FE0B3E7D700B3E7A700B3E7E70076
:10D92000930B2000E38807DE930B30006FF09FDE3F
:10D9300093040000930B10006FF0DFDD33676A0182
:10D94000336757013367F700630C0712638E0704D0
:10D9500013850700EF201023130745FF9357574007
:10D960001377F701630E07069306C0FFB386D7024D
:10D970001308000293952700130E00FF3308E840B8
:10D980009386C6FF6396C60993060108B385B60061
:10D99000832601049387F7FF3397E60023A0E5FC75
:10D9A0009306F0FF6F00C00A638A0A0013850A001D
:10D9B000EF20501D130505026FF01FFA630A0B00DC
:10D9C00013050B00EF20101C130505046FF0DFF8A2
:10D9D00013050A00EF20101B130505066FF0DFF793
:10D9E0001306C0FF3386C7021307010493063000F5
:10D9F000B305C70083A5C5009386F6FF1307C7FFCD
:10DA00002328B700E3D6F6FE9387F7FF6FF05FF9A0
:10DA1000130601043303D600B388D500B3081601FA
:10DA20000326C30003230301335606013313E30027
:10DA30003366660023A8C8006FF09FF41397270091
:10DA4000130601043307E600232007009387F7FF3E
:10DA5000E396D7FEB7C7FFFF938717013385A7402B
:10DA60006FF05FD4336A6A01B36A5A01B3EAFA000D
:10DA700013072000E38A0AD2130730006FF0DFD2C9
:10DA800013050000130710006FF01FD203270103D6
:10DA9000032E0104370501009306F5FF935F07018C
:10DAA000935A0E013377D700337EDE00B387EA0244
:10DAB0003306EE023388CF03B3850701935706017F
:10DAC000B387B700338B5F0363F40701330BAB00FD
:10DAD000032F410493D20701B3F7D7003376D60062
:10DAE00093970701B387C70093540F01337FDF007B
:10DAF0002322F1022320F106B306EF02B387E402EA
:10DB00003386EF033385C70093D70601B387A70099
:10DB1000338A9F0263F6C70037060100330ACA0042
:10DB2000370601009305F6FF33F5B70093DD0701D3
:10DB300083274103B3F6B6001315050113D9070176
:10DB4000B3F5B7003305D500B387BA02B382A2009C
:10DB5000B306BE023303C9033388670093D70601B7
:10DB6000B3870701B3882A0363F46700B388C8004A
:10DB700093D90701B3891901B70801001386F8FF8B
:10DB800033F8C700B3F6C600131808013308D800ED
:10DB90003386E503B307E903935E0601B386B40257
:10DBA000B386F600B386DE003383240363F4F60005
:10DBB0003303130193D70601832E8104B3876700D3
:10DBC000B70301002324F1029387F3FF13D40E015E
:10DBD000B3FEFE00B308E4023376F600B3F6F600B7
:10DBE00093960601B386C6003383EE02B38BDF0340
:10DBF000B387780193580301B388F80033868F0206
:10DC000063F478013306760093D70801370C0100DE
:10DC1000B387C7001306FCFF2326F102B3F7C80041
:10DC2000832881033373C3009397070193D30801BB
:10DC300033F6C800B3876700B308C603B38CC303C9
:10DC400013DD08013383CA023303930133036D00EC
:10DC5000B38B7A0263749301B38B8B01135C030162
:10DC6000B30B7C01370C0100B3025B00930CFCFF8B
:10DC700033B5A20033739301B38DAD0013130301C9
:10DC8000B3F89801338A4D01B308130133830201BD
:10DC900033380301232A61002322610633033A014A
:10DCA000330B0301B339330133380B0133E8090176
:10DCB0003335AA003305A80003288102B302DB0034
:10DCC00083298102B3B6D200330505010323C102C3
:10DCD0003308D500B382F20033353501B336D800AE
:10DCE000B3B7F200B30D6800B366D5000325C102D7
:10DCF0003383FD00B3821201B3B81201B337F300CE
:10DD0000232C510023245106B30273010323C104C1
:10DD1000338D1201B3BDAD00B3E7FD00B3BB72019B
:10DD2000B3381D01B386F6009352030133EA1B0199
:10DD300033739301B307E302338A46013387E20268
:10DD400093D80701B3866F023307D700B388E80082
:10DD5000B38F5F0263F4D800B38F8F018329C103AF
:10DD6000B70601001385F6FF13D70801B3F8A80022
:10DD70003307F701B3F7A70093DF09019398080170
:10DD8000B3F9A900B388F800338BFA03930D0700A9
:10DD9000B3073E03B38A3A0313D80701338ECF0388
:10DDA000B38ACA01B30A580163F4CA01330BDB001A
:10DDB00013D80A0133076801370B01002324E1025D
:10DDC0001307FBFF33F8EA00B3F7E7001318080165
:10DDD0003308F800B386BE02330ED90313D506010B
:10DDE000B307B402B387C701B307F500330789024D
:10DDF00063F4C7013307670113D507013307E50053
:10DE0000370B01002326E1021307FBFF33F5E70080
:10DE1000B3F6E600338EE303131505013305D50091
:10DE20003307E603B387C40293560701B387C701DC
:10DE3000B387F600B38A740263F4C701B38A6A0138
:10DE4000B7060100138EF6FFB3F6C70193DB070197
:10DE5000B3071D013377C701B3B81701330ABA01FD
:10DE600093960601B386E600330D1A01032781025B
:10DE7000B3381D01333ABA01B3870701336A1A0177
:10DE80008328810233B80701330BED000327C10259
:10DE9000B30C0B01B387A700333B1B0133B80C0154
:10DEA00033B5A7003387EC00336B0B010328C102A5
:10DEB000330CA700B38B5B01B387D700B3B6D70091
:10DEC000B30A7C01338EDA00333707013335AC00F7
:10DED0003367A700B336DE00330A6A01B3BA7A01AA
:10DEE000330AEA00B3EADA00B3065A013388CE02F5
:10DEF0002326F106338AD303135508013307C402DE
:10DF0000330747013307E500B3087402637647011E
:10DF100037050100B388A800370A0100135507012F
:10DF2000930AFAFFB3081501337557013378580186
:10DF300013150501B30A6902330505013308B3025D
:10DF4000B385B20213570801B38555013307B700F3
:10DF5000330959026374570133094901B70A0100B3
:10DF600093550701138AFAFF337848013389250155
:10DF7000B3754701939505013387E903B38505011F
:10DF8000338FEF0313580701338AF403B384340348
:10DF9000B384E401B304980063F4E401330A5A0142
:10DFA00013DB0401330B4B01370A0100130FFAFF97
:10DFB00033F8E4013377E701B384630213180801EF
:10DFC0003308E800330F66023386C20213570F018D
:10DFD000330696003306C700B3835302637496007A
:10DFE000B3834301370A0100135706019304FAFF74
:10DFF000B303770033779600337F9F001317070131
:10E000003307E70133063403338F3E03B38EDF0358
:10E01000935A0F013306D6013386CA00B304F403C2
:10E020006374D601B3844401135C0601B70C01008C
:10E03000330C9C00330EAE009384FCFF3335AE00EE
:10E04000B386160133769600B38DA600337F9F000A
:10E05000330EBE00131606013306E601B335BE00CB
:10E06000338F2D01330E0E01330DBF00B30E6D0142
:10E070002328C107333E0E01338ACE01B3B6160101
:10E08000B335BD0033B5AD0033392F0133E5A600FC
:10E090003369B900B3BE6E01333ECA0133052501B1
:10E0A000B3EECE013308EA003305D5013337E8007B
:10E0B00033057500B306E500B3337500330533034C
:10E0C0003308C80033B7E6003336C800B38686018C
:10E0D000B385C60033BC860133B6C500232A0107C9
:10E0E00033E7E30033836F02935605013366CC00B8
:10E0F000B3893203B3896900B38FF203B382360167
:10E1000063F46200B38F9F01B3F692009396060109
:10E11000B3749500B384960093D20201B385950041
:10E12000B382E2008326410103274102B382C20089
:10E13000B3B49500B3829200B38FF201B362D700FB
:10E14000032781019397D700232EF107B36257006D
:10E15000232CB106B3E7570013070106130600008E
:10E16000130540008326C700832507011306160008
:10E1700093D636019395D500B3E6B6002320D70099
:10E1800013074700E310A6FE032701068326810636
:10E19000B337F000B3E7E700232CD1040327C1060F
:10E1A000832641062328F104232EE104232AD104E7
:10E1B0009316B70063D406249397F701130701055C
:10E1C000130600001305300083260700832547004F
:10E1D0001306160093D616009395F501B3E6B60024
:10E1E0002320D70013074700E310A6FE0327C1052D
:10E1F000B337F00013571700232EE104032701055E
:10E20000B367F7002328F1040327C101B7470000D3
:10E210009387F7FFB307F7006354F0200327010546
:10E2200093767700638406049376F7001306400024
:10E23000638EC60283264105130747002328E104A5
:10E2400013374700B306D70033B7E600232AD104BB
:10E2500083268105B306D700232CD104B3B6E6008C
:10E260000327C105B386E600232ED1040327C10589
:10E270009316B70063D00602B707F0FF9387F7FF46
:10E280003377F700232EE1040327C101B7470000CD
:10E29000B307F7001307010513060000130530004C
:10E2A00083260700832547001306160093D6360001
:10E2B0009395D501B3E6B6002320D7001307470096
:10E2C000E310A6FE378700009306E7FF63CEF61241
:10E2D0000327C10513573700232EE1040327C10587
:10E2E000B70601809386F6FF2316E1063787000004
:10E2F0001307F7FFB3F7E7000327C106939707015A
:10E300008320C10B3377D700B367F70003270101E0
:10E31000B706008093C6F6FF1317F701B3F7D700CF
:10E32000B3E7E7008326C100032701050324810B1F
:10E3300023A6F60023A0E600032741058324410B12
:10E340000329010B23A2E600032781058329C10AC3
:10E35000032A810A23A4E600832A410A032B010A27
:10E36000832BC109032C8109832C4109032D010949
:10E37000832DC108138506001301010C678000007E
:10E3800023283101832701032328F1048327410334
:10E39000232AF10483278103232CF1048327C1035B
:10E3A000232EF104930720006380FB28930730009D
:10E3B000638AFB2893071000E398FBE4232E0104F3
:10E3C000232C0104232A0104232801046F00C02107
:10E3D0002328210183270104930B07002328F1043C
:10E3E00083274104232AF10483278104232CF10489
:10E3F0008327C104232EF1046FF0DFFA8327010283
:10E40000232EF1006FF05FE0232E0104232C010482
:10E41000232A0104232801049307F7FF6FF01FEC60
:10E4200093061000B387F640130740076342F71CBA
:10E4300013D6574093F6F701130700009307000027
:10E44000931527006312C702639806041305300072
:10E45000130601053305E5406354D50293064000D9
:10E460003387E6406F00400813050105B305B5008A
:10E4700083A5050013071700B3E7B7006FF05FFC33
:10E480003308B600032808009386160013064600DA
:10E49000232E06FF6FF05FFC130601083306B6005B
:10E4A000032606FD130800023308D8403316060180
:10E4B000B3E7C700130630009308010513030000FB
:10E4C0003306E6406346C302930540003387E540C8
:10E4D00013162600930501083386C5008325C10560
:10E4E000B3D6D5002328D6FC130640006F000004E5
:10E4F000338EB80003250E00032E4E0013031300C5
:10E500003355D500331E0E013365C50123A0A80085
:10E51000938848006FF01FFB9316270093050105B1
:10E52000B386D50023A0060013071700E316C7FE25
:10E5300083260105B337F000B3E7D7002328F104A1
:10E5400093F677006382060493F6F700638EE60283
:10E5500003274105938747002328F10493B7470019
:10E560003387E700B337F700232AE1040327810547
:10E570003387E700232CE1043337F7008327C105F5
:10E580003307F700232EE1048327C1051397C70043
:10E59000635E0700232E0104232C0104232A0104B7
:10E5A00023280104930710006FF05FD39307010540
:10E5B000930600009305300003A7070003A6470059
:10E5C00093861600135737001316D6013367C7001A
:10E5D00023A0E70093874700E390B6FE8327C10599
:10E5E00093D73700232EF104930700006FF01FCF5D
:10E5F00083274105032701053367F700832781053A
:10E600003367F7008327C1053367F70093070000DE
:10E61000E30607CC232E0104232C0104232A010442
:10E62000232801046FF09FCBB7870000232E01043D
:10E63000232C0104232A0104232801049387F7FFD4
:10E640006FF0DFC9B7870000232EF104232C0104EB
:10E65000232A0104232801049387F7FF23280100BC
:10E660006FF0DFC7130101FA83A785002328210576
:10E6700003A9C50083A6050003A74500232A91042A
:10E68000232CF10293040500232CF100032E060035
:10E690009317090103234600832886000325C6003B
:10E6A000232C810493D7070113141900232E21036F
:10E6B000232E11042326310523244105232251054D
:10E6C0002328D102232AE1022328D100232AE100B2
:10E6D000232EF100135414011359F90113080101F9
:10E6E0009305C10183A7050003A7C5FF9385C5FF57
:10E6F000939737001357D701B3E7E70023A2F5003C
:10E70000E312B8FE832601019317050113161500C5
:10E710009396360093D70701232A6102232C110315
:10E72000232EA10223226102232411032328D100D6
:10E730002328C1032320C1032326F1021356160107
:10E740001355F501930801021303C1028327030047
:10E750000327C3FF1303C3FF939737001357D70152
:10E76000B3E7E7002322F300E39268FE8327010268
:10E77000378700001307F7FF939737002320F10234
:10E780006310E602032E8102032741023367C701AB
:10E79000032EC1023367C7013367F7006314070014
:10E7A000134515003307C440E31825116354E030C6
:10E7B0006318061403254102832581020328C10240
:10E7C0003366B500336606013366F600631406024D
:10E7D000832741012328D10213040700232AF102D1
:10E7E00083278101232CF1028327C101232EF1020B
:10E7F0006F0080301306F7FF631E060C03274101EC
:10E80000B387F600B3B6D7003306E5002328F1023C
:10E81000B307D600B3B6D700232AF10283278101BC
:10E820003337E600B366D7003387F5003306D700E9
:10E83000B337F7000327C101B336D600B3E7D700DB
:10E840003308E800B3870701232CC102232EF1020D
:10E85000130410008327C1031397C700635E0728C2
:10E860003707F8FF1307F7FFB3F7E700232EF1028E
:10E870008327010313041400130701039397F7017F
:10E880001306000013053000832607008325470088
:10E890001306160093D616009395F501B3E6B6005D
:10E8A0002320D70013074700E310A6FE0327C10368
:10E8B000B337F00013571700232EE102032701039B
:10E8C000B367F7002328F102B78700009387F7FFAB
:10E8D0006F00007DB78700009387F7FFE30AF7EE2C
:10E8E0009307400763D2C70693071000232601024F
:10E8F00023240102232201022320F1026F00C0140D
:10E90000B78700009387F7FF6312F4028327410162
:10E910002328D102232AF10283278101232CF1022B
:10E920008327C101232EF1026F00001D8327C1023E
:10E93000B7060800B3E7D7002326F1029307400784
:10E94000E3C4E7FA13060700935656401377F6011F
:10E950009307000013060000939527006390D702E9
:10E960006314070493063000B386F64063D2E602D0
:10E9700013074000B307F7406F00C007B385B80026
:10E9800083A50500938717003366B6006FF0DFFCA0
:10E990003305B300032505001307170013034300D5
:10E9A000232EA3FE6FF09FFC93060104B386B600EE
:10E9B00083A606FE130800023308E840B39606015A
:10E9C0003366D60093063000130E0000B386F6407F
:10E9D0006346DE0293054000B387F5409396260018
:10E9E00093050104B386D5008325C10233D7E50022
:10E9F00023A0E6FE930640006F00C003B30EB300F1
:10EA000003A50E0083AE4E00130E1E003355E50025
:10EA1000B39E0E013365D5012320A30013034300E9
:10EA20006FF01FFB139727003387E80023200700B0
:10EA300093871700E398D7FE832701023336C0007F
:10EA400033E6C7002320C102832601018327010288
:10EA50000327410183258102B387F600B3B6D700AF
:10EA60002328F102832741020325C102B307F700DF
:10EA70003386D70033B7E700B337D600B367F70064
:10EA8000032781018326C101232AC102B305B700F0
:10EA90003386F50033B7E500B337F600B386A6003A
:10EAA0003367F7003387E600232CC102232EE102EF
:10EAB0006FF05FDA6300073E631604248328410188
:10EAC00003258101032EC10133E3A8003363C30191
:10EAD0003363D300631E03182328F1028327410206
:10EAE00013040600232AF10283278102232CF1025A
:10EAF0008327C102232EF1028327010313F7770036
:10EB00006304070413F7F70093064000630ED7026F
:10EB100003274103938747002328F10293B7470057
:10EB20003387E700B337F700232AE1020327810385
:10EB30003387E700232CE1023337F7008327C10333
:10EB40003307F700232EE1028327C1031397C70081
:10EB50006352070237870000130414001307F7FFFE
:10EB6000E308E47A3707F8FF1307F7FFB3F7E70086
:10EB7000232EF10293070103930600009305300052
:10EB800003A7070003A64700938616001357370014
:10EB90001316D6013367C70023A0E7009387470009
:10EBA000E390B6FE8327C103B786000013D7370072
:10EBB000232EE1029387F6FF631AF4020326410332
:10EBC00083270103B3E7C70003268103B3E7C70028
:10EBD000B3E7E700638C0700232ED102232C010248
:10EBE000232A010223280102130900008327C103FD
:10EBF000370701801307F7FF2316F100B7870000DE
:10EC00009387F7FF3374F400931704010324C100C2
:10EC10008320C105138504003374E4003364F400D9
:10EC20009317F901370900801349F9FF3374240160
:10EC30003369F400832701030324810523A62401FB
:10EC400023A0F40083274103032901058329C1047C
:10EC500023A2F40083278103032A8104832A410429
:10EC600023A4F400832441051301010667800000FA
:10EC70001303F0FF6310670683254102B386F60095
:10EC8000B3B7F6003388B8003307F800B337F7009E
:10EC9000232AE10203278102B335B800B3E7F50068
:10ECA0002328D102B306E500B385F600B3B7F5001B
:10ECB00033B7E6003367F7008327C102232CB10284
:10ECC000330EFE003307C701232EE10213040600B2
:10ECD0006FF05FB8B78600009386F6FFE30ED6DECE
:10ECE0001347F7FF9307400763D2E7049307100029
:10ECF000232E0100232C0100232A01002328F100E8
:10ED00006F00C012B78600009386F6FFE306D6DCDC
:10ED10008327C101B7060800B3E7D700232EF1000F
:10ED20009307C0F8E344F7FC3307E040935657409D
:10ED3000130500001377F70193070000939827004D
:10ED40006390D7026314070493063000B386F6403D
:10ED500063D2E60213074000B307F7406F00C00715
:10ED6000B308180183A808009387170033651501BD
:10ED70006FF0DFFC33831501032303001307170033
:10ED80009385450023AE65FE6FF09FFC930601045A
:10ED9000B386160183A606FD130E0002330EEE4065
:10EDA000B396C6013365D50093063000930E00007C
:10EDB000B386F64063C6DE0293054000B387F54094
:10EDC0009396260093050104B386D5008325C101DF
:10EDD00033D7E50023A8E6FC930640006F00C0038C
:10EDE000338F150103230F00032F4F00938E1E0056
:10EDF0003353E300331FCF013363E30123A06500E6
:10EE0000938545006FF01FFB139727003307E80039
:10EE10002320070093871700E398D7FE832701017B
:10EE20003335A00033E5A7002328A1008326010283
:10EE3000832701010327410203258101B387F600DF
:10EE4000B3B6D7002328F102832741010328C1016B
:10EE5000B307F700B385D70033B7E700B3B7D500E2
:10EE6000B367F700032781028326C102232AB10278
:10EE70003305A700B305F5003337E500B3B7F50058
:10EE8000B38606013367F700232CB1023387E6000F
:10EE90006FF09FE3378F000093051400930EFFFF80
:10EEA000B3F2D501930F100003264102032781021C
:10EEB0000325C102032E4101832881010323C101DF
:10EEC0001308010363C65F14B3651E01B3E5650053
:10EED000B3E5D5006316040A639C05002328F102FC
:10EEE000232AC102232CE102232EA1026FF0DFC0EE
:10EEF000B365E600B3E5A500B3E5F500639C050046
:10EF00002328D102232AC103232C1103232E6102BB
:10EF10006FF09FBEB387F6003306C6012328F102C7
:10EF2000B3B7D700B306F600232AD1023336C601A1
:10EF3000B3B6F600B366D600B3051701B387D500A4
:10EF400033B71501B3B6D700B366D70033076500F2
:10EF50003387E600232CF1029317C70063C607002E
:10EF6000232EE1026FF05FB9B706F8FF9386F6FF34
:10EF70003377D700232EE102130410006FF0DFB7C0
:10EF8000639E05002328F102232AC102232CE102FB
:10EF9000232EA10213840E006FF01FB63367E60024
:10EFA0003367A700B367F700639C07002328D102EB
:10EFB000232AC103232C1103232E61026FF09FFD2E
:10EFC000232EE103232C0102232A0102232801021C
:10EFD0009307C10303A7070083A6C7FF9387C7FF53
:10EFE0001317370093D6D6013367D70023A2E70063
:10EFF000E312F8FE83270103378400001304F4FFB3
:10F00000939737002328F102130900006FF0DFAE59
:10F01000B387F6003306C6012328F102B3B7D70041
:10F02000B306F600232AD1023336C601B3B6F60082
:10F03000B366D600330717013306D700B336D600C0
:10F0400033371701B366D700330765003387E6000F
:10F05000232CC102232EE10293070800930600002F
:10F060001305300003A7070003A647009386160088
:10F07000135717001316F6013367C70023A0E700E4
:10F0800093874700E390A6FE8327C10313840500FE
:10F0900093D71700232EF102B78700009387F7FF5D
:10F0A000E31CF4A4232E0102232C0102232A0102D3
:10F0B000232801026FF05FA46354E0286310060E5A
:10F0C0000325410283258102032EC1023368B50066
:10F0D0003368C8013368F800630C08EE1306F7FFC5
:10F0E0006318060883284101B387F64033B7F6005A
:10F0F0003388A84033B308013308E8402328F102DD
:10F10000232A01031307000063F6F60033071541B5
:10F11000133717000328810133676700B306B8402F
:10F120003335D800B386E640232CD10263060700AE
:10F13000B385054113B615008327C1013366A600C8
:10F1400013041000B387C7413386C740232EC10282
:10F150008327C1031397C700E350079A37070800B6
:10F160001307F7FFB3F7E700232EF1026F00407398
:10F17000B78700009387F7FF630CF7E49307400716
:10F1800063D2C7049307100023260102232401023F
:10F19000232201022320F1026F00C012B787000072
:10F1A0009387F7FF6304F4F68327C102B7060800CC
:10F1B000B3E7D7002326F10293074007E3C4E7FC37
:10F1C0001306070013575640930600001376F60106
:10F1D00093070000939527006390E70263140604E9
:10F1E000130730003307F7406352C702130740008C
:10F1F000B307F7406F00C007B385B80083A50500CB
:10F2000093871700B3E6B6006FF0DFFC3305B30059
:10F21000032505001306160013034300232EA3FE47
:10F220006FF09FFC130701043307B700032707FEA5
:10F23000130800023308C84033170701B3E6E6009D
:10F2400013073000130E00003307F7406346EE0249
:10F2500093054000B387F540131727009305010479
:10F260003387E5008325C10233D6C5002320C7FEBE
:10F27000130640006F00C003B30EB30003A50E00D9
:10F2800083AE4E00130E1E003355C500B39E0E0113
:10F290003365D5012320A300130343006FF01FFB48
:10F2A000139727003387E800232007009387170070
:10F2B000E398C7FE83270102B336D000B3E6D70038
:10F2C0002320D10283264101832501010327010266
:10F2D000832741023387E540B387F64033B6F60013
:10F2E000B3B6E500B386D740232AD1022328E10232
:10F2F0009306000063F4E50093B61700B3E6C6007A
:10F3000003278102032681013307E640B307D74074
:10F31000232CF102B335E6001306000063840600D7
:10F32000133617008327C1010327C1023366B600D5
:10F33000B387E740B387C740232EF1026FF05FE148
:10F34000630E0728631C040E0323410183288101F7
:10F35000832EC101336E1301336EDE01336EDE0086
:10F3600063160E022328F1028327410213040600CC
:10F37000232AF10283278102232CF1028327C10271
:10F38000232EF102130905006FF00FF7130EF0FFA3
:10F39000631EC70703284102B386D74033B7D7009F
:10F3A000B3056840333EB800B385E5402328D10259
:10F3B000232AB1021307000063F6D7003307034185
:10F3C00013371700032881023367C7019306000033
:10F3D000B30518413333B800B385E540232CB1029F
:10F3E00063060700B388084193B618008327C1025B
:10F3F000B3E86600B387D741B3871741232EF102E4
:10F4000013040600130905006FF09FD4B7860000AF
:10F410009386F6FFE308D6F41347F7FF93074007F8
:10F4200063D2E70493071000232E0100232C010070
:10F43000232A01002328F1006F00C012B7860000C4
:10F440009386F6FFE300D6F28327C101B7060800D2
:10F45000B3E7D700232EF1009307C0F8E344F7FC8D
:10F460003307E04093565740930800001377F701A5
:10F4700093070000139327006390D70263140704D7
:10F4800093063000B386F64063D2E60213074000CD
:10F49000B307F7406F00C00733036800032303007E
:10F4A00093871700B3E868006FF0DFFC338E6500C8
:10F4B000032E0E00130717009385450023AEC5FFEA
:10F4C0006FF09FFC93060104B386660083A606FDD9
:10F4D000930E0002B38EEE40B396D601B3E8D80087
:10F4E00093063000130F0000B386F6406346DF0238
:10F4F00093054000B387F5409396260093050104D9
:10F50000B386D5008325C10133D7E50023A8E6FCE7
:10F51000930640006F00C003B38F650003AE0F0079
:10F5200083AF4F00130F1F00335EEE00B39FDF0168
:10F53000336EFE0123A0C501938545006FF01FFBCC
:10F54000139727003307E80023200700938717004D
:10F55000E398D7FE83270101B3381001B3E8170100
:10F5600023281101832641020328010203270101F8
:10F57000832741013307E840B387F640B3B5F6006F
:10F58000B336E800B386D740232AD1022328E1020C
:10F59000930600006374E80093B61700B3E6B60064
:10F5A00003278101832581023387E540B307D740D4
:10F5B000232CF10233B8E5009305000063840600B4
:10F5C000933517008327C1020327C101B3E5050165
:10F5D000B387E740B387B7406FF05FE2B78F0000B3
:10F5E000130814009382FFFF33785800130F1000A4
:10F5F000832541020326410183288101832EC10115
:10F6000003238102032EC102634E0F1D33E8650000
:10F61000336F16013368C801336FDF013368F800B8
:10F62000336FDF006318041063120F022328F10206
:10F63000232AB102232C6102232EC103E31408D430
:10F6400013040000130900006FF00FD0631C0800C2
:10F650002328D102232AC102232C1103232ED103F4
:10F660006FF08FC93388F640B302B640B3BF0601CE
:10F67000333F5600B382F24123280103232A51026B
:10F68000930F000063F60601B38FC54093BF1F00C0
:10F69000B3836840B3EFEF01338AF341232C410376
:10F6A000B3BA78009309000063840F0093B9130084
:10F6B000338FCE41B3E95901330F3F41232EE1038C
:10F6C000931FCF0063DE0F04B386D7403386C54057
:10F6D00033B8D70033080641232A01032328D10277
:10F6E000B3B5C5001308000063F4D7001338160043
:10F6F000B3071341B365B800B336F300B387B7401F
:10F70000232CF1026384050013B71300B307DE4115
:10F710003367D7003387E740232EE1026FF09FC69F
:10F7200033685800336848013368E801E30A08F099
:10F730006FF08FBC93030103631E0F04631E080266
:10F74000232EF103232C0102232A01022328010284
:10F750009307C10303A7070083A6C7FF9387C7FFCB
:10F760001317370093D6D6013367D70023A2E700DB
:10F77000E392F3FE6FF01F882328F102232AB102DF
:10F78000232C6102232EC1031309050013840200F8
:10F790006FF08FB6631C08002328D102232AC10210
:10F7A000232C1103232ED1036FF05FFE232EF103D0
:10F7B000232C0102232A0102232801029307C103FB
:10F7C00003A7070083A6C7FF9387C7FF1317370058
:10F7D00093D6D6013367D70023A2E700E392F3FE66
:10F7E0006FF05F813388F640B302B640B3BF0601C5
:10F7F000333F5600B382F24123280103232A5102EA
:10F80000930F000063F60601B38FC54093BF1F003E
:10F81000B3836840B3EFEF01338AF341232C4103F4
:10F82000B3BA78009309000063840F0093B9130002
:10F83000338FCE41B3E95901330F3F41232EE1030A
:10F84000931FCF0063DC0F0AB386D7403386C540D1
:10F8500033B8D70033080641232A01032328D102F5
:10F86000B3B5C5001308000063F4D70013381600C1
:10F87000B3071341B365B800B336F300B387B7409D
:10F88000232CF1026384050013B71300B307DE4194
:10F890003367D7003387E740232EE10213090500C1
:10F8A0000325C10363060506EF00D02D130545FFB0
:10F8B000930600023368D502B347D50263060808F1
:10F8C0001307C0FF93952700130E00FFB386064170
:10F8D0003387E7021307C7FF6310C70B1307010441
:10F8E000B305B700032701039387F7FF3318070118
:10F8F00023A805FF9306F0FF6F00000C3368580043
:10F90000336848013368E801E30C08D26FF05FF90F
:10F910000325810363080500EF00D02613050502C7
:10F920006FF0DFF80325410363080500EF00902521
:10F93000130505046FF09FF703250103EF009024E2
:10F94000130505066FF09FF61306C0FF3386C70246
:10F950001307010393063000B305C70083A5C50054
:10F960009386F6FF1307C7FF2328B700E3D6F6FEFA
:10F970009387F7FF6FF01FF8130601033303E600C8
:10F98000B388E500B30816010326C300032303016F
:10F990003356D600331303013366660023A8C8002C
:10F9A0006FF05FF313972700130601033307E60098
:10F9B000232007009387F7FFE396D7FE634E851257
:10F9C000330485401307000213041400B347E40214
:10F9D000130500003364E40213070000634AF702D2
:10F9E0001387070063D40700130700001393270051
:10F9F000631A04049306300013070103B386F6402C
:10FA000063D6860213074000B307F7406F00C008B3
:10FA10009316270013060103B306D60083A606003B
:10FA2000130717003365D5006FF05FFB33066700DF
:10FA3000032606001304140013074700232EC7FEF5
:10FA40006FF01FFC13172700930601043387E600AD
:10FA5000032707FF13060002330686403317C7004B
:10FA60003365E50013073000930501031308000018
:10FA70003307F7406346E80293064000B387F64039
:10FA800013172700930601043387E6008326C1037A
:10FA900033D48600232887FE930630006F000004CD
:10FAA000B388650083A6080083A8480013081800DF
:10FAB000B3D68600B398C800B3E6160123A0D500DC
:10FAC000938545006FF01FFB139727001306010372
:10FAD0003307E6002320070093871700E3D6F6FEDE
:10FAE00003270103B337A00013040000B367F70036
:10FAF0002328F1026FF04F808327C1033707F8FFF7
:10FB00001307F7FF3304A440B3F7E7006FE09FE16A
:10FB1000232E0102232C0102232A010223280102A1
:10FB20006FF04F8503274500832785000326C50016
:10FB300083260500130101FE2322E1002324F100A6
:10FB4000232AE100232CF100374700009317160009
:10FB50002320D1002328D1002326C10093D61701EA
:10FB60009307E7FF1305000063D0D7029307D7017F
:10FB7000931506011356F60163DCD70037050080A4
:10FB80001345F5FF3305A60013010102678000004D
:10FB9000B707010093D50501B3E5F5009307F70614
:10FBA000B387D74013D75740232EB10093F7F701FF
:10FBB0006392070A9305300093060101131527008D
:10FBC000B385E54063DEF502930740003387E740E5
:10FBD0009306010193172700B387F60093064000B0
:10FBE00023A007001307170093874700E31AD7FEE7
:10FBF00003250101E30A06F83305A0406FF0DFF8A2
:10FC00003388A600032808009387170093864600D0
:10FC100023AE06FF6FF01FFB832605FF032307FFBC
:10FC2000B39616013353F300B3E666002328D100E0
:10FC300093061000E3C206FF1387160013050102A6
:10FC400093962600B306D500B3D7F50023A8F6FE99
:10FC50006FF01FF813051700930801021308300016
:10FC6000131525003308E8403385A8001317270033
:10FC7000930800021303010293060000B388F840C2
:10FC80003307E3006FF01FFB130101FD23229102F4
:10FC9000232611022324810223202103930405003B
:10FCA000638605141384050013D9F50163D4050098
:10FCB0003304B04013050400EF00C06C9305150534
:10FCC000B74700009387E70113D7554023288100E9
:10FCD000232A0100232C0100232E010093F5F501B6
:10FCE000B387A740638C050293062000631CD70EE0
:10FCF00093060002B386B640B356D400232ED1003B
:10FD00009306F7FF13060102131727003307E600D7
:10FD10003314B400232887FE6F004003930630009D
:10FD2000B386E6401306010293962600B306D6007A
:10FD300083A606FF13062000232ED1009306200081
:10FD40006316C700232C81009306100013060101DF
:10FD5000139726003307E6001306F0FF2320070061
:10FD60009386F6FF1307C7FFE39AC6FE0327C10178
:10FD7000B70601809386F6FF2316E100378700005F
:10FD80001307F7FFB3F7E700139707018327C100B5
:10FD90001319F9018320C102B3F7D700B3E7E700D5
:10FDA000370700801347F7FFB3F7E7000327010188
:10FDB00003248102B3E7270123A0E40003274101C4
:10FDC00023A6F4001385040023A2E4000327810185
:10FDD0000329010223A4E400832441021301010347
:10FDE00067800000130730006FF09FF1232E0100A1
:10FDF000232C0100232A010023280100930700007F
:10FE0000130900006FF09FF6935746013707100063
:10FE10001307F7FF93F7F77F130101FD3377C7004F
:10FE20009386170023248102232291021354F601A2
:10FE3000232611022328B100232AE100232E0100EA
:10FE4000232C010093F6F67F13061000930405009F
:10FE50006354D60AB7460000938606C013D5450002
:10FE6000B387D700935647001317C7013367A7001E
:10FE70009395C501232ED100232CE100232AB10044
:10FE8000232801000327C101378500001305F5FF72
:10FE90002316E1000327C100B7060180B3F7A700CE
:10FEA0009386F6FF3377D70093970701B367F70080
:10FEB000370700801347F7FFB3F7E7001314F40187
:10FEC00033E487008327010123A684008320C10235
:10FED00023A0F40083274101032481021385040039
:10FEE00023A2F4008327810123A4F4008324410288
:10FEF00013010103678000003365B700639A070EA2
:10FF0000E30205F86300070613050700EF008047CA
:10FF10009306150313D7564093F6F601638A060439
:10FF20001306C0FF3306C70213080002930701013E
:10FF3000130300FF3308D8401306C6FF9387C7FF9B
:10FF400063166608930701021306F7FF13172700CD
:10FF50003387E70083270101B396D7002328D7FE14
:10FF60006F00C003EF000042130505026FF05FFA57
:10FF70001306C0FF3306C702930601019307300042
:10FF8000B385C60083A5C5009387F7FF9386C6FF98
:10FF900023A8B600E3D6E7FE1306F7FF9307010197
:10FFA000131726003387E7009307F0FF232007008D
:10FFB0001306F6FF1307C7FFE31AF6FEB747000064
:10FFC0009387C7C0B387A7406FF0DFEB93050101AC
:10FFD000B388C50083A5C80083A80801B3D505016F
:10FFE000B398D800B3E5150123A8B7006FF0DFF48C
:10FFF000B7870000630805029317C70193D6450031
:02000004800179
:10000000B3E7D700232CF10013574700B787000050
:100010009395C5013367F700232AB1002328010017
:10002000232EE1009387F7FF6FF0DFE58325C500FE
:100030008327850003274500130101FE8326050061
:100040002324F100232CF100939705012322E100E2
:10005000232AE10093D70701139715002326B10047
:100060002320D1002328D100232EF100135717019C
:1000700093D5F501130301011306C101832706007F
:100080008326C6FF1306C6FF9397370093D6D60183
:10009000B3E7D7002322F600E312C3FE8326010153
:1000A0009307170013953600B78600009386F6FF76
:1000B000B3F7D7002328A1009306100063DCF61ADB
:1000C000B7C7FFFF938707403307F7009307E07F29
:1000D00063CEE71E6358E006032881010326C101B1
:1000E000832741019356C801131646003366D60094
:1000F00093964700B3E6A60093D7C70113184800AC
:10010000B336D000B3E70701B3E6F600232AC100F7
:100110002328D100832601018327410113F67600AD
:10012000630C061A13F6F600130540006306A61AC0
:1001300013864600B336D600B387D7009306060071
:100140006F0080199307C0FC635AF700232A01004F
:100150002328D100130700006FF0DFFB8327C101C4
:10016000B706080093080000B3E7D700232EF1007C
:100170009307D0033387E740135557409307030095
:100180001377F7019306000003A807009386160073
:1001900093874700B3E80801E318D5FE939E260035
:1001A000631A070293073000B387D74063D8E7008C
:1001B00093074000B386D7406F0080063305D60111
:1001C000032505001307170013064600232EA6FE7D
:1001D0006FF0DFFD93070102B387D70183A707FF05
:1001E000130800023308E840B3970701B3E8F800AA
:1001F00093073000130E0000B387D7406348FE0416
:1002000013064000B306D640939727001306010259
:10021000B307F6000326C1013357E60023A8E7FE23
:100220001307400093972600B307F30023A00700AD
:1002300093861600E398E6FE03270101B337100109
:10024000B367F7002328F1006FF0DFF0330FD6011A
:1002500003250F00032F4F00130E1E003355E5003A
:10026000331F0F013365E5012320A6001306460066
:100270006FF0DFF803264101832781010328C101C4
:10028000B366F600B3E60601B3E6A60063180700FE
:10029000B336D000930700006FF05FE8638A060C66
:1002A0009356C601131848001396470093D7C70109
:1002B00037074000B3E6C600B3E70701B3E7E7003E
:1002C00093F686FF1307F07F6FF05FE5930700005A
:1002D000930600001307F07F13968700635E060005
:1002E000130717001306F07F6308C708370680FF5F
:1002F0001306F6FFB3F7C7001396D70193D636005F
:10030000B366D6001306F07F93D73700631EC7008D
:10031000B3E6F6009307000063880600B7070800FD
:100320009306000093050000370610001306F6FF41
:10033000B3F7C700370610801377F77F1306F6FF71
:1003400013174701B3F7C700B3E7E700370700808B
:100350001347F7FF9395F501B3F7E70033E7B700CD
:100360001385060093050700130101026780000052
:10037000930700006FF01FF693070000930600003C
:100380006FF09FF7B7070100637AF5029307F00F4C
:10039000B3B7A70093973700130700023307F7405E
:1003A000B357F50017150000130585F3B307F500E3
:1003B00003C507003305A740678000003707000129
:1003C00093070001E36AE5FC930780016FF0DFFC0F
:1003D000130101FF2326110023248100930500004F
:1003E00013060000930600001307000093070000A7
:1003F000930890037300000013040500635A05007E
:1004000033048040EF00402E232085001304F0FFCA
:10041000130504008320C10003248100130101019E
:1004200067800000130101F8232A9106232E11068C
:1004300093840500232C8106930581001306000098
:1004400093060000130700009307000093080005BF
:100450007300000013040500635A05003304804054
:10046000EF008028232085001304F0FF138504008B
:1004700093058100EF008020130504008320C1074D
:1004800003248107832441071301010867800000CA
:10049000130101FB9305410023261104EFF09FF89F
:1004A0009307F0FF6308F500032581001355D5007D
:1004B000137515008320C104130101056780000036
:1004C000130101FF2326110023248100930600005D
:1004D00013070000930700009308E0037300000077
:1004E00013040500635A050033048040EF00C01F69
:1004F000232085001304F0FF130504008320C100AE
:10050000032481001301010167800000130101FF32
:100510002326110023248100930600001307000006
:10052000930700009308F003730000001304050014
:10053000635A050033048040EF00001B2320850030
:100540001304F0FF130504008320C100032481007D
:100550001301010167800000130101FF23229100B4
:10056000972400009384C49B83A7040023202101C7
:10057000232611002324810013090500639C07042E
:100580001305000093050000130600009306000009
:10059000130700009308600D7300000013040500AA
:1005A00063560502EF004014330480402320850089
:1005B0001305F0FF8320C100032481008324410040
:1005C0000329010013010101678000009727000043
:1005D00023A8A79403A504009305000013060000B8
:1005E0003305A900930600001307000093070000DD
:1005F0009308600D7300000013040500635A0500A2
:1006000033048040EF00400E232085001304F0FFE8
:1006100083A704001305F0FF3309F900E31C24F954
:1006200017270000232E878E138507006FF09FF891
:10063000130101FF232611002324810093060000EB
:1006400013070000930700009308000473000000E4
:1006500013040500635A050033048040EF00C0080E
:10066000232085001304F0FF130504008320C1003C
:1006700003248100130101016780000083A70500A6
:100680002310F50083A785002311F50083A705013A
:100690002322F50083A745012314F50083A78501D4
:1006A0002315F50083A7C5012316F50083A70502CE
:1006B0002317F50083A705032328F50083A7050466
:1006C0002328F50283A785032326F50283A7850443
:1006D000232AF50083A70505232EF50083A78505AA
:1006E0002322F50267800000972700009387878107
:1006F00003A50700678000004D69616F7520212107
:100700000000000058FFFEFFEC10FFFFEC10FFFFA1
:100710006CFFFEFFEC10FFFFEC10FFFFEC10FFFF83
:1007200004FFFEFFEC10FFFFEC10FFFF74FFFEFF65
:1007300094FFFEFFEC10FFFF8CFFFEFF9CFFFEFF0F
:10074000EC10FFFFF4FFFEFFFCFFFEFFFCFFFEFFCF
:10075000FCFFFEFFFCFFFEFFFCFFFEFFFCFFFEFFB9
:10076000FCFFFEFFFCFFFEFFFCFFFEFFEC10FFFFA7
:10077000EC10FFFFEC10FFFFEC10FFFFEC10FFFF91
:10078000EC10FFFFEC10FFFF7001FFFFEC10FFFF0C
:100790009000FFFFC400FFFF7001FFFF7001FFFF2B
:1007A0007001FFFFEC10FFFFEC10FFFFEC10FFFFEC
:1007B000EC10FFFF3000FFFFEC10FFFFEC10FFFF1D
:1007C000E40AFFFFEC10FFFFEC10FFFFEC10FFFF4F
:1007D000B00BFFFFEC10FFFF940EFFFFEC10FFFFCC
:1007E000EC10FFFFA8FEFEFFEC10FFFFEC10FFFF78
:1007F000EC10FFFFEC10FFFFEC10FFFFEC10FFFF11
:10080000EC10FFFFEC10FFFF7001FFFFEC10FFFF8B
:100810009000FFFFC800FFFF7001FFFF7001FFFFA6
:100820007001FFFF3800FFFFC800FFFF8000FFFFDF
:10083000EC10FFFF6400FFFFEC10FFFF780AFFFFE2
:10084000E80AFFFF780BFFFF8000FFFFEC10FFFFBF
:10085000B00BFFFF68FEFEFF980EFFFFEC10FFFFDE
:10086000EC10FFFFFC0EFFFFEC10FFFF68FEFEFF29
:100870002020202020202020202020202020202078
:100880003030303030303030303030303030303068
:10089000494E4600696E66004E414E006E616E0024
:1008A00030313233343536373839616263646566E6
:1008B00000000000303132333435363738394142A8
:1008C00043444546000000003000000000000000E6
:1008D0000000000000000000000000000000000018
:1008E0000000000000000000000000000000000008
:1008F0000080FF3F7665924A4A803F154CC99A971F
:10090000208A025260C42575326A52CE9A32CE28AD
:100910004DA7E45D3DC55D3B8B9E925A6C52CE5017
:100920008BF1283D0D65170C7581867576C9484D8C
:10093000669CF85850BC545C65CCC6910EA6AEA01F
:1009400019E3A3461E85B7EAFE981B90BBDD8DDE3A
:10095000F99DFBEB7EAA514335023701B1366C336A
:100960006FC6DF8CE980C947BA93A841F850FB25D0
:100970006BC7716BBF3CD5A6CFFF491F78C2D34070
:10098000000000000000000020F09DB5702BA8AD15
:10099000C59D69400000000000000000000000004C
:1009A0000004BFC91B8E344000000000000000009E
:1009B0000000000000000020BCBE19400000000044
:1009C000000000000000000000000000409C0C40FF
:1009D0000000000000000000000000000000000017
:1009E00000C80540000000000000000000000000FA
:1009F0000000000000A00240FFFFFEFFFCFFF8FF28
:100A0000F0FFE0FFC0FF80FF00FF00FE00FC00F8E9
:100A100000F000E000C00080000000003020FCCFAB
:100A2000C3A12381E32DDE9FCED2C804DDA6D80A60
:100A30006482CBD2EAF2D4122549E42D36344F53E6
:100A4000AECE6B253FF598F6D36B5801A687BDC097
:100A500057DAA582A6A2B53231E7D404F2E332D345
:100A600032711CD223DB32EE49905A393EA2085330
:100A7000FBFE551191FA39197A63254331C0AC3C1C
:100A80006DE2DEDB5DD0F6B37CACA0E4BC647C46FA
:100A9000D0DD553E202A2462B347D798233FA5E9ED
:100AA00039A527EA7FA82A3F5B0BF24A81A5ED18FA
:100AB000DE67BA943945AD1EB1CF943F71BFB3A97B
:100AC000897968BE2E4C5BE14DC4BE9495E6C93F62
:100AD0004D3D3D7CBA362B0DC2FDFCCE61841177B5
:100AE000CCABE43F55C1A8A44E401361C3D32B65E2
:100AF00019E25817B7D1F13F0AD7A3703D0AD7A31F
:100B0000703D0AD7A3703D0AD7A3F83FCDCCCCCC1B
:100B1000CCCCCCCCCCCCCCCCCCCCCCCCCCCCFB3F73
:100B2000204E614E20000000202D496E66696E69DE
:100B30007479200020496E66696E6974792000001E
:100B40004E614E004525640043000000504F53495C
:100B5000580000002E0000000500000019000000F1
:100B60007D00000000000000000000000000F03FD9
:100B70000000000000002440000000000000594078
:100B80000000000000408F40000000000088C340CB
:100B900000000000006AF8400000000080842E4140
:100BA00000000000D01263410000000084D797418C
:100BB0000000000065CDCD41000000205FA0024292
:100BC000000000E876483742000000A2941A6D4207
:100BD000000040E59C30A2420000901EC4BCD642FA
:100BE00000003426F56B0C430080E03779C34143A5
:100BF00000A0D8855734764300C84E676DC1AB431B
:100C0000003D9160E458E143408CB5781DAF154438
:100C100050EFE2D6E41A4B4492D54D06CFF0804413
:100C2000F64AE1C7022DB544B49DD9794378EA4428
:100C3000BC89D897B2D29C3C33A7A8D523F64939B2
:100C40003DA7F444FD0FA5329D978CCF08BA5B25D4
:100C5000436FAC642806C80A0080E03779C341437B
:100C6000176E05B5B5B89346F5F93FE9034F384D12
:100C7000321D30F94877825A3CBF737FDD4F1575BE
:100C80002464FFFFF475FFFFF475FFFF3864FFFF76
:100C9000F475FFFFF475FFFFF475FFFFD063FFFFEE
:100CA000F475FFFFF475FFFF4064FFFF6064FFFF12
:100CB000F475FFFF5864FFFF6864FFFFF475FFFFE2
:100CC000C064FFFFC864FFFFC864FFFFC864FFFF84
:100CD000C864FFFFC864FFFFC864FFFFC864FFFF6C
:100CE000C864FFFFC864FFFFF475FFFFF475FFFFE2
:100CF000F475FFFFF475FFFFF475FFFFF475FFFF58
:100D0000F475FFFF3C66FFFFF475FFFF5C65FFFFB6
:100D10009065FFFF3C66FFFF3C66FFFF3C66FFFF00
:100D2000F475FFFFF475FFFFF475FFFFF475FFFF27
:100D3000FC64FFFFF475FFFFF475FFFFEC6FFFFF2E
:100D4000F475FFFFF475FFFFF475FFFFB870FFFF48
:100D5000F475FFFF9C73FFFFF475FFFFF475FFFF51
:100D60007463FFFFF475FFFFF475FFFFF475FFFF79
:100D7000F475FFFFF475FFFFF475FFFFF475FFFFD7
:100D8000F475FFFF3C66FFFFF475FFFF5C65FFFF36
:100D90009465FFFF3C66FFFF3C66FFFF3C66FFFF7C
:100DA0000465FFFF9465FFFF4C65FFFFF475FFFFCF
:100DB0003065FFFFF475FFFF806FFFFFF06FFFFFEF
:100DC0008070FFFF4C65FFFFF475FFFFB870FFFFF9
:100DD0003463FFFFA073FFFFF475FFFFF475FFFF9F
:100DE0000474FFFFF475FFFF3463FFFF2020202011
:100DF00020202020202020202020202030303030B3
:100E00003030303030303030303030303083FFFFF1
:100E1000588BFFFF588BFFFF4483FFFF588BFFFF6A
:100E2000588BFFFF588BFFFFDC82FFFF588BFFFFC3
:100E3000588BFFFF4C83FFFF6483FFFF588BFFFF3E
:100E40005C83FFFF6C83FFFF588BFFFFC083FFFFB6
:100E5000C883FFFFC883FFFFC883FFFFC883FFFF6E
:100E6000C883FFFFC883FFFFC883FFFFC883FFFF5E
:100E7000C883FFFF588BFFFF588BFFFF588BFFFF86
:100E8000588BFFFF588BFFFF588BFFFF588BFFFFDE
:100E9000588BFFFF588BFFFF3484FFFF5484FFFF04
:100EA000588BFFFF588BFFFF588BFFFF588BFFFFBE
:100EB000588BFFFF588BFFFF588BFFFF588BFFFFAE
:100EC000588BFFFF588BFFFF4885FFFF588BFFFFB4
:100ED000588BFFFF588BFFFF0486FFFF588BFFFFE7
:100EE0000089FFFF588BFFFF588BFFFF8C82FFFFAD
:100EF000588BFFFF588BFFFF588BFFFF588BFFFF6E
:100F0000588BFFFF588BFFFF588BFFFF588BFFFF5D
:100F1000588BFFFF588BFFFF3484FFFF5884FFFF7F
:100F2000588BFFFF588BFFFF588BFFFFF483FFFFA9
:100F30005884FFFF2484FFFF588BFFFF1484FFFFBA
:100F4000588BFFFFF884FFFF4C85FFFFD485FFFF20
:100F50002484FFFF588BFFFF0486FFFF5882FFFFAA
:100F60000489FFFF588BFFFF588BFFFF6089FFFF4D
:100F7000588BFFFF5882FFFF2020202020202020B8
:100F800020202020202020203030303030303030E1
:100F900030303030303030300020202020202020F1
:100FA0002020282828282820202020202020202019
:100FB0002020202020202020208810101010101029
:100FC0001010101010101010100404040404040475
:100FD000040404101010101010104141414141410F
:100FE00001010101010101010101010101010101F1
:100FF0000101010110101010101042424242424201
:1010000002020202020202020202020202020202C0
:101010000202020210101010200000000000000068
:1010200000000000000000000000000000000000C0
:1010300000000000000000000000000000000000B0
:1010400000000000000000000000000000000000A0
:101050000000000000000000000000000000000090
:101060000000000000000000000000000000000080
:101070000000000000000000000000000000000070
:101080000000000000000000000000000000000060
:10109000000000000000000000000000E0A0FFFFD2
:1010A00008A9FFFF08A9FFFFF4A0FFFF08A9FFFFA1
:1010B00008A9FFFF08A9FFFF8CA0FFFF08A9FFFFF9
:1010C00008A9FFFFFCA0FFFF14A1FFFF08A9FFFF75
:1010D0000CA1FFFF1CA1FFFF08A9FFFF70A1FFFFEC
:1010E00078A1FFFF78A1FFFF78A1FFFF78A1FFFFA4
:1010F00078A1FFFF78A1FFFF78A1FFFF78A1FFFF94
:1011000078A1FFFF08A9FFFF08A9FFFF08A9FFFFBB
:1011100008A9FFFF08A9FFFF08A9FFFF08A9FFFF13
:1011200008A9FFFF08A9FFFFE4A1FFFF04A2FFFF3A
:1011300008A9FFFF08A9FFFF08A9FFFF08A9FFFFF3
:1011400008A9FFFF08A9FFFF08A9FFFF08A9FFFFE3
:1011500008A9FFFF08A9FFFFF8A2FFFF08A9FFFFEA
:1011600008A9FFFF08A9FFFFB4A3FFFF08A9FFFF1D
:10117000B0A6FFFF08A9FFFF08A9FFFF3CA0FFFFE3
:1011800008A9FFFF08A9FFFF08A9FFFF08A9FFFFA3
:1011900008A9FFFF08A9FFFF08A9FFFF08A9FFFF93
:1011A00008A9FFFF08A9FFFFE4A1FFFF08A2FFFFB6
:1011B00008A9FFFF08A9FFFF08A9FFFFA4A1FFFFDF
:1011C00008A2FFFFD4A1FFFF08A9FFFFC4A1FFFFF2
:1011D00008A9FFFFA8A2FFFFFCA2FFFF84A3FFFF57
:1011E000D4A1FFFF08A9FFFFB4A3FFFF08A0FFFFE2
:1011F000B4A6FFFF08A9FFFF08A9FFFF10A7FFFF84
:1012000008A9FFFF08A0FFFF202020202020202089
:10121000202020202020202030303030303030304E
:10122000303030303030303074BAFFFF88B9FFFFD3
:1012300094B9FFFF88B9FFFF60BAFFFF88B9FFFFCD
:1012400094B9FFFF74BAFFFF74BAFFFF60BAFFFFE3
:1012500094B9FFFF60B9FFFF60B9FFFF60B9FFFFFE
:101260009CB9FFFF1CBFFFFF1CBFFFFF40BFFFFF7C
:1012700010BFFFFF10BFFFFF00C0FFFF40BFFFFF19
:1012800010BFFFFF00C0FFFF10BFFFFF40BFFFFF09
:101290000CBFFFFF0CBFFFFF0CBFFFFF00C0FFFF35
:1012A00034D1FFFF34D1FFFF30D1FFFFE4D0FFFF87
:1012B000E4D0FFFFA4D3FFFF30D1FFFFE4D0FFFF56
:1012C000A4D3FFFFE4D0FFFF30D1FFFFE0D0FFFF4A
:1012D000E0D0FFFFE0D0FFFFA4D3FFFF0001020238
:1012E00003030303040404040404040405050505BE
:1012F000050505050505050505050505060606069A
:10130000060606060606060606060606060606067D
:101310000606060606060606060606060707070769
:10132000070707070707070707070707070707074D
:10133000070707070707070707070707070707073D
:10134000070707070707070707070707070707072D
:101350000707070707070707070707070808080819
:1013600008080808080808080808080808080808FD
:1013700008080808080808080808080808080808ED
:1013800008080808080808080808080808080808DD
:1013900008080808080808080808080808080808CD
:1013A00008080808080808080808080808080808BD
:1013B00008080808080808080808080808080808AD
:1013C000080808080808080808080808080808089D
:1013D00008080808080808080808080800000000AD
:1013E000000000000000F03F00000000000024406A
:1013F000000000000000504310000000000000004A
:10140000017A5200017C01011B0D02001000000056
:1014100018000000BCEDFEFF080000000000000006
:10142000100000002C000000B0EDFEFF08000000DE
:10143000000000001000000040000000A4EDFEFFCE
:101440000800000000000000100000005400000030
:1014500098EDFEFF040000000000000010000000F6
:101460006800000088EDFEFF08000000000000009A
:10147000100000007C0000007CEDFEFF0800000072
:1014800000000000100000009000000070EDFEFF62
:101490000C000000000000001C000000A400000080
:1014A00068EDFEFF3800000000440E1048880281FD
:1014B0000160C144C8440E0024000000C4000000C4
:1014C00080EDFEFF5000000000440E105092048199
:1014D000018802890364C144C848C944D2440E004B
:1014E00018000000EC000000ACEDFEFF2C00000036
:1014F00000480E1048810148C1500E001000000045
:10150000080100008CEDFEFF040000000000000058
:101510001000000000000000017A5200017C01016F
:101520001B0D020010000000180000006CA8FFFF57
:101530003404000000000000100000000000000063
:10154000017A5200017C01011B0D02001000000015
:101550001800000078ACFFFF10040000000000003D
:10156000000000004C180180B41801801C19018093
:10157000000000000000000000000000000000006B
:10158000000000000000000000000000000000005B
:10159000000000000000000000000000000000004B
:1015A000000000000000000000000000000000003B
:1015B000000000000000000000000000000000002B
:1015C000000000000000000000000000000000001B
:1015D000000000000000000000000000000000000B
:1015E00000000000000000000000000000000000FB
:1015F00000000000000000000000000000000000EB
:1016000000000000000000000100000000000000D9
:101610000E33CDAB34126DE6ECDE05000B0000009E
:1016200000000000000000000000000000000000BA
:1016300000000000000000000000000000000000AA
:10164000000000000000000000000000000000009A
:10165000000000000000000000000000000000008A
:101980000000000000000000430000000000000014
:101990000000000000000000000000000000000047
:1019A00000000000000000004300000000000000F4
:1019B0000000000000000000000000000000000027
:1019C00000000000000000004300000000000000D4
:1019D0000000000000000000000000000000000007
:1019E00000000000000000004300000000000000B4
:1019F00000000000000000000000000000000000E7
:101A00000000000000000000430000000000000093
:101A100000000000000000000000000000000000C6
:101A20000000000000000000430000000000000073
:101A300000000000000000000000000000000000A6
:101A40000000000000000000430000000000000053
:101A50000000000000000000000000000000000086
:101A60000000000000000000249C00802459008039
:101A700000000000980F0180540B018000070180D6
:101A80000007018000070180000701800007018036
:101A90000007018000070180000701800007018026
:101AA000FFFFFFFFFFFFFFFFFFFFFFFFFFFF000044
:101AB00001004153434949000000000000000000BC
:101AC0000000000000000000000000000000000016
:101AD000000041534349490000000000000000009D
:101AE00000000000000000000000000000000000F6
:101AF000000000000000000000000000F41A018057
:101B0000F41A0180FC1A0180FC1A0180041B018078
:101B1000041B01800C1B01800C1B0180141B018025
:101B2000141B01801C1B01801C1B0180241B0180D5
:101B3000241B01802C1B01802C1B0180341B018085
:101B4000341B01803C1B01803C1B0180441B018035
:101B5000441B01804C1B01804C1B0180541B0180E5
:101B6000541B01805C1B01805C1B0180641B018095
:101B7000641B01806C1B01806C1B0180741B018045
:101B8000741B01807C1B01807C1B0180841B0180F5
:101B9000841B01808C1B01808C1B0180941B0180A5
:101BA000941B01809C1B01809C1B0180A41B018055
:101BB000A41B0180AC1B0180AC1B0180B41B018005
:101BC000B41B0180BC1B0180BC1B0180C41B0180B5
:101BD000C41B0180CC1B0180CC1B0180D41B018065
:101BE000D41B0180DC1B0180DC1B0180E41B018015
:101BF000E41B0180EC1B0180EC1B0180F41B0180C5
:101C0000F41B0180FC1B0180FC1B0180041C018073
:101C1000041C01800C1C01800C1C0180141C018020
:101C2000141C01801C1C01801C1C0180241C0180D0
:101C3000241C01802C1C01802C1C0180341C018080
:101C4000341C01803C1C01803C1C0180441C018030
:101C5000441C01804C1C01804C1C0180541C0180E0
:101C6000541C01805C1C01805C1C0180641C018090
:101C7000641C01806C1C01806C1C0180741C018040
:101C8000741C01807C1C01807C1C0180841C0180F0
:101C9000841C01808C1C01808C1C0180941C0180A0
:101CA000941C01809C1C01809C1C0180A41C018050
:101CB000A41C0180AC1C0180AC1C0180B41C018000
:101CC000B41C0180BC1C0180BC1C0180C41C0180B0
:101CD000C41C0180CC1C0180CC1C0180D41C018060
:101CE000D41C0180DC1C0180DC1C0180E41C018010
:101CF000E41C0180EC1C0180EC1C0180F41C0180C0
:101D0000F41C0180FC1C0180FC1C0180041D01806E
:101D1000041D01800C1D01800C1D0180141D01801B
:101D2000141D01801C1D01801C1D0180241D0180CB
:101D3000241D01802C1D01802C1D0180341D01807B
:101D4000341D01803C1D01803C1D0180441D01802B
:101D5000441D01804C1D01804C1D0180541D0180DB
:101D6000541D01805C1D01805C1D0180641D01808B
:101D7000641D01806C1D01806C1D0180741D01803B
:101D8000741D01807C1D01807C1D0180841D0180EB
:101D9000841D01808C1D01808C1D0180941D01809B
:101DA000941D01809C1D01809C1D0180A41D01804B
:101DB000A41D0180AC1D0180AC1D0180B41D0180FB
:101DC000B41D0180BC1D0180BC1D0180C41D0180AB
:101DD000C41D0180CC1D0180CC1D0180D41D01805B
:101DE000D41D0180DC1D0180DC1D0180E41D01800B
:101DF000E41D0180EC1D0180EC1D0180F41D0180BB
:101E0000F41D0180FC1D0180FC1D0180041E018069
:101E1000041E01800C1E01800C1E0180141E018016
:101E2000141E01801C1E01801C1E0180241E0180C6
:101E3000241E01802C1E01802C1E0180341E018076
:101E4000341E01803C1E01803C1E0180441E018026
:101E5000441E01804C1E01804C1E0180541E0180D6
:101E6000541E01805C1E01805C1E0180641E018086
:101E7000641E01806C1E01806C1E0180741E018036
:101E8000741E01807C1E01807C1E0180841E0180E6
:101E9000841E01808C1E01808C1E0180941E018096
:101EA000941E01809C1E01809C1E0180A41E018046
:101EB000A41E0180AC1E0180AC1E0180B41E0180F6
:101EC000B41E0180BC1E0180BC1E0180C41E0180A6
:101ED000C41E0180CC1E0180CC1E0180D41E018056
:101EE000D41E0180DC1E0180DC1E0180E41E018006
:101EF000E41E0180EC1E0180EC1E01806015018053
:0C1F000060150180FFFFFFFF00000200E1
:0400000580000090E7
:00000001FF
